:020000040800F2
:1000000000500020518D0008457B0008477B000808
:10001000517B0008577B00085D7B00080000000052
:10002000000000000000000000000000615C00080B
:10003000637B000800000000F15C0008355D0008EB
:10004000998D0008998D0008998D0008998D0008F8
:10005000998D0008998D0008998D0008998D0008E8
:10006000998D0008998D0008998D0008998D0008D8
:10007000998D0008998D0008998D0008998D0008C8
:10008000998D0008717B0008998D0008998D0008F2
:100090007D7B0008998D0008998D0008998D0008D6
:1000A000998D0008998D0008998D0008998D000898
:1000B000897B0008998D0008998D0008998D0008AA
:1000C000998D0008998D0008998D0008998D000878
:1000D000998D0008957B0008998D0008998D00087E
:1000E000A17B0008A97B0008998D00080000000092
:1000F0000000000000000000000000000000000000
:0C01000000000000000000005FF808F1A3
:1001100010B5054C237833B9044B13B10448AFF341
:1001200000800123237010BDC807002000000000DC
:10013000608F000808B5034B1BB103490348AFF3B8
:10014000008008BD00000000CC070020608F000880
:1001500010F8012B11F8013B012A28BF9A42F7D071
:10016000D01A7047034613F8012B002AFBD1181A46
:1001700001387047074A08B51368032043F010039D
:10018000136000F01BF8002007F0A0FC07F09EFBB6
:10019000002008BD00200240034A044B11681B7870
:1001A0000B441360704700BF58100020000000206F
:1001B000014B1868704700BF58100020C31E042B65
:1001C00010B5044603D99221094807F0A1F9094A5C
:1001D0002402D36804F4E06423F4E0631B041B0CE2
:1001E00043F0BF6343F400331C43D46010BD00BF31
:1001F000EC8F000800ED00E00F2A70B505460C46B4
:10020000164603D9AA211B4807F082F90F2C03D9FF
:10021000AB21184807F07CF9174BDA68C2F30222C9
:10022000C2F10703111D042B28BF042306294FF038
:10023000FF3198BF002201FA03F388BF033A24EA92
:100240000303934001FA02F226EA0206002D43EA74
:100250000603A8BF05F160454FEA0313B8BF074A7C
:10026000DBB2ABBF05F5614505F00F0585F800333E
:10027000535570BDEC8F000800ED00E014ED00E078
:10028000002803DABE21064807F042B901234209DB
:1002900000F01F0003FA00F0024B43F82200704701
:1002A000EC8F000800E100E010B50446002800F0E3
:1002B00081800368404A934215D01432934212D091
:1002C000143293420FD0143293420CD01432934222
:1002D00009D01432934206D01432934203D09A21AB
:1002E000364807F015F9636833F0100206D0B3F50D
:1002F000804F03D09B21314807F00AF9A36833F0FF
:10030000400303D09C212D4807F002F9E36833F045
:10031000800303D09D21294807F0FAF8236933F4BC
:10032000807206D0B3F5007F03D09E21234807F0EA
:10033000EFF8636933F4806206D0B3F5006F03D041
:100340009F211E4807F0E4F8A36933F0200303D08F
:10035000A0211A4807F0DCF8E36933F4405303D0D6
:10036000A121164807F0D4F814222168144B0B443D
:10037000B3FBF2F39B002364124B0A68E363D4E9F6
:1003800001300343E06822F47F520343206922F0E6
:100390003002034360690343A0690343E0690343F8
:1003A00013430B6000200123A06384F8213084F8FC
:1003B000200010BD0120FCE7080002402790000843
:1003C000F8FFFDBF000002402DE9F04117469846B6
:1003D0005A1E4FF6FE739A4204460E4604D940F266
:1003E0006F11214807F094F894F82030012B38D091
:1003F000012394F8215084F820309D424FF00200F0
:100400004FF000032AD12168A36384F82100086813
:10041000D4E90F3220F00100954008605D60636808
:10042000C1F80480102BE36A22680BBF8F608E60D6
:10043000CE60CF6053B10B6843F00E0300200B6019
:10044000136843F001031360BDE8F0810B6823F0EB
:1004500004030B600B6843F00A03EFE784F82030D5
:10046000F2E70220F0E700BF2790000890F8213063
:1004700010B5022B03D004238363012010BD036851
:100480001A6822F00E021A601A6822F001021A603D
:10049000184A93421FD0143293421ED01432934212
:1004A0001DD0143293421DD0143293421DD0143209
:1004B00093420CBF4FF480134FF080730E4A002418
:1004C0005360012380F82130436B80F820407BB1DA
:1004D00098472046D2E70123F0E71023EEE74FF4D8
:1004E0008073EBE74FF48053E8E74FF48033E5E7A0
:1004F0001846C3E7080002400000024070B404251B
:10050000C66B026C3468036895402542196832D086
:100510004D0730D51A6896065EBF1A6822F00402AD
:100520001A603E4A934219D01432934218D01432C2
:10053000934217D01432934217D01432934217D0FB
:10054000143293420CBF4FF480034FF08063344A5F
:100550005360C36A002B5ED070BC18470423F6E7D3
:100560004023F4E74FF48063F1E74FF48043EEE774
:100570004FF48023EBE702259540254235D08D07C7
:1005800033D51A68940606D41A6822F00A021A6053
:10059000012280F82120214A934219D0143293423B
:1005A00018D01432934217D01432934217D0143219
:1005B000934217D0143293420CBF4FF400134FF004
:1005C0000073174A5360002380F82030836AC1E724
:1005D0000223F6E72023F4E74FF40073F1E74FF42A
:1005E0000053EEE74FF40033EBE708259540254232
:1005F00011D009070FD5196821F00E0119600123E8
:1006000003FA02F27260836380F82130002380F8DD
:100610002030036B9EE770BC704700BF08000240AB
:100620000000024090F8203010B5012B04461AD08B
:10063000012380F8203090F82100984211D103293D
:100640000FD8DFE801F002080A0CA26200200023A4
:1006500084F8203010BDE262F8E72263F6E76263B7
:10066000F4E70120F3E70220F4E70000114AD36821
:1006700013F0100305D01049CB6943F00203CB619E
:100680001023D268500706D50B4943F00403CA690A
:1006900042F00102CA61074AD169C90708D5064874
:1006A000C16941F00401C161D16921F00101D16149
:1006B000D36070470020024060100020064B18698C
:1006C00010F0800007D0054A5A6002F188325A6063
:1006D0001869C0F3C010704700200240230167452D
:1006E000034A0020136943F080031361704700BF81
:1006F00000200240F8B50646FFF75AFD114C0746A8
:100700002546E368D80712D4E368990644BF20233E
:10071000E360EB68DA0606D4EB69DB0703D4E8682C
:1007200010F0040007D0FFF7A1FF012003E0731CC5
:10073000E7D00EB90320F8BDFFF73AFDC01BB04269
:10074000DFD9F7E7002002402DE9F84F334D1F466F
:100750002B7E0446012B0E4690465DD001232B765E
:10076000431E022B03D9B2212D4806F0D1FEB6F16B
:10077000006F06D32B4B1B88802B44D12A4B9E4203
:1007800003D9B321264806F0C3FE4CF25030FFF7E0
:10079000B1FFA0BB012C03D0022C0CBF0224042407
:1007A0004FF00009CB46DFF890A04FEA0913C3F1E0
:1007B0002001A3F1200207FA01F128FA03F3C5F89A
:1007C0001CB00B4327FA02F21343DAF810209BB255
:1007D00042F00102CAF810204CF2503026F81930CD
:1007E000FFF788FFDAF8103023F00103CAF8103061
:1007F00028B909F101095FFA89F39C42D5D8002391
:100800002B76BDE8F88F402B01D1084BB7E7202BA2
:100810000CBF074B074BB2E70220F2E76010002045
:100820005F900008E0F7FF1FFFFF0108FFFF0008CF
:10083000FF7F0008FF3F0008002002400022064B17
:10084000DA61064B1A6942F002021A6158611A69AC
:1008500042F040021A617047601000200020024000
:100860002DE9F041464D04462B7E0E46012B00F04B
:10087000858001232B76036833F0020303D0A8217F
:10088000404806F045FE2368022B1CD14CF2503044
:10089000FFF730FF20B1012000232B76BDE8F08167
:1008A000394CE86123694CF2503043F00403236172
:1008B000236943F040032361FFF71CFF236923F002
:1008C00004032361E8E7A368B3F1006F06D32F4A5E
:1008D0001288802A3DD12E4A934203D9E921294822
:1008E00006F016FE294B1A88D4E90231802A03F15A
:1008F000FF3303EB812335D1254A93428CBF00237C
:1009000001231BB9EA211F4806F002FE4CF25030C9
:10091000FFF7F0FE0028BED14FF0FF330120336017
:10092000A768DFF86480D4E9023203EB8223BB427C
:10093000B2D93846FFF782FF4CF25030FFF7DAFEAB
:10094000D8F8103023F00203C8F8103098B137609F
:10095000A2E7402A01D10F4ABEE7202A0CBF0E4A67
:100960000E4AB9E7402A01D10A4AC6E7202A0CBF3D
:10097000094A0A4AC1E707F58067D4E702208DE7F4
:10098000601000209990000800200240E0F7FF1F4F
:10099000FFFF0108FFFF0008FF7F0008FF3F00087E
:1009A0002DE9F04FA94A85B0904204468B4601924A
:1009B00013D002F5806290420FD002F5806290421F
:1009C0000BD002F58062904207D002F5806290421F
:1009D00003D0BD219E4806F09BFDDBF8002091B2BC
:1009E00011B1120C12041AB1BE21994806F090FD03
:1009F000DBF80420032A17D9A2F11101012913D928
:100A0000944822F4001181420ED000F580108242F9
:100A10000AD0A0F57020814206D08F498A4203D0C7
:100A2000BF218B4806F074FD0025A846DFF840A2E0
:100A30008A4EDBF8007037FA08F302D105B0BDE842
:100A4000F08F012202FA08F907EA0907B94540F0D8
:100A50008F80019B9C4211D081498C420ED0814BEA
:100A60009C420BD001F500618C4207D001F58061FA
:100A70008C4203D0CD21764806F04AFDDBF8041005
:100A8000122900F0CC8000F28780022900F0BA80A1
:100A900071D8002900F08D80012900F0A780FF2F78
:100AA00082BF08F1804CACF1080C4FEA8C014FF08A
:100AB0000F0C9DBF204622684FEA880162680CFA3D
:100AC00001FE22EA0E0205FA01F188BF201D114342
:100AD0000160DBF80400C3004AD5DAF8182028F0DA
:100AE000030142F00102CAF81820DAF8182001F1D7
:100AF000804102F00102039201F5803108F0030EFB
:100B0000019B039A4FEA8E0E8A680CFA0EFC9C42F7
:100B100022EA0C0C00F09480514A944200F092803A
:100B2000504B9C4200F0908002F50062944214BF4A
:100B30000422032202FA0EF242EA0C028A603268B0
:100B4000C1034CBF3A43BA433260726883034CBF5F
:100B50003A43BA437260B268C1024CBF3A43BA43E7
:100B6000B260F26883024CBF174322EA0707F760BE
:100B700008F101085DE703295ED011298FD1DBF868
:100B80000C20013A022A03D9DC21314806F0C0FCCE
:100B9000DBF80C50043582E73348814209D01BD87A
:100BA000A0F58010814204D000F5803081427FF4AE
:100BB00076AFDBF80810022903D9F721244806F0A4
:100BC000A7FCDBF80810C9B301290CBFC4F81090CA
:100BD000C4F81490082562E724488142E9D000F562
:100BE00080308142E5D0A0F58010DFE7DBF80C20F3
:100BF000013A022A03D9D521154806F089FCDBF811
:100C00000C504CE7DBF80C20013A022A03D9E3210F
:100C10000F4806F07DFCDBF80C5008353FE7DBF8A9
:100C20000C20013A022A03D9EA21094806F070FC97
:100C3000DBF80C500C3532E7002530E704252EE7B1
:100C4000002277E7012275E7022273E700080140DE
:100C5000D69000080000111000002210000401408E
:100C6000000C014000100140000021100000311074
:100C70000010024038B505460C4621B94FF4DA7130
:100C8000044806F045FCAB681C4214BF012000205C
:100C900038BD00BFD690000870B5054616460C4614
:100CA00021B94FF4EA71084806F032FC012E06D94A
:100CB00040F2D511044806F02BFC2C6170BD002ECB
:100CC000FBD12404F9E700BFD690000808B5044B17
:100CD0005969014202D0586106F096F908BD00BF7B
:100CE00000040140F0B5044687B058B302683C4B9D
:100CF0009A4203D08C213B4806F00AFC94F8293232
:100D000003F0FF0223B984F82822204607F098FD5B
:100D1000254603236E4655F8100B84F8293202F05D
:100D2000DCFC0FCD0FC62B6825463360271D97E8E6
:100D30000E0055F8100B02F0C1FC064620B102234C
:100D400084F82932012548E00146206802F0CFFCF2
:100D500030464FF0010C6168C3B2994200F10100C6
:100D600017D800221046D3B2994202F101021DD8D1
:100D70000FCD6E460FC62B68336097E80E002068D3
:100D800002F0B7FC0123054600B3022284F82922B1
:100D9000D8E704EB431282F829C082F82830D386C2
:100DA00082F82B60C2E90E661664D5E704EB4316A1
:100DB00086F828310A335B0186F8290186F82B0171
:100DC000C6F83801C6F83C01E050CCE784F82400AE
:100DD00084F82932206802F02EFF284607B0F0BDC3
:100DE000005C00400F91000890F8283210B5012BEC
:100DF00004460ED0012180F8281207F04EFE20682C
:100E000002F017FF206802F060FC002084F828023E
:100E100010BD0220FCE790F8282210B5012A0446F4
:100E20000BD0012280F8282284F82410006802F0F8
:100E3000FAFE002084F8280210BD0220FCE770B5FD
:100E4000044601F0070511F0800F4FEA451014BF6A
:100E500000F1280100F5947104EB000617BF012092
:100E60000020091986F8290004BF091986F829010C
:100E70000A614A780D70CB7002B1CD81022B04BF9C
:100E800000230B7194F82832012B09D0012320682C
:100E900084F8283202F048FC002084F8280270BD53
:100EA0000220FCE701F0070211F0800F4FEA421325
:100EB00010B5044618BF03F1280118440BBF03F511
:100EC00094710123002309190ABF091980F82930F8
:100ED00080F829310A7094F82832012B09D00123B7
:100EE000206884F8283202F079FD002084F8280276
:100EF00010BD0220FCE770B5002601F007014D018E
:100F0000441984F8281105F594710144C4F83C2172
:100F1000C4F84031C4F8446184F82961006802F0E3
:100F2000A1FE304670BD01F0070100EB4111D1F880
:100F30004401704701F0070170B54D014419C4E93F
:100F40000F230026012384F8281005F1280101440D
:100F5000666484F82930006802F084FE304670BD73
:100F60002DE9F84F0446006802F067FE02040BD535
:100F7000DFF80C94DFF80CA4DFF80CB42068B0F8AC
:100F800044301B0400F19E80206802F056FE4305A9
:100F90000FD522682046B2F8443023F480631B0446
:100FA0001B0CA2F8443007F084FC00212046FFF718
:100FB00032FF206802F041FE470408D52268B2F8EB
:100FC000443023F480431B041B0CA2F844302068F7
:100FD00002F033FE860408D52268B2F8443023F4C8
:100FE00000531B041B0CA2F84430206802F025FEBD
:100FF000C5041CD522682046B2F8403023F0040313
:101000001B041B0CA2F84030B2F8403023F0080358
:101010001B041B0CA2F8403007F06EFC2268B2F8EB
:10102000443023F480531B041B0CA2F84430206886
:1010300002F003FE000524D52068B0F8403043F0EC
:101040000803A0F84030B0F8443023F400631B04D8
:101050001B0CA0F84430B0F8403043F00403A0F873
:10106000403002F0EAFDC10408D52268B2F84430ED
:1010700023F480531B041B0CA2F84430204607F0D5
:101080002BFC206802F0D9FD82050BD52268204692
:10109000B2F8443023F400731B041B0CA2F8443054
:1010A00007F003FC206802F0C8FDC30508D52268DC
:1010B000B2F8443023F480731B041B0CA2F84430B4
:1010C000BDE8F88FB0F8441089B211F00F0640F077
:1010D000B18011F0100103882AD109EA030343F417
:1010E00000430380B0F8503094F8282003EBC2038B
:1010F00000EB4300B0F80434E26BC3F3090363640C
:101100001344E363204607F0C9FB94F82430002B16
:101110003FF434AF226C002A7FF430AF94F82430CF
:10112000216843F08003A1F84C3084F8242025E79F
:101130009BB213F4006520D0B0F8503094F8282109
:1011400004F50C7103EBC20300EB4303B3F80C345A
:10115000B4F82E21C3F30903C4F8443102F056FE5B
:1011600022682046138823F070031B051B0D43F0F3
:101170008003138007F084FB00E71F047FF5FEAEB9
:10118000038823F070031B051B0D43F080030380CD
:10119000B0F8503094F8282103EBC20300EB43036E
:1011A000B3F80C34C3F30903C4F844318BB1D4F859
:1011B0003C1171B1B4F82E2102F028FED4F83C3174
:1011C000D4F8442129461344C4F83C31204607F0A2
:1011D0005DFB2168D4F83851B1F8503001F20C4071
:1011E0009BB2BDB9C25A22F4F8421204120CC25288
:1011F000C25A4AEA020292B2C2520B8823F48043D6
:1012000023F0700383F4405343F4004343F080031E
:101210000B80B3E63E2D05D86A08EE0748BF0132C1
:101220009202E8E76A09ED0608BF02F1FF324AEAD6
:101230008222E0E730F826801FFA88F818F4004F81
:101240003CD030F82630770123F070031B051B0DCE
:1012500043F0800320F82630E11991F8343100F58D
:101260008062002B50D1B0F8503091F828510633ED
:1012700003EBC50332F81350C5F3090535B1B1F8D6
:101280002E212B46D1F83C1102F0C0FDE119D1F816
:101290004431D1F83C212B44C1F84431D1F84031DC
:1012A0002A44C1F83C211BB1D1F8380185425DD2F6
:1012B000274497F82811204607F0E8FA18F0800F25
:1012C0003FF45CAE2368204633F8262009EA020288
:1012D00042F4004223F82620B3F8502004EB4616CF
:1012E00096F82810023202EBC10203EB4203B3F876
:1012F0000024F36BC2F3090272641A44336CF26384
:10130000D3BB07F0CBFA39E691F8283130F82350F7
:10131000DB0015F4804FB0F850502B441BD0023343
:1013200032F81350C5F3090535B12B46B1F8302119
:10133000D1F83C1102F06AFDE31993F828112268F4
:1013400032F821300BEA030343F4004343F0C003B7
:1013500022F821309AE7063332F81350C5F3090515
:10136000002DE9D02B46B1F83221E1E791F82811A0
:101370002046FFF7C0FDA1E7FFF7DCFDFEE500BF5B
:101380000F8FFFFF0080FFFF8F8FFFFF38B543688F
:1013900001F007059D42044628D80B061DD5012201
:1013A0006B0103F128010344014483F82920012340
:1013B0000D708B7094F828229A4219D084F8283244
:1013C000206802F0D1FB25B904F50C71206802F009
:1013D00037FC002084F8280238BD00224B0103F5B9
:1013E00094710344014483F82921E0E70120F3E7E5
:1013F0000220F1E738B5436801F00F029A42044633
:1014000027D801F0070211F0800F4FEA421314BFF2
:1014100003F1280103F5947118444FF0000515BF3E
:10142000012300230919091914BF80F8293080F815
:1014300029318D700A7094F82832012B0BD00123CA
:10144000206884F8283202F0ABFB284684F8285242
:1014500038BD0120FCE70220FAE711F0800F1BBF26
:1014600001F0070100EB411000EB4110283008BFEC
:1014700000F5947099B21AB90273C18000207047C8
:1014800001221B0C027301814381F7E70122014B0A
:101490001A60704720000E422DE9F341044608B956
:1014A000012059E0036833B11A0704D140F26711F3
:1014B000A04806F02DF82368DB0718D423689F079F
:1014C00071D42368190700F1B98023685A0700F125
:1014D000EB80E369022B04D940F2AF21954806F076
:1014E00017F8E069002840F05D81002034E063686F
:1014F00033F4803207D0B3F5A02F04D040F26D1141
:101500008C4806F005F88C4D6B6803F00C03042B37
:1015100007D06B6803F00C03082B09D16B68DE035E
:1015200006D52B689D03C9D56368002BC6D1B7E7E4
:101530006368B3F5803F12D12B6843F480332B608E
:10154000FEF736FE06462B689803B7D4FEF730FE4A
:10155000801B6428F7D9032002B0BDE8F0819BB955
:101560002B6823F480332B602B6823F480232B60BB
:10157000FEF71EFE06462B6899039FD5FEF718FE60
:10158000801B6428F7D9E6E7B3F5A02F2B6803D1B9
:1015900043F480232B60CFE723F480332B602B6848
:1015A00023F48023CBE72369012B04D940F2A11156
:1015B000604805F0ADFF63691F2B04D94FF4D1716A
:1015C0005C4805F0A5FF5C4D6B6813F00C0F07D06D
:1015D0006B6803F00C03082B11D16B68DA030ED48F
:1015E0002B689B0703D52369012B7FF459AF2B6828
:1015F000626923F0F80343EAC2032B6061E72269C2
:101600004E4B6AB101221A60FEF7D2FD06462B68E6
:101610009F07ECD4FEF7CCFD801B0228F7D99AE790
:101620001A60FEF7C5FD06462B6898077FF549AF9F
:10163000FEF7BEFD801B0228F6D98CE7A369012BBB
:1016400004D94FF4F1713B4805F062FFA2693A4DAD
:101650003B4BDAB101221A60FEF7AAFD06466B6A1F
:101660009B070DD54FF4FA52364B1B68B3FBF2F3D0
:10167000019300BF019B5A1E0192002BF9D124E770
:10168000FEF796FD801B0228E9D964E71A60FEF791
:101690008FFD06466B6A9F077FF517AFFEF788FD43
:1016A000801B0228F6D956E7E368012B06D9052BE3
:1016B00004D040F211211F4805F02AFF1E4DEB69AE
:1016C000D80024D40127EB6943F08053EB61EB6928
:1016D00003F080530093009B1B4E3368D90518D547
:1016E000E368012B32D12B6A43F001032B62FEF732
:1016F0005FFD41F2883680462B6A9B074BD5002F51
:101700003FF4E7AEEB6923F08053EB61E1E600279D
:10171000E2E7336843F480733360FEF749FD8046A7
:101720003368DA05DCD4FEF743FDA0EB080064283B
:10173000F6D910E74791000800100240000042422D
:10174000800442425C03002000700040ABB92B6A69
:1017500041F2883823F001032B622B6A23F0040343
:101760002B62FEF725FD06462B6A9807C7D5FEF7C4
:101770001FFD801B4045F7D9EDE6052B2B6A03D1F1
:1017800043F004032B62AEE723F001032B622B6AC4
:1017900023F00403AAE7FEF70BFDA0EB0800B0421C
:1017A000AAD9D8E6404B5A681D4602F00C02082A16
:1017B00069D002283D4E57D1236A33F4803304D0D8
:1017C0004FF42E713A4805F0A3FE636A33F44022C9
:1017D00023F4802110D0B2F5801F0DD0B2F5001F88
:1017E0000AD0B1F5401F07D0B3F5601F04D040F216
:1017F000B9212F4805F08CFE00233360FEF7D8FC9A
:1018000007462B68990129D4236AB3F5803F0ED18E
:10181000A36833F4003304D040F2CF21244805F00C
:1018200077FE6B68A26823F4003313436B606A6829
:10183000D4E9083122F474120B4313436B60012383
:101840003360FEF7B5FC04462B689A013FF54DAEB8
:10185000FEF7AEFC001B0228F6D97CE6FEF7A8FCDA
:10186000C01B0228CDD976E600233360FEF7A0FC2A
:1018700004462B689B017FF538AEFEF799FC001BF0
:101880000228F6D967E601283FF466AE5868236A55
:1018900000F480329A427FF403AE636A00F4701061
:1018A000C01A18BF012057E60010024060004242F3
:1018B0004791000830B5184B87B002AC03F1100512
:1018C000224618685968083303C2AB421446F7D160
:1018D00040F201231149ADF804304B6803F00C02CB
:1018E000082A17D1C3F3834206A80244DB0312F887
:1018F000102C0CD54B680A48C3F34043504306AA4A
:10190000134413F8143CB0FBF3F007B030BD0548A6
:101910005043FAE70248F8E7788F000800100240C9
:1019200000127A0000093D002DE9F0410D46044601
:1019300010B90120BDE8F08103681E0704D14FF4FF
:101940004E716D4805F0E4FD022D04D940F23931A5
:10195000694805F0DDFD694A136803F00703AB42EF
:101960003DD32368980745D42368DA076ED4634AC9
:10197000136803F00703AB4200F29A802368604DBE
:1019800013F0040F40F0A08023681B0717D52369CC
:1019900033F480620CD023F40072B2F5A06F07D04C
:1019A000B3F5C06F04D040F2AB31534805F0B0FD41
:1019B0006B68226923F4605343EAC2036B60FFF74C
:1019C00079FF6B684F4AC3F30313D35CD8404E4B87
:1019D00018604E4B186806F079F80020AAE71368E3
:1019E00023F007032B431360136803F00703AB4294
:1019F0009FD1B6E7424E13F0040F1EBF726842F447
:101A0000E0627260190742BF736843F46053736009
:101A1000A36833F0800212D023F02002902A0ED067
:101A200023F04002A02A0AD023F01002C02A06D0D8
:101A3000F02B04D040F25F312F4805F069FD736848
:101A4000A26823F0F003134373608DE76368022BF1
:101A500004D940F26631284805F05AFD6268284EE4
:101A6000012A33681CD113F4003F3FF462AF73685E
:101A700041F2883823F0030313437360FEF798FBA9
:101A800007467368626803F00C03B3EB820F3FF400
:101A90006EAFFEF78DFBC01B4045F2D9032049E72E
:101AA000022A02D113F0007FDFE713F0020FDCE718
:101AB000136823F007032B431360136803F0070335
:101AC000AB427FF436AF59E7E36833F480620CD061
:101AD00023F40072B2F5A06F07D0B3F5C06F04D045
:101AE0004FF46971044805F013FD6B68E26823F454
:101AF000E06313436B6047E7479100080020024012
:101B000000100240284001085C030020040000206F
:101B1000044B054A5B68C3F30223D35C034A106895
:101B2000D840704700100240384001085C03002094
:101B3000044B054A5B68C3F3C223D35C034A1068B5
:101B4000D840704700100240384001085C03002074
:101B500038B50D46044620B940F22351114805F02E
:101B6000D7FC25B940F224510E4805F0D1FC0F23D3
:101B700023600D4B5A6802F0030262605A6802F05B
:101B8000F002A2605A6802F4E062E2605B68DB087F
:101B900003F4E0632361054B1B6803F007032B602C
:101BA00038BD00BF479100080010024000200240ED
:101BB00003682DE9F34113F0130F054603D16C219F
:101BC000454805F0A5FC2B68D90728D56B6833F488
:101BD000407303D07221404805F09AFC3F4CE36902
:101BE000DA0044D40127E36943F08053E361E369F9
:101BF00003F080530193019B394E3368DB0538D5E0
:101C0000236A13F4407348D1236A6A6823F440734B
:101C1000134323621FB1E36923F08053E3612B6810
:101C20009B070ED5AB6833F4404303D0B9212A4853
:101C300005F06EFC294AA968536823F440430B431E
:101C40005360286810F0100024D0EB6833F4800350
:101C500004D040F21511204805F05AFC1F4AE968EB
:101C60005368002023F480030B43536012E00027E5
:101C7000C2E7336843F480733360FEF799FA804615
:101C80003368D805BCD4FEF793FAA0EB08006428AB
:101C9000F6D9032002B0BDE8F0816A6802F4407210
:101CA0009A42B1D001200F4A236A1060002023F429
:101CB000407110602162D907A6D5FEF779FA41F28A
:101CC00088380646236A9A079ED4FEF771FA801B6D
:101CD0004045F7D9DDE700BF7F91000800100240C2
:101CE000007000404004424270B50446384B86B054
:101CF00002AD03F110062A4618685968083303C27A
:101D0000B3421546F7D140F2012314F0130FADF89A
:101D1000043004D14FF4CB712E4805F0F9FB022CAE
:101D200047D0102C17D0012C4FD140F202312A4A53
:101D3000136A1940B1F5817F44D003F44073B3F5C1
:101D4000007F2DD149F64040536A13F0020F08BFBF
:101D5000002006B070BD204B5968186810F08070E4
:101D6000F7D0C1F3834206A8024412F8100CCA034C
:101D700041BF5A6806A9C2F34042521844BF12F844
:101D8000141C164A5B684CBFB2FBF1F2144A5B02AA
:101D900002FB00F0DDD403234000B0FBF3F0D8E7F2
:101DA000B3F5407F11D113684FF2244013F4003F84
:101DB000CDE7FFF7BDFE084B5B68C3F3813301330A
:101DC0005B00EAE74FF40040C3E70020C1E700BF33
:101DD000888F00087F9100080010024000127A00EE
:101DE00000093D00036830B59A69D869996995B2D0
:101DF0008CB2A54217BFD86980B280B240EA0140D8
:101E000008BF40EA024030BD0368186A5B6A9BB2B3
:101E100043EA004070470023092803D840EA031032
:101E2000C0B270470A380133C0B2F5E70A2203098D
:101E300000F00F0002FB0300C0B2704730B5172559
:101E400009234D43022900F5FA64B5FBF3F517D8D1
:101E5000043200F2CF7310194FF4C872B3FBF2F2E0
:101E6000284400EB930010446422B3FBF2F3C01A41
:101E70000723B0FBF3F3C3EBC303C01AC0B230BDFA
:101E80004FF4C873901C64222044B4FBF3F328443D
:101E900000EB9400B4FBF2F41844001BE8E738B5FB
:101EA0000446FEF785F9054623685A68920605D56B
:101EB00000205A6842F010025A6038BDFEF778F9E7
:101EC000401BB0F57A7FEFD90320F6E7026838B5FA
:101ED0005368044623F010035360FEF769F9054682
:101EE00023685B689B0601D5002038BDFEF760F9CA
:101EF000401BB0F57A7FF3D90320F6E738B50546E5
:101F00000C46FFF7CCFF58B92B68220CA4B29A619B
:101F10002846DC61FFF7DAFF003018BF012038BD2A
:101F20000120FCE738B505460C46FFF7B8FF58B965
:101F30002B68220CA4B21A6228465C62FFF7C6FF27
:101F4000003018BF012038BD0120FCE770B50D46F8
:101F50001646044600283DD000293BD0012A04D96A
:101F600040F2CA21434805F0D3FA237C012B4FF0FD
:101F700002037DD0012263742274287866BB17287F
:101F800004D940F2D3213B4805F0C2FA6B783B2BD1
:101F900004D94FF43571374805F0BAFAAB783B2BCA
:101FA00004D940F2D521334805F0B2FA3C206B78D1
:101FB0002E7858434FF4616303FB0606A878064465
:101FC00031462046FFF79AFF054698B30423637411
:101FD00000232374012549E0FFF728FF172804D9BF
:101FE00040F2DD21234805F093FA6878FFF71EFFE1
:101FF0003B2804D940F2DE211E4805F089FAA87872
:10200000FFF714FF3B2804D940F2DF21194805F0FF
:102010007FFA2878FFF70AFF06466878FFF706FF81
:102020003C2358434FF4616303FB0606A878FFF78F
:10203000FDFEC4E722682046536823F00503536081
:10204000FFF7E2FE431C0DD086420BD900F5A83104
:1020500001F5C0712046FFF765FF18B10423257410
:102060006374B7E70123637400232374284670BDAB
:102070001D46FBE7BA9100082DE9F8430D4690464E
:10208000044610B90120BDE8F8830029FAD0012ADE
:1020900004D940F22D31564805F03AFA23685B68BE
:1020A0005807EFD42046FFF79DFE4FF46162B0FB66
:1020B000F2F3074602FB13023C20B2FBF0F100FBF7
:1020C0001122172B6970AA7040F28D801821B3FB82
:1020D000F1F201FB123320462B70FFF795FE411CF5
:1020E000064604D087422CBF4FF0FF36C61B414B3B
:1020F0002046B7FBF3F903FB19794946FFF7FEFECB
:102100000028BFD1721C2ED009EB06012046FFF734
:1021100009FF0028B6D1374B0026B7FBF3F74FF085
:10212000640C4FF4C87E40F2D529E07B617BA27B32
:10213000B7421AD8C9B2D2B2E0736173A273FFF783
:102140007DFE2073B8F1000F0BD02878FFF763FEF7
:1021500028706878FFF75FFE6870A878FFF75BFE6D
:10216000A87000208FE73146D0E74B1E092B0ED810
:1021700029FA03F3DB0738D421F00203042B01D042
:10218000092B0DD11D2A0FD90131012206E00C299E
:10219000F2D11E2A08D90122114601300136C7E7C3
:1021A0000229FBD11B2A01D80132F7E71C2A13D1DF
:1021B00082B2930712D1B2FBFCF30CFB13239BB248
:1021C0007BB9B2FBFEF30EFB13239BB2002B0EBFB9
:1021D0001D2201220321E1E71D2ADFD10122032173
:1021E000DCE71D22DAE72B70ACE71E2ACBE700BF45
:1021F000BA9100088051010070B50D46164604469C
:1022000000284FD000294DD0012A04D94FF467711E
:10221000484805F07DF9237C0220012B00F08980DD
:10222000012360742374E878002E3DD1632804D91B
:1022300040F2A5313F4805F06BF96B78013B0B2B61
:1022400004D940F2A6313B4805F062F9AB78013B76
:102250001E2B04D940F2A731364805F059F9EB7826
:10226000E3736B786373AB78A373A27B617BE07BD2
:10227000FFF7E4FD207328702046FFF7B3FD2E4BD7
:10228000984252D9A3F60F63B0FBF3F503FB150593
:1022900020462946FFF732FE064698B304236374AE
:1022A00000232374012044E0FFF7C0FD632804D914
:1022B0004FF46C711F4805F02BF96878FFF7B6FDF5
:1022C0000138C0B20B2804D940F2B131194805F0E9
:1022D0001FF9A878FFF7AAFD0138C0B21E2804D95B
:1022E00040F2B231134805F013F9E878FFF79EFD8C
:1022F000E0736878FFF79AFD6073A878FFF796FDA2
:10230000A073B2E72046FFF77FFD431C0DD0854246
:102310000BD900F5A83101F5C0712046FFF702FE88
:1023200018B1042326746374BCE70123002063748E
:10233000207470BDBA9100088F5F01000023F7B5CB
:102340000C461746ADF804308DF80630054618B92E
:102350000122104603B0F0BD0029F9D0012A04D9AA
:1023600040F20E41104805F0D3F8002201A928469A
:10237000FFF782FE02460028EAD12B7B2370E87B20
:10238000E0706E7B6670A97BA170002FE1D0FFF733
:1023900042FDE0703046FFF73EFD60700846FFF7F3
:1023A0003AFDA070D5E700BFBA910008F8B50D4618
:1023B00017461C460646A8B3A1B3012B04D940F228
:1023C00017511A4805F0A4F827B14FF4A361174834
:1023D00005F09EF83046FFF717FD4FF461611826AF
:1023E000B0FBF1F2B2FBF6F306FB13233C2601FB34
:1023F0001200B0FBF6F2D1B206FB1202DBB2D2B28F
:102400002B706970AA707CB11846FFF704FD287024
:102410000846FFF700FD68701046FFF7FCFCA87047
:102420000020F8BD0120FCE72046FAE7BA91000839
:10243000036810B51A680446920708D55B689B07C5
:1024400005D504F0E7FD6FF0020223685A604FF4EF
:102450000032024B5A610123637410BD0004014035
:1024600038B50446A8B10268536823F008035360E6
:10247000FDF79EFE054623685B681B0701D500201B
:1024800038BDFDF795FE401BB0F57A7FF3D90320E8
:10249000F6E70120F4E7000010B5044688B30268AF
:1024A000354B9A4204D040F21D11344805F030F803
:1024B000A36833F0800209D023F40073B3F5807F62
:1024C00004D04FF48F712D4805F022F863682C4A30
:1024D000A3F58013934204D840F21F11274805F05A
:1024E00017F8637C03F0FF021BB92274204605F045
:1024F00015FA022320466374FFF7B2FF18B10423D4
:102500006374012037E02046FFF7C9FC0028F6D1AC
:102510002268A068536823F007035360194A18B172
:10252000116B21F001011163D36A23F4607303433B
:10253000D3626068431C05D10120FFF7D5FB00285A
:10254000DDD001382268936823F00F0343EA10437B
:102550009360D36880B21B0C1B041843D0602046E4
:10256000FFF7B4FC012310B104226274C9E7E073E1
:102570006373A373637410BD00280040BA91000810
:10258000FEFFEFFF006C00400A2938B50C461546E7
:1025900004D94FF4F171054804F0BAFFA10001F12C
:1025A000804101F5D841ADB20D6038BDF29100080F
:1025B0000A2910B50C4604D94FF4FE71054804F001
:1025C000A7FFA10001F1804101F5D841086880B260
:1025D00010BD00BFF2910008036A2DE9F04123F01D
:1025E00001030362046AD0F8048086690B6826F050
:1025F00073061E438B6824F002041C431A4B0546E5
:1026000098420F4627D1CB6833F0080304D041F23B
:102610000171164804F07CFFFB6824F008041C4399
:10262000BB6924F0040433F4007304D041F20E714A
:102630000E4804F06DFF7B6933F4807304D041F2DF
:102640000F710A4804F064FFD7E9053228F4407896
:10265000134343EA08087B68C5F80480AE616B63E6
:102660002C62BDE8F08100BF002C01402D920008D3
:10267000036A2DE9F04123F480730362046AD0F801
:102680000480C6690B6826F073061E438B6824F429
:10269000007444EA03241B4B054698420F4628D198
:1026A000CB6833F0080304D041F29771164804F068
:1026B0002FFFFB6824F4006444EA0324BB6924F47C
:1026C000806433F4007304D041F2A4710E4804F026
:1026D0001FFF7B6933F4807304D041F2A5710A486F
:1026E00004F016FFD7E9053228F44058134348EAAE
:1026F00003187B68C5F80480EE61EB632C62BDE8CB
:10270000F08100BF002C01402D920008036A2DE9E2
:10271000F04123F480530362056AD0F80480C7694E
:102720000B6827F4E64747EA03278B6825F4005532
:1027300045EA03350D4B044698420E460DD14B69D0
:1027400033F4807304D041F2E371094804F0E0FEF1
:10275000736928F4804848EA83187368C4F80480D1
:10276000E76123642562BDE8F08100BF002C0140D1
:102770002D9200080368134A10B5934204460FD007
:10278000B3F1804F0CD0A2F59432934208D002F5F9
:102790008062934204D040F285110B4804F0B8FEE9
:1027A000022384F83D30236800209A6802F0070273
:1027B000062A1EBF1A6842F001021A60012384F83B
:1027C0003D3010BD002C01402D9200080368124AD4
:1027D00010B5934204460FD0B3F1804F0CD0A2F550
:1027E0009432934208D002F58062934204D040F2C2
:1027F000B9110A4804F08CFE23680020DA6842F020
:102800000102DA609A6802F00702062A1EBF1A68FF
:1028100042F001021A6010BD002C01402D92000808
:1028200070477047704770477047036810B51A6962
:10283000044691070ED5DA6892070BD56FF00202B5
:102840001A6101229B6902779B0777D0FFF7EAFFA5
:102850000023237723681A69500710D5DA685107D7
:102860000DD56FF004021A6102229B69227713F4DE
:10287000407F204668D0FFF7D5FF002323772368E9
:102880001A6912070FD5DA6810070CD56FF0080225
:102890001A610422DB692277990720465AD0FFF794
:1028A000C1FF0023237723681A69D20610D5DA689E
:1028B000D0060DD56FF010021A610822DB6922776D
:1028C00013F4407F20464BD0FFF7ACFF0023237763
:1028D00023681A69D10708D5DA68D20705D56FF0E1
:1028E000010220461A6104F096FB23681A6910065B
:1028F00008D5DA68110605D56FF0800220461A6106
:1029000000F0D5FC23681A69520608D5DA6850062B
:1029100005D56FF0400220461A61FFF785FF236856
:102920001A69910622D5DA6892061FD56FF0200247
:102930002046BDE810401A6100F0B8BCFFF771FFF7
:102940002046FFF770FF83E7FFF76BFF2046FFF796
:102950006AFF92E7FFF765FF2046FFF764FFA0E7F5
:10296000FFF75FFF2046FFF75EFFAFE710BD0000F7
:102970001A4A036890420AD0B0F1804F07D0A2F5FE
:102980009432904203D002F58062904215D14A6899
:1029900023F070031343114A90420AD0B0F1804FE4
:1029A00007D0A2F59432904203D002F580629042A3
:1029B00003D1CA6823F4407313434A6923F08003A8
:1029C000134303608B68C3620B688362034B9842B6
:1029D00004BF0B690363012343617047002C01406E
:1029E00010B5044600284DD00368274A93420FD003
:1029F000B3F1804F0CD0A2F59432934208D002F587
:102A00008062934204D04FF48971204804F080FD25
:102A1000A36833F010020AD023F04002202A06D027
:102A2000402B04D040F21311184804F071FD2369C3
:102A300033F4807207D0B3F5007F04D04FF48A716D
:102A4000124804F065FDA36933F0800304D040F21E
:102A500015110E4804F05CFD94F83D3003F0FF02C0
:102A600023B984F83C20204604F080FF022320682C
:102A700084F83D30211DFFF77BFF0123002084F8FF
:102A80003D3010BD0120FCE7002C01402D920008D4
:102A900010B5044600284DD00368274A93420FD052
:102AA000B3F1804F0CD0A2F59432934208D002F5D6
:102AB0008062934204D040F29B41204804F028FDFC
:102AC000A36833F010020AD023F04002202A06D077
:102AD000402B04D040F29C41184804F019FD2369B2
:102AE00033F4807207D0B3F5007F04D040F29D41EB
:102AF000124804F00DFDA36933F0800304D040F2C6
:102B00009E410E4804F004FD94F83D3003F0FF02AE
:102B100023B984F83C202046FFF782FE0223206878
:102B200084F83D30211DFFF723FF0123002084F8A6
:102B30003D3010BD0120FCE7002C01402D92000823
:102B4000036A2DE9F04123F010030362046AD0F810
:102B5000048086690B6826F4E64646EA03268B68FD
:102B600024F0200444EA03141A4B054698420F4609
:102B700028D1CB6833F0080304D041F24C711648D9
:102B800004F0C6FCFB6824F0800444EA0314BB692B
:102B900024F0400433F4007304D041F25A710E481B
:102BA00004F0B6FC7B6933F4807304D041F25B71AE
:102BB000094804F0ADFCD7E9053228F44068134316
:102BC00048EA83087B68C5F80480AE61AB632C6279
:102BD000BDE8F081002C01402D92000832F00C037A
:102BE00070B504460D46164606D03C2A04D040F681
:102BF000EB51694804F08CFC2B6823F01003602B28
:102C000004D040F6EC51644804F082FCAB6833F029
:102C1000020304D040F6ED515F4804F079FC2B69C3
:102C200033F0040304D040F6EE515B4804F070FC2E
:102C300094F83C300220012B3AD0012384F83D0067
:102C400084F83C300C2E2DD8DFE806F0072C2C2C15
:102C5000332C2C2C592C2C2C7F0023684F4A934268
:102C60000FD0B3F1804F0CD0A2F59432934208D02C
:102C700002F58062934204D040F6FA51464804F0CF
:102C800047FC29462068FFF7A7FC236829699A6951
:102C900042F008029A619A6922F004029A619A69E4
:102CA0000A439A610123002084F83D3084F83C00F7
:102CB00070BD2368394A93420FD0B3F1804F0CD0D6
:102CC000A2F59432934208D002F58062934204D078
:102CD00040F60B61304804F01BFC29462068FFF7E2
:102CE0002FFF236829699A6942F400629A619A6900
:102CF00022F480629A619A6942EA0122D1E723684C
:102D0000264A93420FD0B3F1804F0CD0A2F59432F3
:102D1000934208D002F58062934204D040F61C61D1
:102D20001D4804F0F5FB29462068FFF7A1FC236845
:102D30002969DA6942F00802DA61DA6922F00402EC
:102D4000DA61DA690A43DA61ACE72368134A93422D
:102D50000FD0B3F1804F0CD0A2F59432934208D03B
:102D600002F58062934204D040F62D610A4804F0D7
:102D7000CFFB29462068FFF7C9FC23682969DA6977
:102D800042F40062DA61DA6922F48062DA61DA69B7
:102D900042EA0122D7E700BF2D920008002C014033
:102DA00010B584680A4324F47F4442EA0323234392
:102DB000836010BD90F83C3070B5012B05460C4681
:102DC0004FF002002BD0012385F83C300B6885F8CA
:102DD0003D00B3F5805F0CD0B3F5005F09D033F050
:102DE000300306D0402B04D041F28A11B04804F0E1
:102DF0008FFB2B689A6822F47F4222F077029A6058
:102E00002268402A00F058812BD8102A0CD007D80D
:102E100052B10123002085F83D3085F83C0070BD9B
:102E2000202A01D0302AF4D1A24A93420FD0B3F124
:102E3000804F0CD0A2F59432934208D002F5806204
:102E4000934204D041F2FC11994804F061FB2968D7
:102E500023688A6843F0070322F0700213438B60F3
:102E6000D7E7702A00F0A38046D8502A00F0DD8012
:102E7000602ACED18F4A93420FD0B3F1804F0CD04D
:102E8000A2F59432934208D002F58062934204D0B6
:102E900041F2D911864804F03BFB6368B3F5004F5B
:102EA00009D033F0020206D00A2B04D041F2DC1123
:102EB0007F4804F02DFBE3680F2B04D941F2DD11AC
:102EC0007B4804F025FB2B686668186AE46820F0EC
:102ED0001000186299691A6A21F4704122F0A00268
:102EE00042EA061241EA043199611A629A6822F0B4
:102EF000700242F06702D8E0B2F5805F3FD0B2F5D1
:102F0000005F86D16B4A93420FD0B3F1804F0CD053
:102F1000A2F59432934208D002F58062934204D025
:102F200041F2B511624804F0F3FAA36833F4405358
:102F300004D041F2B8115E4804F0EAFA6368B3F5D0
:102F4000004F09D033F0020206D00A2B04D041F220
:102F5000B911574804F0DCFAE3680F2B04D941F2A9
:102F6000BA11534804F0D4FAD4E90121E36828687F
:102F7000FFF716FF2A68936843F4804353E04D4AF5
:102F800093423FF446AFB3F1804F3FF442AFA2F516
:102F9000943293423FF43DAF02F5806293423FF496
:102FA00038AF41F29611424804F0B2FA31E7414A93
:102FB00093420FD0B3F1804F0CD0A2F594329342DC
:102FC00008D002F58062934204D041F29D11384846
:102FD00004F09EFAA36833F4405304D04FF48D51AB
:102FE000334804F095FA6368B3F5004F09D033F025
:102FF000020206D00A2B04D041F2A1112C4804F0A1
:1030000087FAE3680F2B04D941F2A211284804F093
:103010007FFAD4E90121E3682868FFF7C1FE2A6836
:10302000936843F077039360F3E6224A93420FD00C
:10303000B3F1804F0CD0A2F59432934208D002F540
:103040008062934204D041F2C911194804F060FA39
:103050006368B3F5004F09D033F0020206D00A2BA3
:1030600004D041F2CC11124804F052FAE3680F2B5D
:1030700004D941F2CD110E4804F04AFA2B68616878
:10308000186AE6681C6A20F00A0024F001041C6239
:103090009A69014322F0F00242EA06129A6119622B
:1030A0009A6822F0700242F057029A60B1E600BFBF
:1030B0002D920008002C0140204A93420FD0B3F11A
:1030C000804F0CD0A2F59432934208D002F5806272
:1030D000934204D041F2E911194804F019FA6368E7
:1030E000B3F5004F09D033F0020206D00A2B04D00A
:1030F00041F2EC11124804F00BFAE3680F2B04D9EB
:1031000041F2ED110E4804F003FA2B686168186A69
:10311000E6681C6A20F00A0024F001041C629A6927
:10312000014322F0F00242EA06129A6119629A689B
:1031300022F0700242F04702B7E700BF002C0140C6
:103140002D920008174B70B5984204460D4616465E
:103150000FD0B0F1804F0CD0A3F59433984208D033
:1031600003F58063984204D041F6C9110E4804F07B
:10317000CFF935F00C0306D03C2D04D041F6CA112E
:10318000094804F0C5F90122236A05F01F05AA4089
:1031900023EA02032362236A06FA05F51D4325622A
:1031A00070BD00BF002C01402D92000838B5184AB0
:1031B0000368044693420D460AD0B3F1804F07D00E
:1031C000A2F59432934203D002F58062934202D179
:1031D00035F00C0304D040F213510E4804F098F976
:1031E000206801222946FFF7ADFF2368084A002026
:1031F000934202BF5A6C42F400425A649A6802F049
:103200000702062A1EBF1A6842F001021A6038BD82
:10321000002C01402D92000838B5224A036804466C
:1032200093420D460FD0B3F1804F0CD0A2F59432EB
:10323000934208D002F58062934204D040F2646168
:10324000194804F065F92B6833F0300306D0402BA1
:1032500004D040F26561144804F05AF96B6833F009
:10326000800304D040F266610F4804F051F994F8ED
:103270003C300220012B14D0216884F83D004A68BC
:1032800028688B6822F070020243686823F080038C
:1032900003434A6000208B60012384F83C0084F8DB
:1032A0003D3038BD002C01406592000870477047E2
:1032B0000368DA6822F49072DA605A6922F0010237
:1032C0005A61202380F83A307047000038B54268D0
:1032D0002E4B05469A4204D940F6FD312C4804F0A5
:1032E00017F9EB6833F4005304D040F6FE31284858
:1032F00004F00EF92B6933F4806207D0B3F5C06F88
:1033000004D040F6FF31224804F002F94FF6F37280
:103310006B69134200D123B94FF440611C4804F09B
:10332000F7F82B68E9681A69286922F440520A43C1
:103330001A61AA68D9680243686921F4B05121F082
:103340000C0102430A43DA605A69A96922F4407207
:103350000A435A610F4A1924934214D1FEF7E8FB3D
:1033600060436C686422A400B0FBF4F0B0FBF2F19F
:1033700002FB11031B013233B3FBF2F32C6803EBA6
:103380000113A36038BDFEF7C3FBE9E720AA4400A0
:10339000A09200080038014010B5044600285BD018
:1033A000816903682D4A00294AD093420CD0A2F5C6
:1033B0007442934208D002F58062934204D04FF4E5
:1033C000A371274804F0A4F8A36933F4407304D030
:1033D00040F24711224804F09BF8A36833F480536D
:1033E00004D040F24D111E4804F092F894F83930A0
:1033F00003F0FF0223B984F83820204604F022FBB2
:103400002423226884F83930D368204623F40053FB
:10341000D360FFF75BFF236800201A6922F4904213
:103420001A615A6922F02A025A61DA6842F400529B
:10343000DA602023E06384F8393084F83A3010BD34
:103440009342CAD0074A9342C7D002F580629342A2
:10345000C3D040F24B11BDE70120F0E70038014036
:10346000A09200080044004090F83930202B18D179
:10347000A9B1A2B190F83830012B12D0C284828455
:103480000023212201620168C36380F83920CA68E1
:1034900080F8383042F08002CA6018467047012038
:1034A00070470220704790F83A30202B20D1E9B1C4
:1034B000E2B190F83830012B1AD0C2858285002302
:1034C0002222C36380F83A2002688162D16880F8C2
:1034D000383041F48071D1605169184641F00101E2
:1034E0005161D16841F02001D160704701207047DF
:1034F0000220704790F83A3010B5222B33D1816802
:103500000469B1F5805F836A026823D15268ECB91F
:10351000C2F3080223F8022B8362C48D013CA4B2DB
:10352000C4858CB90368DA6822F02002DA60DA68B0
:1035300022F48072DA605A6922F001025A61202373
:1035400080F83A3004F01EF900200DE0D2B223F8E2
:10355000012BE1E7591C526881620CB91A70DCE753
:1035600002F07F02FAE7022010BD0000036870B588
:103570001A6804461607D9685D6907D1960658D5BA
:103580008D0656D5BDE87040FFF7B4BF15F00105B4
:1035900002D111F4907F4CD0D30705D5CE0542BFA0
:1035A000E36B43F00103E363500704D51DB1E36B04
:1035B00043F00203E363930704D51DB1E36B43F0CB
:1035C0000403E363160704D51DB1E36B43F008035E
:1035D000E363E36B43B3950604D5880602D5204622
:1035E000FFF788FF236820465D69E26B110702D46C
:1035F00015F0400519D0FFF75BFE23685A695206A3
:103600000FD55A69606B22F040025A6148B1264BCF
:103610004363FCF72BFF38B1606BBDE87040436B30
:103620001847204604F0D8F870BD04F0D5F8E563DB
:10363000FAE7160628D50D0626D594F83920212A52
:10364000F2D1A168226AB1F5805F18D11188C1F367
:1036500008015960216981B902322262E28C013A83
:1036600092B2E284002ADFD1DA6822F08002DA60C6
:10367000DA6842F04002DA60D6E70132EDE7511C29
:10368000216212785A60E9E75006CDD54A06CBD5BB
:10369000DA68204622F04002DA60202384F83930CC
:1036A00004F04EF8C0E700BFAD36000808B50023AF
:1036B000406AC385C38404F08FF808BD84B001A8B4
:1036C00080E80E0004B000207047B0F8403043F4AA
:1036D0003F43A0F8403000207047B0F8403023F45A
:1036E0007C535B045B0CA0F8403000207047002046
:1036F000704784B010B503AC84E80E00BDE81040FC
:103700000123A0F840300023A0F84030A0F8443056
:10371000A0F85030B0F8402004B042F43F42A0F886
:103720004020184670470000F0B50C78034630F88A
:103730002420C87822F4EC4222F07002032803D837
:10374000DFE800F042494446012048F280052A4360
:1037500023F824200E789E4A33F82640354314403F
:103760002C4323F826400D7B0C78002D40F08280FE
:10377000CD884E786D086D0003EB041476B3B3F872
:1037800050603444A4F800540D7833F8254067069F
:1037900008D533F82540224042F4004242F0C002EE
:1037A00023F82520CA780C78012A33F82410894A96
:1037B00002EA010218BF82F0200242F4004242F005
:1037C000800223F82420F0BD42F400720020BCE700
:1037D00042F4C062FAE742F48062F7E7B3F850209F
:1037E0000E691444A4F808540A78B3F8504003EB67
:1037F0000212A4B202F20C4256BB155B25F4F84546
:103800002D042D0C1553155B45F4004515530C780C
:1038100033F8242057040BD533F8242022F0F0028B
:103820001205120D42F4404242F0800223F8242097
:10383000097833F8212022F4804222F0700282F4C9
:10384000405242F4004242F0800223F82120BAE7BD
:103850003E2E06D87508F60748BF0135AD02ADB259
:10386000D4E77709F5065C4D08BF07F1FF3745EA55
:103870008725F4E733F82450154045F4014545F019
:10388000800523F824500C780D89B3F8506003EBC1
:1038900004146D08B6B204F580646D00A5530C786D
:1038A0004D89B3F8506003EB04146D0804F581648E
:1038B0006D00B6B2A5534C780D78002C43D133F887
:1038C0002540660408D533F82540224042F44042A2
:1038D00042F0800223F825200C7833F82420550686
:1038E0000BD533F8242022F0F0021205120D42F419
:1038F000004242F0C00223F824200C7833F8242040
:1039000022F0F0021205120D42F4004242F0C00211
:1039100023F8242048F280040D7833F8252022F47F
:10392000804222F0700282F44052224323F8252084
:10393000097833F8212022F4E04222F040021443B7
:1039400023F821403FE733F82540640408D533F8D5
:103950002540224042F4404242F0800223F82520D4
:103960000C7833F8242052060BD533F8242022F0AB
:10397000F0021205120D42F4004242F0C00223F898
:1039800024200C7833F8242022F0F0021205120DC6
:1039900042F4404242F0800223F82420CA780C7896
:1039A000012A33F824500B4A02EA050218BF82F0BC
:1039B000200242F4004242F0800223F824200978D9
:1039C00033F8212022F0F0029204920C39E700BF74
:1039D0008F8FFFFFBF8FFFFF0080FFFF10B50C7BB5
:1039E0004A780B78BCBBF2B130F8232052060BD5D5
:1039F00030F8232022F0F0021205120D42F40042AA
:103A000042F0C00220F823200A7830F8223023F058
:103A1000C0031B051B0D43F4004343F0800320F853
:103A20002230002010BD30F8232054040BD530F88C
:103A3000232022F0F0021205120D42F4404242F01F
:103A4000800220F823200A7830F8223023F0F00397
:103A50009B049B0CDFE7002A44D130F8232052045A
:103A60000BD530F8232022F0F0021205120D42F49B
:103A7000404242F0800220F823200A7830F82230B9
:103A80005C060BD530F8223023F0F0031B051B0D2C
:103A900043F4004343F0C00320F822300A7830F8A2
:103AA000223023F0F0031B051B0D43F4004343F0C9
:103AB000C00320F8223048F280020C7830F824301D
:103AC00023F4804323F07003134320F82430097853
:103AD00030F8213023F4E04323F040031A4320F868
:103AE00021209EE730F8232052040BD530F8232004
:103AF00022F0F0021205120D42F4404242F0800220
:103B000020F823200A7830F822305B060BD530F8F5
:103B1000223023F0F0031B051B0D43F4004343F058
:103B2000C00320F822300A7830F8223023F0F00366
:103B30001B051B0D43F4404343F0800320F8223063
:103B400048F280020C7830F8243023F4E04323F06C
:103B50004003134320F82430097830F8213023F44F
:103B6000804323F07003B9E74B780A787BB130F8D3
:103B7000223023F4E04323F0400383F0100343F4A6
:103B8000004343F0800320F822300020704730F8D3
:103B9000223023F4804323F0700383F48053EEE754
:103BA0000B7B23BB4B780A781BB330F822305B06C3
:103BB0000BD530F8223023F0F0031B051B0D43F426
:103BC000004343F0C00320F82230CB78012B0ED005
:103BD0000A7830F8223023F4E04323F0400383F0E6
:103BE000200343F4004343F0800320F822300020F8
:103BF000704730F822305B040BD530F8223023F0C8
:103C0000F0031B051B0D43F4404343F0800320F8F1
:103C100022300A7830F8223023F4804323F07003F6
:103C200083F44053DDE711B98023A0F84C30002025
:103C300070470020704700207047B0F8440070477C
:103C40000020704700EB4202013302F580625B08FE
:103C500002EB83039A4200D1704731F8020B22F83D
:103C6000040BF7E770B50D46497804460129AA69A7
:103C70002B69287B5DD19A429DBF0023AB6113461F
:103C8000D21A88BFAA6169699EB2E8B93346EA8848
:103C90002046FFF7D7FFB4F850102A7804F2044307
:103CA00012010B44D6522A7834F8223023F4E04330
:103CB00023F0400383F0300343F4004343F08003D8
:103CC00024F82230002070BD2B7834F82320B4F87B
:103CD000500052064BBF04F20C4204F20442121888
:103CE00012184FEA03134BBFD652D6526A892A895B
:103CF00033462046FFF7A6FF6B782A7863B934F87D
:103D0000223023F0F0031B051B0D43F4004343F066
:103D1000C00324F82230C6E7012BC4D134F8223086
:103D200023F0F0031B051B0D43F4404343F08003D5
:103D3000EFE79A4293BF0023D21AAA61AB6198BF02
:103D400013462A7890B9B4F8501004F20C4001449C
:103D50001201002B3BD18B5A23F4F8431B041B0C9C
:103D60008B528B5A43F400438B5239E081B9B4F83B
:103D7000501004F2044001441201B3B9885A20F4EF
:103D8000F8400004000C8852885A40F400408852E1
:103D900069782A780029D6D0012921D1B4F85000B9
:103DA00004F20C41014412012CE03E2B06D85808C5
:103DB000DE0748BF0130800280B2E8E75E09D8061E
:103DC000114808BF06F1FF3640EA8620F4E73E2B93
:103DD00010D85808DE0748BF0130800280B28852F0
:103DE0002A7834F8223023F4804323F0700383F4DC
:103DF000405361E75809DB06034B08BF00F1FF3071
:103E000043EA80239BB2AFE70080FFFF00EB420252
:103E1000F0B502F580625D08084617462E4602306E
:103E200036B9DB0744BF32F8253001F81530F0BD54
:103E300037F8044B013EA4B200F8024C240A00F803
:103E4000014CECE7D0F8BC3210B56BB1D0F8B842F9
:103E500094F84000FF2807D09B6894F84120214641
:103E60009847FF2384F84030002010BD432303808F
:103E700000487047400000204323038000487047FB
:103E8000840000204323038000487047D4000020B2
:103E90000A23038000487047C800002038B5054653
:103EA000D0F8B84204F0F0FDD5F8B832E06443B180
:103EB000D5F8BC3204F14C01DB68606C98470020F7
:103EC00038BD0220FCE7F8B5D0F8B8320246F3B1AD
:103ED000142505FB0105EE6986B1D0F8C04204EB5C
:103EE0004114A76BB6FBF7F407FB146434B9EC611B
:103EF0002346224604F0ACFD2046F8BD0024D2F84B
:103F0000BC225C651269196D986C9047F4E7022039
:103F1000F3E72DE9F7434FF000080A78054612F061
:103F200060040E46D0F8B8728DF80580ADF80680B2
:103F300028D0202C45D1CC884B78E4B1120611D57D
:103F4000D0F8BC223946D2F8089018462246C84715
:103F5000F2883946284600F038FC4446204603B033
:103F6000BDE8F08387F8403087F841402246394663
:103F700000F040FCF1E7D0F8BC22184695682246D4
:103F8000A847EBE74F780A2F0DD00B2F15D0C7B9F4
:103F900090F89C32032B14D102220DF1060100F09F
:103FA00014FC3C46DAE790F89C32032B09D101223D
:103FB0000DF1050100F009FCD0E790F89C32032BCD
:103FC000CCD03146284600F0D9FB0224C6E738B5EC
:103FD00004460025812104F0F3FC0121E56220461E
:103FE00004F0EEFCC4F86C518221204604F0E8FC99
:103FF000D4F8B83225644BB1D4F8BC325B6898472A
:10400000D4F8B80204F048FDC4F8B852002038BD16
:10401000037C2DE9F0410446ABBB4FF40073022250
:104020008121012504F0BCFC4FF40073E5622946B0
:104030000222204604F0B4FCC4F86C510125082388
:1040400003228221204604F0ABFC25645C2004F0AE
:104050001FFD0646C4F8B80230B30027D4F8BC32BE
:104060001B68984794F810807765B765B8F1000F22
:1040700012D14FF40073726C2946204604F0F6FC0E
:104080004046BDE8F081012540230222812104F051
:1040900087FCE5624023CAE74023726C294620462C
:1040A00004F0E4FC3846ECE72846EAE719B1C0F82A
:1040B000BC120020704702207047D0F8B8320020B0
:1040C00099641A657047D0F8B83200205964704777
:1040D000D0F8B82210B562B1546D01235CB95365B4
:1040E000136D81210363926C9BB204F0B1FC2046F6
:1040F00010BD0220FCE71846FAE7D0F8B82210B548
:104100005AB1047C526C34B94FF40073012104F0AD
:10411000ADFC002010BD4023F8E70220FAE708B507
:1041200080B1D0F8B43213B10023C0F8B43209B171
:10413000C0F8B0120123027080F89C3204F0E0FB5A
:10414000002008BD0220FCE719B1C0F8B41200201D
:1041500070470220704708B504F014FC002008BD29
:1041600008B5D0F8B4320BB9022008BD1B689847D7
:104170000028FAD0F8E708B5D0F8B4325B68984761
:10418000002008BD38B500F52A750446284600F021
:10419000E1FA012394F8A812C4F89432B4F8AE32CC
:1041A000C4F8983201F01F03012B0ED007D3022B65
:1041B00010D001F08001204604F010FC03E02946F5
:1041C000204600F0F5F8002038BD2946204600F0D2
:1041D00013FAF8E72946204600F033FAF3E770B502
:1041E0000546164649BBD0F89432032B1ED1D0F8B1
:1041F0006031D0F8642193420BD99B1A9A42C0F8DF
:1042000060318CBF9AB292B2314600F002FB0020BE
:1042100070BDD0F8B4321B6923B190F89C22032AF8
:1042200000D19847284600F0FCFAF0E7052BEED1C4
:10423000C5F8941204F0D2FBE9E7D0F8B4329B69D8
:104240002BB190F89C22032A01D19847DFE7022086
:10425000DEE770B5134604460E46002947D1D0F874
:104260009422022A3CD1D0E90852954213D9AA1AC5
:104270000262194692B200F0B5FA33461A46194660
:10428000204604F0F3FB94F8A0320020012B01D16A
:1042900084F8A00270BDC369B3FBF2F502FB1535CB
:1042A00065B99A420AD8D0F89822934206D22A4693
:1042B00000F098FAC4F898522B46DFE7D4F8B432ED
:1042C000DB682BB194F89C22032A01D12046984741
:1042D0008021204604F082FB204600F0ADFAD2E7B0
:1042E00032F00403CFD1802104F078FBCBE7D0F883
:1042F000B4325B6933B190F89C22032A02D198470B
:104300000020C7E70220C5E7002270B5044601255A
:1043100040261146402304F043FB33468021C4F875
:104320005851C4F864610022204604F039FB002192
:10433000D4F8B832A561666284F89C52C4F894122D
:104340006160C4F8A41223B1D4F8B43220465B688B
:104350009847002070BD01740020704790F89C328F
:1043600080F89D32042380F89C320020704790F83A
:104370009C32042B04BF90F89D3280F89C320020C0
:10438000704708B590F89C22032A04D1D0F8B432C3
:10439000DB6903B19847002008BD10B504468021B1
:1043A00004F01CFB2046BDE81040002104F016BBC1
:1043B00037B50B78044603F06003202B0D4612D06E
:1043C000402B10D0002B5BD14B78092B58D8DFE85D
:1043D00013F0E90005015700FE00570084001300A8
:1043E0005700D200A000D4F8B43229469B6820467A
:1043F0009847002003B030BD0023ADF806304B884D
:104400001A0A013A062A3BD8DFE802F004202D3AC6
:104410003A525C00D0F8B0321B680DF10601207CE6
:104420009847BDF8062052B1EB8843B19A4228BFA5
:104430001A4601462046ADF8062000F0C6F9EB8882
:10444000002BD6D1204600F0ECF9D2E7027CD0F860
:10445000B43232B99B6A0DF10600984702234370CB
:10446000DFE7DB6AF7E7DBB2052B09D8DFE803F00B
:10447000030C1014181CD0F8B0325B68002BCCD1A0
:104480002046FFF78AFFB4E7D0F8B0329B68F5E723
:10449000D0F8B032DB68F1E7D0F8B0321B69EDE755
:1044A000D0F8B0325B69E9E7D0F8B0329B69E5E754
:1044B000037C002BE4D1D0F8B4320DF106005B6B25
:1044C0009847AEE7037C002BDAD1D0F8B4320DF177
:1044D00006001B6B98470723C1E78B88002BCFD1C1
:1044E000CB88002BCCD14D887F2DC9D890F89C3239
:1044F000032BC5D0E9B280F89E1204F09BFA204647
:1045000000F08FF91DB1022384F89C3271E701237A
:10451000FAE78978374D01292970B1D890F89C3293
:10452000022B08D0032B14D0FFF737FF2978204641
:10453000FFF721FE5DE7002984D0012103234160BC
:1045400080F89C322046FFF70BFE02287FF47AAFFA
:1045500096E731B90223416080F89C32FFF70BFEE9
:1045600070E7416801293FF46DAFC9B2FFF703FE60
:1045700029786160E6E7CA88012A81D190F89C32E7
:10458000002B3FF47DAF022B04D9032B7FF478AFCF
:10459000011D03E00146002341F8083F204600F0DA
:1045A00014F926E790F89C32013B022B3FF668AFE6
:1045B000CB88022B7FF464AF0123C360D0F8A43210
:1045C0000BB10323C360022204F10C01E6E74B8820
:1045D000012B7FF40EAFC4F8A43233E790F89C327D
:1045E000013B022B3FF64CAF4B88012B7FF401AF10
:1045F0000023F0E7E407002038B50B78044603F009
:104600006003202B0D4602D0402B00D0ABB994F8AC
:104610009C32013B022B10D82B79012B0DD8D4F8FA
:10462000B43229469B6820469847EB881BB910B9DD
:10463000204600F0F6F8002038BD2046FFF7ADFE1A
:10464000F9E738B50A78044602F06002202A0B46E2
:1046500014D0402A12D06AB95A788D88012AE9B25A
:1046600020D036D3032A05D190F89C22022A27D0E5
:10467000032A0BD02046FFF790FE05E0D4F8B422C1
:104680001946926820469047002038BD5A882AB9BA
:104690004A0603D0DB880BB904F0A0F9204600F0ED
:1046A000C0F8F1E790F89C22022A09D0032AE1D150
:1046B0005B88002BE8D14D06F0D004F09DF9EDE7C2
:1046C0004B06D7D004F08AF98021204604F086F901
:1046D000DAE790F89C32022B18D0032BCAD11423AE
:1046E00001F00F0215F0800F03FB02021FD0926948
:1046F000002ABFD001F07F0505FB0335054411F00A
:104700007F031FD12B60022229460CE04A06B1D15B
:104710002B064FF000034FF002024CBF00F11401D2
:1047200000F5AA710B60204600F04FF8ACE7D2F814
:104730005821002A9ED001F07F0503FB050505F5F1
:10474000AA75DCE7204604F065F908B10123D9E732
:104750002860D8E70B7803704B784370CA788B7861
:1047600003EB022343804A790B7903EB0223838016
:10477000CA798B7903EB0223C380704710B50446D6
:10478000802104F02BF92046BDE81040002104F000
:1047900025B930B588B105462B1A15F8014BDBB2A7
:1047A000002CF9D101335B0013800B7003234B7095
:1047B0000223013810F8015F05B930BD5A1CCD54F1
:1047C000D2B20233DBB28C54F4E71346022210B5A6
:1047D000C0F89422C0E907330A46002104F038F9F2
:1047E000002010BD08B513460A46002104F030F938
:1047F000002008BD1346032210B5C0F89422C0F86B
:104800005C310A46C0F86031002104F02FF9002025
:1048100010BD08B513460A46002104F027F9002010
:1048200008BD08B50423C0F8943200231A4619467F
:1048300004F00EF9002008BD08B50523C0F8943235
:1048400000231A46194604F011F9002008BD08B5E6
:1048500000F0FAFC002008BD70B5054646690B461D
:10486000D0E9001086B02A69B5F9084076B1AD6983
:1048700065B1842C0CBF00240334CDE9016500949C
:1048800000F07AFC0590059806B070BD842C0CBF32
:104890000024033405AD92B2CDE9004500F0A5FC3B
:1048A0000128F0D00020EFE708B5002808BF01205C
:1048B00000F018FE002008BD4FF0FF3200F10803A1
:1048C0004360C0E9022303610023036070470023B3
:1048D0000361704743689A684B608A609A685160C8
:1048E0009960036808610133036070470A6830B556
:1048F000531C0AD103695A684A6091608B60596001
:10490000036808610133036030BD00F108035C688F
:1049100025689542EFD82346F9E70369D0E90112EB
:104920008A60826851605968814208BF5A600022DB
:1049300002611A68013A1A601868704710B5044697
:1049400001F0A0F9A46B01F0BFF9B4FA84F04009BA
:1049500010BD70B51546026C0446866B42B90568F9
:104960009DB9406800F048FF65600136A66370BDE0
:104970006DB9806804F06AFAA368226C1344626817
:10498000A360934201D32368A3600020EDE7C068D1
:1049900004F05CFA236CE2685B4221681A448A42A4
:1049A000E2603EBF62689B18E360022DEDD10EB15C
:1049B000013EEAE73046D8E770B5044601F062F9F7
:1049C00094F8455004F124066DB2002D14DCFF2349
:1049D00084F8453001F078F901F054F994F8445026
:1049E00004F110066DB2002D12DCFF2384F8443070
:1049F000BDE8704001F068B9636A002BE7D030462B
:104A000000F006FE08B100F08DFE013D6DB2DCE75E
:104A10002369002BE9D0304600F0FAFD08B100F020
:104A200081FE013D6DB2DEE738B50D46044640B962
:104A30004FF0500383F31188BFF36F8FBFF34F8F95
:104A4000FEE701F01FF9D4E90F3043432268D11883
:104A50001B1A13446160E3600021FF23A163A2607D
:104A600084F8443084F8453095B9236963B104F182
:104A7000100000F0CDFD38B14FF08052094B1A60A4
:104A8000BFF34F8FBFF36F8F01F01EF9012038BDC8
:104A900004F11000FFF710FF04F12400FFF70CFFF2
:104AA000F2E700BF04ED00E013B51C4640B94FF03B
:104AB000500383F31188BFF36F8FBFF34F8FFEE76F
:104AC00043B94FF0500383F31188BFF36F8FBFF3E7
:104AD0004F8FFEE74AB191B94FF0500383F311882D
:104AE000BFF36F8FBFF34F8FFEE741B14FF050031D
:104AF00083F31188BFF36F8FBFF34F8FFEE750230F
:104B00000193019B502B08D04FF0500383F3118881
:104B1000BFF36F8FBFF34F8FFEE70123002908BF5C
:104B20002246C4E90F0184F8463019462260204627
:104B3000FFF77AFF20469DF8103084F84C3002B021
:104B400010BD00002DE9FF47884601921F4604462C
:104B500040B94FF0500383F31188BFF36F8FBFF359
:104B60004F8FFEE751B9036C43B14FF0500383F30D
:104B70001188BFF36F8FBFF34F8FFEE7022F0BD16A
:104B8000E36B012B08D04FF0500383F31188BFF380
:104B90006F8FBFF34F8FFEE700F0CAFD50B9019E43
:104BA0004EB14FF0500383F31188BFF36F8FBFF303
:104BB0004F8FFEE700264FF00009DFF8E8A037E04E
:104BC000019D1DB901F080F8002050E016B902A83F
:104BD00000F060FD01F078F800F074FB01F052F88D
:104BE00094F84430FF2B08BF84F8449094F8453083
:104BF000FF2B08BF84F8459001F066F801A902A8D0
:104C000000F054FD002846D101F03CF8A26BE36BA4
:104C10009A422FD101F058F8019904F1100000F0E8
:104C2000DDFC2046FFF7C8FE00F0E6FB50B301268E
:104C300001F028F8A26BE36B9A4201D3022FBFD197
:104C40003A4641462046FFF784FE636A1BB104F1F1
:104C5000240000F0DDFC38B14FF08052114B1A6097
:104C6000BFF34F8FBFF36F8F01F02EF8012004B018
:104C7000BDE8F08701F028F82046FFF79DFE00F020
:104C8000BBFBD4E74FF08053CAF80030BFF34F8F1F
:104C9000BFF36F8FCBE72046FFF78EFE00F0ACFB33
:104CA00092E700BF04ED00E0002213B50B46009030
:104CB00011460120FFF7F8FE044638B10023C0E991
:104CC0000033C3601A461946FFF73CFF204602B086
:104CD00010BD00002DE9FF410446019140B94FF09D
:104CE000500383F31188BFF36F8FBFF34F8FFEE73D
:104CF000056C45B14FF0500383F31188BFF36F8FFC
:104D0000BFF34F8FFEE700F013FD50B9019D45B191
:104D10004FF0500383F31188BFF36F8FBFF34F8FB2
:104D2000FEE72E460027DFF82C814FE0019B63B998
:104D300045B14FF0500383F31188BFF36F8FBFF37A
:104D40004F8FFEE700F0C0FF5EE016B902A800F04A
:104D5000A1FC00F0B9FF00F0B5FA00F093FF94F861
:104D60004430FF2B08BF84F8447094F84530FF2B83
:104D700008BF84F8457000F0A7FF01A902A800F061
:104D800095FC00284AD12046FFF7D8FD00283FD0E7
:104D900023683BB900F076FF606800F0D9FC054657
:104DA00000F092FF019904F1240000F017FC204666
:104DB000FFF702FE00F020FB38B94FF08053C8F82F
:104DC0000030BFF34F8FBFF36F8F012600F05AFF03
:104DD000A36B002BAAD0013BA363236813B900F097
:104DE000B3FD6060236963B104F1100000F010FCB2
:104DF00038B14FF08052174B1A60BFF34F8FBFF39B
:104E00006F8F00F061FF0125284604B0BDE8F081F6
:104E10002046FFF7D1FD00F0EFFAD6E72046FFF776
:104E2000CBFD00F0E9FA2046FFF788FD0028CCD042
:104E3000002DE9D000F026FF616A19B1236B1968D3
:104E4000C1F10701606800F027FD002500F03CFF7C
:104E5000DAE700BF04ED00E02DE9F041044600F080
:104E600011FF2F4B2F4D1A682F4F01321A602E68F9
:104E7000002E49D12C601B68012B1FD14FF0140864
:104E800008FB06700136FFF717FD072EF8D1DFF893
:104E9000C480264E4046FFF70FFD3046FFF70CFD5D
:104EA0002348FFF709FD2348FFF706FD2248FFF7D7
:104EB00003FD224BC3F80080214B1E60214A22498A
:104EC000136808680133136063640123E26A934046
:104ED000034314200B6000FB0270211DFFF7FAFC56
:104EE00000F0F2FE194B1B6863B12B68DA6AE36AC3
:104EF0009A4207D24FF08052154B1A60BFF34F8F82
:104F0000BFF36F8FBDE8F081104B1B68002BD5D12C
:104F10002B68DA6AE36A9A4298BF2C60CEE700BF3A
:104F200080080020E8070020F4070020AC080020DB
:104F3000C8080020F4080020E0080020EC0700204A
:104F4000F00700209008002094080020DC080020D2
:104F500004ED00E09808002010B50446583003F036
:104F600095FF94F885343BB9206B01F089F8204611
:104F7000BDE8104001F084B8012BF8D0022B08D016
:104F80004FF0500383F31188BFF36F8FBFF34F8F40
:104F9000FEE710BD80B5DFF85C80124F124C134D58
:104FA000236863B9124B1B68012BF8D94FF080536B
:104FB000C8F80030BFF34F8FBFF36F8FEEE700F0FC
:104FC00061FEFB68DE68301DFFF7A7FC2B68013B24
:104FD0002B602368013B236000F076FE3046FFF72C
:104FE000BBFFDDE7F40800208408002080080020D3
:104FF000F407002004ED00E0064A13681968064B28
:1050000019B94FF0FF321A6070471268D268D2683F
:105010005268F8E7EC070020C00800202DE9F047AF
:105020000D46DDE90974960032468046A521206BC5
:10503000994603F016FF236B043E1E4426F0070634
:105040006B1E04F134020F3513F8011F02F8011B27
:10505000197809B1AB42F7D1089D4FF0000A062D2F
:1050600028BF0625201DE562C4E9135A84F843A031
:10507000FFF72DFCC5F1070504F11800FFF727FC29
:10508000C4F880A44FF4856251462461A56164622E
:1050900084F884A404F1580003F0E3FE04F551738E
:1050A000E36504F56B73236604F21443636601231E
:1050B000C4F800310A4B4A46C4F80831094B41464E
:1050C000C4F80C31084B3046C4F810310B23A4F857
:1050D000143100F0B1FD206007B13C60BDE8F087FD
:1050E0000E33CDAB34126DE6ECDE0500F8B51B4B8C
:1050F0001B4E1C68054630680F460430FFF70DFC58
:10510000334640B901203168164EC96A326888407A
:1051100022EA000232606A1C07D137B119681248CE
:105120000431BDE8F840FFF7D5BB1A686419546034
:1051300007D30E4A10681968BDE8F8400431FFF73C
:10514000D5BB0B4A106819680431FFF7CFFB094B38
:105150001A68A24288BF1C60F8BD00BF0809002081
:10516000E807002094080020E0080020F007002055
:10517000EC070020C008002070B586B0DDE90B54B4
:1051800045B94FF0500383F31188BFF36F8FBFF31E
:105190004F8FFEE744B94FF0500383F31188BFF3FC
:1051A0006F8FBFF34F8FFEE74FF491660496049E16
:1051B000B6F5916F08D04FF0500383F31188BFF319
:1051C0006F8FBFF34F8FFEE72563022584F8855468
:1051D00005AD01950A9D02940095FFF71FFF20463B
:1051E000FFF73AFE059806B070BD2DE9F04307467B
:1051F00085B0900088461646994600F0C5FE0546E3
:10520000F0B14FF4916000F0BFFE0446A8B1002356
:1052100080F885340D9B056301930C9B02900093ED
:1052200032464B4641463846FFF7F8FE2046FFF728
:1052300013FE012005B0BDE8F083284600F020FFF2
:105240004FF0FF30F6E7000010B5002488B007AA41
:1052500006A905A8CDE9054401F042FE059B079A81
:105260000293069B1049CDE9004310482346FFF7FF
:1052700083FFB8B14FF0500383F31188BFF36F8FF2
:10528000BFF34F8F0A4B0B4A1B68583313604FF024
:10529000FF32094B1A600122084B1A60084B1C6050
:1052A00000F078FD08B010BDD9920008954F0008B5
:1052B000E8070020F8050020C0080020DC080020D6
:1052C00008090020024A136801331360704700BFC9
:1052D0008C0800202DE9F84F3C4B1B68002B6ED149
:1052E0003B4B1C6801341C60BCB93A4B1A6812680D
:1052F00042B14FF0500383F31188BFF36F8FBFF3B8
:105300004F8FFEE7344A1968106818601160334AFD
:10531000136801331360FFF76FFE314D4FF0000B40
:105320002B68304FA34211D93A682F4BD16A14220F
:105330004A439A58022A28BF4FF0010B2B4A1268A1
:10534000002A0CBF58460120BDE8F88FDFF884A082
:10535000DFF8A090DAF8002012681AB94FF0FF3297
:105360002A60E1E7DAF80020D268D66871688C42DA
:1053700001D22960D8E706F104084046FFF7CDFACC
:10538000B16A19B106F11800FFF7C7FA01224FF010
:10539000140CF06AD9F8003002FA00F11943124BEC
:1053A000C9F800100CFB00304146FFF793FA38684B
:1053B000F16AC26A914228BF4FF0010BCAE70C4A5A
:1053C0004FF0000B136801331360B7E78C0800201F
:1053D00008090020EC070020F0070020C408002086
:1053E000C0080020E8070020F40700200C09002076
:1053F00088080020940800202DE9F843304C2368E9
:1054000043B94FF0500383F31188BFF36F8FBFF39D
:105410004F8FFEE700F036FC2368013B23602468D1
:105420002CB1002400F050FC2046BDE8F883254B49
:105430001B68002BF5D0244D244EDFF8A4801FE01C
:10544000EB680127DC6804F1040904F11800FFF798
:1054500064FA4846FFF761FA1420E26A316807FAF5
:1054600002F30B4300FB028049463360FFF732FA38
:10547000174BE26A1B68DB6A9A4201D3154B1F6027
:105480002B68002BDCD10CB1FFF7B6FD124D2C6858
:1054900044B101270F4EFFF71DFF00B13760013CFB
:1054A000F9D12C600B4B1B68002BBAD04FF0805207
:1054B0000A4B1A60BFF34F8FBFF36F8F0124B1E720
:1054C0008C08002080080020C808002094080020D4
:1054D000E80700200C0900208808002004ED00E007
:1054E000F407002008B540B94FF080520D4B1A6008
:1054F000BFF34F8FBFF36F8F08BD0B4B196841B1DE
:105500004FF0500383F31188BFF36F8FBFF34F8FBA
:10551000FEE7FFF7D7FEFFF7E9FDFFF76DFF002875
:10552000E2D0E9E704ED00E08C08002038B5254B17
:105530001A68254B12B101221A6038BD234C1A603B
:1055400023681B6B1A68B2F1A53F0BD15A68B2F100
:10555000A53F07D19A68B2F1A53F03D1DB68B3F14B
:10556000A53F04D020682168343101F047FD184B75
:105570001B68B3FA83F31422DBB2C3F11F035A434F
:1055800014498D58881845B94FF0500383F311889A
:10559000BFF36F8FBFF34F8FFEE7456808326D682A
:1055A0000A44954208BF6A68456008BF42601422F9
:1055B00002FB03135B68084ADB68236023685833E7
:1055C0001360BAE78C0800200C090020E8070020CF
:1055D00094080020F4070020F805002010B50C46C0
:1055E00040B94FF0500383F31188BFF36F8FBFF3BF
:1055F0004F8FFEE7054B19681831FFF777F9204602
:10560000BDE810400121FFF771BD00BFE807002091
:1056100038B5C368DC6844B94FF0500383F3118890
:10562000BFF36F8FBFF34F8FFEE704F118052846D5
:10563000FFF773F9114B1B68E3B9251D2846FFF7E7
:105640006CF901230E49E26A086893400343142071
:105650000B6029460B4B00FB0230FFF73BF90A4B6E
:10566000E26A1B68DB6A9A4285BF0120074B002073
:10567000186038BD29460648EFE700BF8C080020B7
:1056800094080020F4070020E80700200C090020FF
:10569000C8080020034B1B680360034B1B68436072
:1056A000704700BFC408002008090020F8B50C4668
:1056B000054640B94FF0500383F31188BFF36F8F55
:1056C000BFF34F8FFEE741B94FF0500383F31188CA
:1056D000BFF36F8FBFF34F8FFEE700F0D3FA0F4B8E
:1056E0006868196823680A1A5E1C0DD00C4E2F6872
:1056F0003668B74201D088420DD9934209D99B1A26
:1057000023602846FFF7C6FF002400F0DDFA20469C
:10571000F8BD002323600124F7E700BF080900203B
:10572000C40800200122014B1A6070470C090020B8
:10573000054B1B6833B1054B1B68002B0CBF0220C7
:105740000020704701207047DC0800208C080020F2
:105750002DE9F041044660B3244AC36A1168174634
:10576000C96A8B4239D214268269214D002AA8BF0A
:105770003A6806FB0353A2BFD26AC2F107028261F4
:1057800042699A4217D100F104084046FFF7C5F874
:10579000184BB0B13A681968D26AE262012404FA7F
:1057A00002F0084318601420414600FB0250FFF746
:1057B00091F8204603E03B68DB6AC3620120BDE844
:1057C000F081E06A4643AA59002AE3D101211A6810
:1057D000814022EA01021A60DCE71368C06CDC6ACF
:1057E000A0422CBF00200120E9E700BFE80700200D
:1057F000F407002094080020F8B5044608B90020FA
:10580000F8BD224B1B68834208D04FF0500383F34E
:105810001188BFF36F8FBFF34F8FFEE71B6D43B946
:105820004FF0500383F31188BFF36F8FBFF34F8F97
:10583000FEE7C16AC26C013B91420365DFD0002BD9
:10584000DDD1051D2846FFF768F8114E114A50B901
:105850001421E76A794373582BB901201368B840C3
:1058600023EA00031360E36CC3F10701A161E36263
:105870000124116804FA03F008431060142029463B
:1058800000FB0360FFF726F82046B9E7E807002091
:10589000F407002094080020F8B5044600284CD0F6
:1058A000026D42B94FF0500383F31188BFF36F8F3D
:1058B000BFF34F8FFEE7C36C994238BF1946C36AE6
:1058C0008B423AD0012A38D11C4A1268824208D150
:1058D0004FF0500383F31188BFF36F8FBFF34F8FE7
:1058E000FEE71426164D826906FB0353002A42691F
:1058F000C162A4BFC1F1070181619A421DD1071D98
:105900003846FFF70AF8E26A0E4C48B901235643BD
:10591000A85903FA02F118B9236823EA01032360A6
:1059200001231420216893400B432360394600FB78
:105930000250BDE8F840FEF7CDBFF8BDE8070020F3
:10594000F407002094080020044B1A681AB1196863
:105950000A6D01320A651868704700BFE807002029
:105960002DE9F041214C1E4680460F46154600F0B9
:1059700089F9236893F88434022B16D00121236817
:10598000D3F8802422EA0802C3F88024236883F82D
:10599000841456B13046FFF7A9FB4FF08052144BE8
:1059A0001A60BFF34F8FBFF36F8F00F08DF900F0D7
:1059B00069F91DB12368D3F880342B602368002275
:1059C00093F88434022B09BF012500252368D3F8FE
:1059D000801404BFB943C3F88014236883F8842477
:1059E00000F072F92846BDE8F08100BFE80700200A
:1059F00004ED00E0F8B50F4616461D46044640B9D2
:105A00004FF0500383F31188BFF36F8FBFF34F8FB5
:105A1000FEE700F037F915B1D4F880342B6002238B
:105A200094F88454721EEDB284F88434032A0ED89C
:105A3000DFE802F002080514D4F880140F43C4F81C
:105A4000807404E0D4F880340133C4F88034012D2C
:105A500008D0012500F038F92846F8BD022DEED116
:105A60000025F7E7261D3046FEF757FF1349E26A87
:105A7000086805FA02F3034314200B60104B31460B
:105A800000FB0230FEF726FFA36A43B14FF050033C
:105A900083F31188BFF36F8FBFF34F8FFEE7094B7E
:105AA000E26A1B68DB6A9A42D3D94FF08052064BF8
:105AB0001A60BFF34F8FBFF36F8FCBE794080020BE
:105AC000F4070020E807002004ED00E02DE9F8438A
:105AD000089F894690461D46044640B94FF0500342
:105AE00083F31188BFF36F8FBFF34F8FFEE700F092
:105AF000ABF9EFF311864FF0500383F31188BFF336
:105B00006F8FBFF34F8F15B1D4F880342B60022311
:105B100094F8845408F1FF32EDB284F88434032AF7
:105B200009D8DFE802F0020F1715D4F8801441EA13
:105B30000901C4F88014012D0FD0012086F31188CB
:105B4000BDE8F883D4F880340133C4F88034F2E738
:105B5000022D33D0C4F88094EDE7A36A43B14FF02F
:105B6000500383F31188BFF36F8FBFF34F8FFEE7AE
:105B7000134B1B68DBB904F104084046FEF7CDFE69
:105B8000104A1420E36A11689D400D434146156098
:105B90000D4A00FB0320FEF79DFE0C4BE26A1B68DA
:105BA000DB6A9A42C9D901202FB13860C6E704F1F7
:105BB00018010748EFE7074B1860BFE70020BDE773
:105BC0008C08002094080020F4070020E80700203B
:105BD000C80800200C090020002382B001930D4B5F
:105BE0001B68013308D04FF0500383F31188BFF3D3
:105BF0006F8FBFF34F8FFEE74FF0500383F3118891
:105C0000BFF36F8FBFF34F8F019B002BFCD002B00F
:105C1000704700BF1801002006480068006880F344
:105C2000088862B661B6BFF34F8FBFF36F8F00DF96
:105C300000BF000008ED00E04FF0807340F8043C26
:105C4000054B21F0010140F8081C40F80C3C40F8DD
:105C5000202C4038704700BFD95B000800000000CE
:105C6000074B19680868B0E8F00F80F30988BFF3A4
:105C70006F8F4FF0000080F311884EF00D0E7047CB
:105C8000E80700204FF0500383F31188BFF36F8FB4
:105C9000BFF34F8F0A4A13680133012B13600DD1F4
:105CA000084B1B6813F0FF0F08D04FF0500383F32D
:105CB0001188BFF36F8FBFF34F8FFEE7704700BFB0
:105CC0001801002004ED00E0084A136843B94FF0C2
:105CD000500383F31188BFF36F8FBFF34F8FFEE73D
:105CE000013B13600BB983F3118870471801002042
:105CF000EFF30980BFF36F8F0D4B1A6820E9F00FA7
:105D000010602DE908404FF0500080F31188FFF734
:105D10000DFC4FF0000080F31188BDE808401968C1
:105D20000868B0E8F00F80F30988BFF36F8F704701
:105D3000E807002008B54FF0500383F31188BFF344
:105D40006F8FBFF34F8FFFF7C5FA18B14FF0805236
:105D5000024B1A60002383F3118808BD04ED00E0B4
:105D60000023084A084913600B604FF47A71074B0F
:105D70001B68B3FBF1F30649013B0B60072313607B
:105D8000704700BF10E000E018E000E05C03002076
:105D900014E000E013B5274B00211A78D2B201922B
:105DA000FF221A701B78244ADBB28DF803309DF86D
:105DB000033003F0500313700722204B1A609DF844
:105DC0000300541E00060DD401B11A601A68032A9C
:105DD00011D04FF0500383F31188BFF36F8FBFF3DF
:105DE0004F8FFEE79DF8032001215200D2B28DF8BB
:105DF00003202246E3E70024120202F4E0621A6064
:105E0000019B0C4ADBB213700D4B1A6842F470020E
:105E10001A601A6842F070421A60FFF7A1FF094B3E
:105E20001C60FFF7F9FEFFF781FBFFF7D5FE204668
:105E300002B010BD00E400E01009002014090020A9
:105E400020ED00E018010020EFF305830F2B0ED9A1
:105E5000104A9B5C104A12789A4208D94FF05003BE
:105E600083F31188BFF36F8FBFF34F8FFEE70B4BA8
:105E70000B4A1B68126803F4E063934208D94FF0A1
:105E8000500383F31188BFF36F8FBFF34F8FFEE78B
:105E9000704700BFF0E300E0100900200CED00E0C7
:105EA000140900201C4A70B5530708BF14464FF070
:105EB000000318BFD41D1949194818BF24F007045E
:105EC00020F007050C604B601649C5E900332B1B19
:105ED000C4E9005302F580560D60A21ADD21A0F638
:105EE000F87002F0BEFF05F10800321A0E4EDD21F7
:105EF00002F0B7FF65683268ED2125EA0202083A30
:105F000004F1080002F0ADFF084B1D60084B1D6056
:105F10004FF00043336070BD481100202809002075
:105F200040210020180900201C090020240900201D
:105F30002009002010B4124B1A6882421ED35C68FC
:105F40001919884201BF4168184609195960446807
:105F500001198A4207D10B4909688A421FBF51685B
:105F600012680919416002604268984218BF1860BF
:105F7000083AFD21083010BC02F073BF1346DBE77E
:105F800028090020180900202DE9F041374D04466A
:105F9000FFF798F92A680AB9FFF784FF344B1F68A6
:105FA000274205D0FFF728FA01F0B0FA00254EE0AD
:105FB000002CF7D004F1080358071CBF23F0070397
:105FC0000833002BEED02B4A166890469E42E9D348
:105FD00029490C6862689A4201D22068A0B92868F1
:105FE000A042DFD02068D21A102A0D68086012D9AA
:105FF000E01841070BD04FF0500383F31188BFF333
:106000006F8FBFF34F8FFEE721460446E2E7426001
:106010006360FFF78FFF194962680868B61A47EA9C
:1060200002038642636020464FF0000322EA070223
:1060300038BF0E60083540F8083B083ACD21C8F853
:10604000006002F00EFFFFF7D7F9002DACD06B0710
:1060500008D04FF0500383F31188BFF36F8FBFF365
:106060004F8FFEE72846BDE8F08100BF18090020E9
:106070001C090020200900202809002024090020F4
:1060800010B5044670B3184A50F8043C1268134225
:1060900008D14FF0500383F31188BFF36F8FBFF324
:1060A0004F8FFEE750F8081C41B14FF0500383F3C7
:1060B0001188BFF36F8FBFF34F8FFEE723EA020310
:1060C00040F8043CFFF7FEF8084A54F8043C116815
:1060D000A4F108000B441360FFF72CFFBDE810404B
:1060E000FFF78AB910BD00BF1C090020200900205D
:1060F00037B502AC04F8011D85694FF0FF3301226A
:106100002146A84703B030BD70B5044608460D4689
:10611000FAF728F8A669024629462046B446BDE8A3
:1061200070404FF0FF3360470149FFF7EDBF00BFFC
:10613000F994000870B5064604464D1E15F8013F57
:106140004BB102F063FE2B78184442785207F5D524
:1061500004F8013BF2E72370A01B70BD08B50A49A3
:10616000FFF7D2FF4FF4FA70FEF79EFBBFF34F8F9D
:106170000649074BCA6802F4E0621343CB60BFF3E1
:106180004F8F00BFFDE700BF1B95000800ED00E04A
:106190000400FA051FB50446684602F00FFD694683
:1061A0002046FFF7B1FF04B010BD0378302B04D1B7
:1061B000437803F0DF03582B06D0431E0A2100204A
:1061C00013F8012F92B97047421C002012F8013FCA
:1061D00003B97047392B4FEA001002D8303B1844FE
:1061E000F4E7462B94BF373B573BF8E7303A01FBC7
:1061F0000020E5E730B5044685B008460D46F9F7BE
:10620000B1FF0A2806D920461F49FFF77DFF00206D
:1062100005B030BD294601A8FFF78CFF082805D03E
:1062200019492046FFF770FF0120F1E70024FBF732
:106230002DF921460DF10A008DF8004002F018FDFD
:1062400021468DF8020002A88DF80A4002F010FDE8
:1062500021468DF8010001A88DF8084002F008FDE4
:10626000303022468DF8030069460848FBF7C4FF2A
:106270000A210648FCF79CF90A2140F480420348B1
:10628000FCF782F9D0E700BF16930008C821002070
:1062900030B5044685B008460D46F9F763FF082877
:1062A00006D920461E49FFF72FFF002005B030BD5C
:1062B000294601A8FFF73EFF20F00200042805D080
:1062C00017492046FFF720FF0120EFE7FBF7DEF834
:1062D000002102A802F0CCFC00248DF80200214627
:1062E0000DF106008DF8084002F0C2FC21468DF841
:1062F000010001A88DF8064002F0BAFC04A922466C
:1063000001F8100D0748FBF721FE0A210548FCF7AC
:106310004FF90A2140F480420248FCF735F9D3E7EF
:1063200031930008C82100200149FFF7EDBE00BFEE
:10633000DE9200080149FFF7E7BE00BF1393000893
:10634000F8B504460D461D4E29B30B78ABB10A22B1
:106350003146284600F01CFD431C0ED00C2303FBE5
:10636000006081682046FFF7CFFE2046FFF7DCFE85
:106370002046FFF7DFFF0020F8BD2B785BB1104906
:106380002046FFF7C1FE29462046FFF7BDFE0D4916
:106390002046FFF7B9FE0C492046FFF7B5FE002561
:1063A0000C2707FB05F32046F158FFF7ADFE01353A
:1063B0002046FFF7B9FE0A2DF3D1D9E774960008FD
:1063C0008B94000899940008B094000810B5044616
:1063D00001F0E4FE2046FFF7ADFF002010BD0000F5
:1063E0002DE9F04F044687B00D4649B95649FFF7ED
:1063F0008BFE2046FFF79EFF012007B0BDE8F08F1F
:106400002846F9F7AFFE8046023000F0C3FD0027B2
:106410008146B84525DC0A2309F80830002308F135
:10642000010A802009F80A3000F0B4FD0646CDF8D4
:106430000C9005AB04AA5146039802F0E8F8F8B1B5
:10644000304600F0A9FD484600F0A6FD284600F0C1
:10645000B8FC05460028D3D12046FFF76BFF28463D
:10646000CBE7EE5D02F0D2FC33463044427802F0D6
:106470000302012A08BF203309F807300137C8E7B3
:10648000DDE90403A3EB000B8023304A0093594657
:10649000334602F0F9F8B0F100084EDD06EB0803D0
:1064A00013F8013C042B07D9032206F80820022226
:1064B00008F10103F25490445A46A7694FF0FF33A4
:1064C00004992046B84722492046FFF71DFE37466B
:1064D000B346B0441BF8011B20460909092994BFA3
:1064E00030315731FFF704FE1BF8011C204601F044
:1064F0000F01092994BF30315731FFF7F9FD2021F1
:106500002046FFF7F5FDD845E4D12046FFF70CFE05
:106510000F492046FFF7F8FD17F8011B0D4B2046E9
:1065200003EB8101FFF7F0FD20212046FFF7E0FD9E
:10653000BB45F1D12046FFF7F7FD059B039A039376
:106540009A1AAAEB020A74E757960008404001081D
:1065500088940008EC9600082DE9F04F814685B03C
:106560000C4649B93D49FFF7CFFD4846FFF7E2FE2B
:10657000012005B0BDE8F08F2046F9F7F3FD824613
:10658000023000F007FD00270646BA4526DC4FF032
:106590000A0306F80A304FF000030AF101088020D0
:1065A00006F8083000F0F6FC3746054603AB02AAB1
:1065B0004146384602F02BF8F0B1284600F0ECFCDA
:1065C000304600F0E9FC204600F0FBFB04460028C2
:1065D000D2D14846FFF7AEFE2046CAE7E55D02F09D
:1065E00015FC2B462844417801F00301012908BF1E
:1065F0002033F3550137C8E78023029803990093AD
:10660000174A2B46091A02F03FF8B0F1000A05DCE0
:10661000039BDF1BA8EB07081F46C7E705EB0A0330
:1066200013F8013C042B07D9032205F80A200222A3
:106630000AF10103EA5492444FF0000BBAF1000F43
:10664000E6D0514605EB0B0001F0D0FDBAEB000A95
:106650008344DDD0C820FEF727F9EFE73D96000818
:106660004040010837B504460D46F9B91A49FFF70D
:106670004BFD2046FFF75EFE012003B030BD392BF5
:106680001ED9462B8CBF573B373BDBB21B01392A47
:10669000DBB217D8303A1344DBB28DF80730012152
:1066A0000DF1070001F0A2FD88B102352B7813B17E
:1066B0006A78002AE3D12046FFF73CFE0020DCE7A1
:1066C000303BE2E7462A94BF373A573AE3E73220B5
:1066D000FEF7EAF8E3E700BFFC9400082DE9F84F65
:1066E00004460D4641B94E49FFF70EFD2046FFF71F
:1066F00021FE0120BDE8F88F084600F062FB064647
:1067000010B948492046EFE72846FFF74EFD82467C
:106710003046FFF74AFD074608B94349F2E7B0F5AE
:10672000005F01D94149EDE741492046FFF7ECFC04
:1067300040492046FFF7E8FC0026BD1B102D0AEB60
:106740000609A8BF1025CB464FF008084FEA1B7278
:10675000092AD1B294BF303157312046FFF7C8FC27
:10676000B8F101084FEA0B1BF0D133492046FFF77F
:10677000CBFCA8451BDB25EAE578C346BBF10F0F30
:1067800033DD20212046FFF7B3FC4FF0000BAB4573
:1067900032DBB8F10F0F3CDD20462E44FFF7C4FC7E
:1067A000B742CAD82046FFF7C5FD0020A2E718F877
:1067B000091008EB090B0909092994BF3031573139
:1067C0002046FFF795FC9BF80010204601F00F01D2
:1067D000092994BF30315731FFF78AFC2021204628
:1067E000FFF786FC08F10108C3E714492046FFF7CC
:1067F0008BFC0BF1010BC1E71BF809102046A1F13E
:1068000020025F2A88BF2E21FFF772FC0BF1010BDB
:10681000BDE720212046FFF76BFC08F10108B8E72F
:10682000819300089C930008B4930008D893000853
:10683000FD930008399400088894000887940008A4
:1068400010B5044600F0F8F940B105492046FFF7BD
:106850005BFC2046FFF76EFD002010BD0149F5E707
:106860004A9300086193000810B5044600F088F9C7
:1068700040B105492046FFF747FC2046FFF75AFD87
:10688000002010BD0149F5E7C9940008DE94000816
:10689000F0B585B004460D4600F06EF90746002DB0
:1068A00040F0A480914E2A4669463046FBF7E4FB4F
:1068B0002A4601A93046FBF741FD8D492046FFF7E6
:1068C00023FC9DF80710042201F5FA612046FFF72A
:1068D00061FC2D212046FFF70BFC02229DF80510DC
:1068E0002046FFF757FC2D212046FFF701FC02222E
:1068F0009DF806102046FFF74DFC20212046FFF7AB
:10690000F7FB02229DF800102046FFF743FC3A21D6
:106910002046FFF7EDFB02229DF801102046FFF70D
:1069200039FC3A212046FFF7E3FB02229DF80210D2
:106930002046FFF72FFC2046FFF7F6FB33681B6865
:106940009B0726D52B462A4602A93046FBF72EFD8B
:1069500068492046FFF7D8FB02229DF80810204620
:10696000FFF718FC3A212046FFF7C2FB02229DF8F0
:1069700009102046FFF70EFC3A212046FFF7B8FB2E
:10698000204602229DF80A10FFF704FC2046FFF77C
:10699000CBFB59492046FFF7B7FB3B79012B1AD0B7
:1069A00014D3022B19D02046FFF7BEFB53492046D3
:1069B000FFF7AAFB7B7993B1012B15D02046FFF797
:1069C000B3FB2046FFF7B6FC002024E04C492046EC
:1069D000FFF79AFBE7E74B49F9E74B49F7E74B49E4
:1069E0002046FFF791FBE9E74949F9E7284600F01F
:1069F000E8F9064688B947492046FFF785FB29464E
:106A00002046FFF781FB44492046FFF77DFB2046E7
:106A1000FFF790FC012005B0F0BD29463F48F9F78B
:106A200097FB40B931462046FFF7E4FB3C4920463E
:106A3000FFF76AFBC5E729463A48F9F789FB20B911
:106A400031462046FFF724FCF0E729463648F9F79F
:106A50007FFB70B9304600F0B4F9054608B93349F8
:106A6000D2E731462046FFF7C5FB0028DED0294695
:106A7000E7E729462E48F9F76BFB78B9337803F03E
:106A8000DF03432B01D13871D0E7422B02D1012320
:106A90003B71CBE7542B14D10223F9E72946254853
:106AA000F9F756FBB8B9337803F0DF03502B03D165
:106AB000787101F08FFBB9E7532B02D10120787177
:106AC000F7E71D492046FFF71FFB31462046FFF739
:106AD0001BFB1A4998E71A492046FFF715FB294680
:106AE0002046FFF711FB17498EE700BFC8210020A1
:106AF00027950008339500084F9500086B9500080E
:106B0000589500086095000867950008759500087D
:106B10007E950008889500088D950008A9950008C5
:106B200036960008B2950008AE950008B7950008A3
:106B3000DF950008FC950008E5950008F895000829
:106B400003960008189600080020094B09491A68A6
:106B5000B2F1FF3F0AD0012A07D103F108028A42AD
:106B6000184600D170471346F1E70020704700BF78
:106B700000FC0108000002080048704730090020AE
:106B800070B586B0FFF7E0FFF8B9214B214A1968CC
:106B9000013102D110339342F9D11F4A934229D8CF
:106BA00000250195F9F78AFD0123194C01A902A8D6
:106BB0000295CDE90443F9F753FEB8B1F9F790FD1A
:106BC00000F030FA002006B070BD124B00F1100545
:106BD0009D42E5D810F10804E2D0F9F76FFD0F4EA1
:106BE000AC420AD3F9F77CFD0120ECE7F9F778FD18
:106BF0000B4DF2E70A4D064CEFE756F8042F002341
:106C000021460220F9F7A0FD0028D7D10434E7E798
:106C100000FC010800000208FFFF01082C09002009
:106C200008FC01080122034B1A6000221A715A71F4
:106C3000704700BF3009002010B5FFF785FF0446FC
:106C400038B1054B0068616803C3201C18BF0120E0
:106C500010BDFFF7E7FFF8E730090020174B30B50C
:106C6000D1E9005253F8224010F0040F4FEAE40338
:106C700018BF1B1910F0020F18BF03EB640310F0CC
:106C8000010F18BF03EBA40304070D4C4CBFEB1A14
:106C90005B19A342B8BF234647F6FF74A342A8BFBF
:106CA0002346084C0B6054F820000244582AA8BF21
:106CB000582222EAE2724A60184630BDB0990008B4
:106CC0000180FFFF7099000837B502AC04F8011D80
:106CD00085694FF0FF3301222146A84703B030BD3C
:106CE00070B5044608460D46F9F73CFAA669024617
:106CF00029462046B446BDE870404FF0FF33604758
:106D000000222248F8B501261446134617460546C8
:106D1000395C0137202911D006D839B309290DD0A3
:106D2000E954002601331FE0272903D05C2915D040
:106D30002229F5D13AB984F001040CE014B1E954E8
:106D4000013308E00AB1E9540DE0D6B9EE543246F9
:106D5000344601260133802FDAD10CE00CB1C15446
:106D6000EEE782B1C15401330022F4E7C3F180029F
:106D7000184402F076F8002385F87F3085F87E30DD
:106D8000F8BD1446E7E714460122E4E7801000202E
:106D90002DE9F04106460F46154600244FF00C0839
:106DA000AC4202D14FF0FF3007E008FB04F331465C
:106DB000F858F9F7CDF910B92046BDE8F081013453
:106DC000EEE760B103784BB103461A780130002A30
:106DD000FAD15B78002B08BF002070471846704737
:106DE00070B50D4616460446FFF78AFF294632461F
:106DF0000F48FFF7CDFF431C01460BD00C48FFF7AF
:106E0000E0FF0C2303FB01514B6801462046BDE81F
:106E10007040184720460749FFF762FF20460449A3
:106E2000FFF75EFF20460449FFF75AFF012070BDBF
:106E3000801000208B940008999400082DE9F743F6
:106E4000254F0446884691463D46244E3B687F2B9D
:106E50002FD8636901220DF107012046984718B920
:106E6000032003B0BDE8F0839DF807100A290FD076
:106E70000AD8082926D02046FFF726FF2B689DF860
:106E80000720F254013325E00D2901D07F29F1E7D5
:106E90000D212046FFF718FF0A212046FFF714FFB7
:106EA00028680021C0F18002304401F0DAFF00239D
:106EB0002B603378002BC9D04A4641462046FFF765
:106EC0008FFFCEE72B68002BC0DD2046FFF7FCFECE
:106ED0002B68013B2B60B9E73809002080100020A7
:106EE000034B0360034B0B6080231360704700BFAC
:106EF000400B00203C09002000224FF400510148C3
:106F0000F9F7CABE0010014001224FF400510148B8
:106F1000F9F7C2BE0010014030B5486085B00C469C
:106F20001546F9F745F92060A847002304AA42F85E
:106F3000043D0A4800924FF4803101220068FEF7B8
:106F4000C5FD039B3BB14FF08052054B1A60BFF368
:106F50004F8FBFF36F8F05B030BD00BF0011002011
:106F600004ED00E038B51468154634B1041B5068D0
:106F7000A04203D2984700232B6038BD0B68001B4A
:106F8000834288BF0860F8E700F04ABF00F028BFDE
:106F900070477047FEF7F8BFFFF772B80846FFF773
:106FA0006FB8000070B5104C88B0264601AD0FCE0A
:106FB0000FC596E8070085E80700002101A8FDF746
:106FC0004BFC0A4B01AD1C3418600FCC0FC594E884
:106FD000070085E80700002101A8FDF73DFC044BF0
:106FE000186008B070BD00BF988F0008F40F002033
:106FF000D80F002000F00EBE00F02CBE002382B09F
:107000000193019B02B07047B0F5006F01D100F011
:1070100077BE704770470368B3F1804F01D1F9F72D
:10702000BBB87047002382B00193019B02B0704748
:1070300010B594B0142200210CA801F012FF142204
:1070400000210DEB020001F00CFF1022002101A82D
:1070500001F007FF02244FF4803305210122CDE91E
:107060000A13CDE911434FF4E0130AA8CDE90D222C
:107070001393FAF711FA08B1FFF7D4FF0F234FF477
:107080008062CDE905340023022105A8CDE907324D
:107090000993FAF749FC08B1FFF7C4FF4FF4807376
:1070A0001122CDE90123002301A80493FAF780FD02
:1070B00008B1FFF7B7FF14B010BD00000024B94AB3
:1070C00080B5D36892B043F08073D360B64BB74DB0
:1070D0005C601A68012742F001021A60F9F74AF869
:1070E00001F05AFBFFF7A4FF2046FEF74DFFFEF725
:1070F000C7FFFFF7A1FD102221460BA801F0B1FE4A
:10710000AB69012243F01003AB61AB694FF400514E
:1071100003F010030193019BAB69A54843F02003E2
:10712000AB61AB694FF0020803F020030293029BAE
:10713000AB69032643F00403AB61AB6903F00403BE
:107140000393039BAB6943F00803AB61AB6903F0A6
:1071500008030493049BF9F79FFD224640F27F1138
:107160009448F9F799FD012202219348F9F794FD1B
:107170004FF400530BA98E48CDE90B370D94CDF891
:107180003880F9F70DFC7F230BA98A48CDE90B372E
:10719000CDE90D48F9F704FC48F280030BA98548B6
:1071A000CDE90B36F9F7FCFB0BA98348CDE90B873A
:1071B000CDE90D46F9F7F4FB40F204430BA97E48F4
:1071C000CDE90B340D94F9F7EBFB4FF4006C7B4BDE
:1071D0000BA97948CDE90BC30D94F9F7E1FB4FF208
:1071E000F8330BA97448CDE90B36F9F7D9FB4FF406
:1071F00080730BA96F48CDE90B37CDE90D46F9F740
:10720000CFFB224605212820F8F7F6FF2820F9F7C2
:1072100037F86B6922463B436B616B6905213B4044
:1072200000931120009BF8F7E7FF1120F9F728F8E9
:107230004FF0FF336248DFF8ACE1ADF81C408DF849
:107240001E400B94C0E900E38460FBF725F908B108
:10725000FFF7E8FEFAF71AF90A215948FBF7A8F9EF
:1072600010F4804240F0D38007A95548ADF81C20A7
:107270008DF81E20FAF76AFE08B1FFF7D3FE514BD6
:1072800000220BA94E480B93FAF7B6FF08B1FFF79F
:10729000C9FE00241022002107A801F0E2FD1C22F3
:1072A00021460BA8CDE9054401F0DBFD0523464846
:1072B000464D8460C0E90053FE238461C0E9033475
:1072C000FBF78EFB08B1FFF7ADFE4FF4805307A923
:1072D0003D480793FBF76EFD08B1FFF7A3FE3A4860
:1072E000FBF7D6FB08B1FFF79DFE002305A9364842
:1072F000CDE90533FBF790FF08B1FFF793FE60215E
:107300008023CDE90B13002308220BA92E480D93EF
:107310000F93FBF763FC08B1FFF784FE2A4800F0E7
:1073200069FB102200210BA801F09BFD00232848D7
:10733000284ACDE90733C0E9002342F227328360AF
:10734000C0E903238361FBF74BFB08B1FFF76AFE3B
:107350004FF480530BA91E480B93FBF72BFD08B18C
:10736000FFF760FE002307A91948CDE90733FBF7B3
:1073700053FF08B1FFF756FE4FF4E1331648174AA2
:10738000C0E9002300230C22C0E902330361C0E9F5
:107390000523C361FCF700F808B1FFF743FE104D69
:1073A0000BAC21E0F0ED00E0001000E00010024026
:1073B0000010014000080140000C014000002110B5
:1073C000C8210020010504144821002000040040C9
:1073D00004110020000800408821002000380140EE
:1073E000D08F00080028004000F0BCFE00F008FC30
:1073F0000FCD0FC495E8070084E8070000210BA813
:10740000FDF72AFA044B1860FDF721FAFEE703485E
:10741000FBF726F83DE700BF00110020C82100203F
:107420007FB501F079F900F0D9F900F041FA2B4B62
:107430002B4A2C481A60FBF79DF908212948FBF7D5
:10744000B5FE08B1FFF7EEFD274C284D2046FBF7AF
:1074500091F9274A00212748F9F7E4F8264A012143
:107460002448F9F7DFF8254A02212248F9F7DAF82B
:10747000234A03211F48F9F7D5F822682149D36828
:107480004FF47A7043F48073D3601F4AFFF744FDD2
:10749000FFF788FD019B00234FF47A724FF0FF3411
:1074A000184E01934FF47A735A434FF0FF31B2FBF9
:1074B000F3F3002002AAFEF753FAF8F779FE04A9C5
:1074C0002B46324641F8044DFFF74CFD40F6B833E9
:1074D000039A9A4288BF0393039AE3E7D40F0020EC
:1074E000044001084821002004110020096F000811
:1074F000896F0008682800208D6F0008936F0008CE
:10750000916F0008C80F0020F96E0008FFF78ABDD0
:10751000002382B00193019B02B070472DE9F04730
:107520000746894616469A46F8F742FE00258046E9
:10753000741B01D120460FE009EB05017B6922464F
:107540003846984784420544F2D0F8F731FEA0EB64
:107550000800504502D9701BBDE8F0870120FDF7F7
:10756000A3F9E5E72DE9F047161E074688469A4637
:1075700003DA0846F8F7F6FD0646F8F719FE002587
:107580008146741B01D120460FE008EB0501BB6862
:1075900022463846984784420544F2D0F8F708FE60
:1075A000A0EB0900504502D9701BBDE8F08701200F
:1075B000FDF77AF9E5E7000010B5EFF311844FF01D
:1075C000500383F31188BFF36F8FBFF34F8F0348CE
:1075D00001F080FB84F3118810BD00BF3C02002045
:1075E0002DE9F0410F461546EFF311864FF0500399
:1075F00083F31188BFF36F8FBFF34F8F0A4801F0F9
:1076000069FB854228BF05460024DFF81C80AC4298
:1076100004D186F311882046BDE8F081391940462F
:1076200001F07FFB0134F2E73C02002010B5EFF3DC
:1076300011844FF0500383F31188BFF36F8FBFF3B2
:107640004F8F034801F040FB84F3118810BD00BF49
:107650003C02002010B5EFF311844FF0500383F388
:107660001188BFF36F8FBFF34F8F034801F02CFBDE
:1076700084F3118810BD00BFCC02002070B5EFF379
:1076800011864FF0500383F31188BFF36F8FBFF360
:107690004F8F064C204601F01BFB0546204601F0AB
:1076A00019FB86F31188281A70BD00BFCC02002098
:1076B00010B5064C0648214601F033FB2146BDE8D3
:1076C000104001220348FBF7CFBE00BFD00F0020BF
:1076D000CC020020882100202DE9F0410F46904681
:1076E000EFF311864FF0500383F31188BFF36F8FD0
:1076F000BFF34F8F104801F0EBFA05460E4801F03A
:10770000E9FA00242D1A454528BF4546DFF82880B0
:10771000AC420BD1094B93F83930202B01D1FFF744
:10772000C7FF86F311882046BDE8F081391940462D
:1077300001F0DDFA0134EBE7CC02002088210020C3
:1077400002680E4B10B59A4211D1EFF311844FF03D
:10775000500383F31188BFF36F8FBFF34F8F084837
:1077600001F0BAFA20B9FFF7A3FF84F3118810BD26
:1077700084F31188FFF740FCF9E700BF00380140AF
:10778000CC0200200268104B10B59A421AD1EFF3D8
:1077900011844FF0500383F31188BFF36F8FBFF351
:1077A0004F8F0A4801F09DFA18B90949074801F0BE
:1077B0009EFA012206490748FBF775FE84F31188FB
:1077C000FFF718FC10BD00BF003801403C0200204C
:1077D000AC280020882100207047000008B506482A
:1077E00001F072FA054801F06FFABDE80840012285
:1077F00003490448FBF757BECC0200203C0200209E
:10780000AC280020882100202DE9F04107460D46D4
:10781000EFF311864FF0500383F31188BFF36F8F9E
:10782000BFF34F8F0A4801F055FA854228BF05463D
:107830000024DFF81C80AC4204D186F31188204676
:10784000BDE8F0813919404601F06BFA0134F2E7E6
:10785000AC0100202DE9F04107468846EFF3118680
:107860004FF0500383F31188BFF36F8FBFF34F8F37
:107870000D4801F02DFA05460B4801F02BFA0024C3
:107880002D1A454528BF4546DFF81C80AC4204D17F
:1078900086F311882046BDE8F0813919404601F091
:1078A00026FA0134F2E700BF1C0100207047704740
:1078B00008B5044801F008FABDE80840024801F0A4
:1078C00003BA00BFAC0100201C010020114B07B51A
:1078D0009A690F2142F001029A619A696FF00100E2
:1078E00002F001020092009ADA6942F08052DA61F5
:1078F000DB69002203F080530193019BF8F77CFCC5
:10790000054A536823F0E06343F00073536003B00B
:107910005DF804FB001002400000014007B5104B69
:1079200002689A4219D1F9F7B1FD0E4B0521DA69C7
:10793000292042F00062DA610122DB6903F0006372
:107940000193019B084B1A600022F8F755FC29208F
:1079500003B05DF804EBF8F793BC03B05DF804FBEB
:1079600000280040001002403C04424237B5036842
:107970001B4A054693420BD11A4BDA6942F00202C8
:10798000DA61DB6903F002030093009B03B030BDB2
:10799000154A9342FAD1134B144CDA69204642F04F
:1079A0000402DA61DB69124A03F004030193019BCC
:1079B0001023C4E9002300238022C4E902324FF4DB
:1079C0008072A361C4E904234FF40053E361F8F724
:1079D0006BFC08B1FFF726FB2C626562D6E700BF9F
:1079E0000004004000100240000800406828002009
:1079F0008000024010B5044686B01022002102A883
:107A000001F02FFA22680D4B9A4214D103F503338B
:107A10009A6902A942F008029A619B69012203F067
:107A200008030193019B0223CDE9022303230448A9
:107A30000593F8F7B5FF06B010BD00BF0004004085
:107A4000000C014010B5044686B01022002102A8A7
:107A500001F007FA22681B4B9A4230D103F55843D4
:107A60009A6902A942F480429A619A69164802F41E
:107A700080420092009A9A69002442F004029A61BE
:107A80009B694FF4007203F004030193019B0223EE
:107A9000CDE9022303230593F8F782FF4FF48063B7
:107AA00002A90948CDE902340494F8F779FF2520AA
:107AB00022460521F8F7A0FB2520F8F7E1FB06B0E8
:107AC00010BD00BF003801400008014010B501465C
:107AD00088B000221C20F8F78FFB1C20F8F7D0FBA1
:107AE000154B01A9DA6903A842F00102DA61DB69EA
:107AF000124C03F001030293029BFAF729F8FAF7FC
:107B000007F84FF08043236040F2E733E3600C4B0B
:107B10004000B0FBF3F00023013860602046236191
:107B2000A360FAF75DFF20B92046FAF74FFE08B0D0
:107B300010BD0120FBE700BF00100240B02800206C
:107B400040420F007047002382B00193019AFCE786
:107B500008B5FFF7F8FF08B5FFF7F5FF08B5FFF721
:107B6000F2FF002382B00193019B02B07047000036
:107B70000148F8F7C3BC00BF682800200148F9F7A6
:107B8000EFB900BFB43D00200148FAF74EBE00BF78
:107B9000B02800200148FBF7E9BC00BF8821002085
:107BA0004FF40060F9F792B80148FAF741BC00BF02
:107BB000C82100200F4B1A6842F001021A60596870
:107BC0000D4A0A405A601A6822F0847222F4803208
:107BD0001A601A6822F480221A605A6822F4FE029F
:107BE0005A604FF41F029A604FF00062034B9A6094
:107BF000704700BF001002400000FFF800ED00E0F9
:107C000008B5FEF7B9FF024B02791A7008BD00BF34
:107C1000F02800201FB50D4B186898B1002304AA66
:107C200042F8043D00924FF480210122FDF74EFFFF
:107C3000039B3BB14FF08052054B1A60BFF34F8F4F
:107C4000BFF36F8F05B05DF804FB00BFD80F0020B5
:107C500004ED00E01FB50D4B186898B1002304AA8D
:107C600042F8043D00924FF400210122FDF72EFF5F
:107C7000039B3BB14FF08052054B1A60BFF34F8F0F
:107C8000BFF36F8F05B05DF804FB00BFD80F002075
:107C900004ED00E0F7B5154D154F164E4FF47A730D
:107CA00001AA4FF0FF310020FDF75AFE0128F5D15F
:107CB000019BD90307D52B782BB93068FEF734FB2D
:107CC0003068FEF737FB019B5A0306D52B7823B9A2
:107CD0003A6809493068FFF7B1F8019CE302DDD545
:107CE000FEF74AFFE4B204712C70D7E7F0280020B9
:107CF000EC970008D40F002074960008704700002D
:107D00001FB50D4B186898B1002304AA42F8043D32
:107D100000924FF480310122FDF7D8FE039B3BB166
:107D20004FF08052054B1A60BFF34F8FBFF36F8F38
:107D300005B05DF804FB00BFF40F002004ED00E087
:107D4000044A00F03F00D3689BB223F03F03034393
:107D5000D36070470008014008B50221002208489E
:107D6000F8F79AFF074B59685A68521A502AFBD9FC
:107D7000BDE80840012202210148F8F78DBF00BF8D
:107D8000000C0140001000E008B540210122084825
:107D9000F8F782FF074B59685A68521AB2F5E16F3B
:107DA000FAD3BDE80840002240210148F8F774BF2B
:107DB00000080140001000E008B5FFF7C1FFBDE872
:107DC0000840FFF7C9BF000008B54FF40061034841
:107DD000F8F750FFB0FA80F0400908BD000C0140F0
:107DE0001FB50D4B186898B1002304AA42F8043D52
:107DF00000924FF400310122FDF768FE039B3BB176
:107E00004FF08052054B1A60BFF34F8FBFF36F8F57
:107E100005B05DF804FB00BFF40F002004ED00E0A6
:107E20007FB5EFF311844FF0500383F31188BFF354
:107E30006F8FBFF34F8F4FF4027000231B4D1C4A0E
:107E4000296800FB01260131012988BF19462960F4
:107E5000184DC6F80032C6F804322B68013B2B607F
:107E6000CBB9154A106890B104AA42F8043D0092BB
:107E70004FF440310122FDF729FE039B3BB14FF047
:107E800080520E4B1A60BFF34F8FBFF36F8F84F396
:107E9000118804B070BD00FB0121094B09481A6824
:107EA000D1F800323C32F8F78FFAF0E79005002065
:107EB00060360020EC0F0020F40F002004ED00E0FD
:107EC00048210020682800202DE9F04F5D4D87B043
:107ED000FDF7D8FE2B68022B04D1FDF7F5FE07B0A5
:107EE000BDE8F08F584B4FF402761C6800930134C4
:107EF000022C28BF00244FF0000BFDF7E5FE66437F
:107F0000DFF864A1DFF86491DAF80030002B43DB7E
:107F1000DFF85C8109EB0607D7F80022B2F5007F95
:107F20003AD24A4AD8F800C052F833104FEA6C00EF
:107F3000085C0192464A1CF0010F114614BF00F084
:107F40000F00001103930292FEF788FE4FF4807138
:107F5000019B90FBF1F01A46D7F800C2039B8038D2
:107F60000CF1010107F80C00C7F8001202EBC30086
:107F7000D8F80010C08801318142C8F800104FF0D5
:107F8000010B029AC8D14FF0FF33CAF8003000232A
:107F9000C2E90033C8F8003009EB0603D3F8003219
:107FA000B3F5007F31D22B4F4FF47A713868FCF76C
:107FB00091FE0128804628D1274800F08DFE002838
:107FC0003DD10290244800F08CFE0DF11701019084
:107FD000214800F0A6FEDDE901239DF81710CAF83C
:107FE000001032B11D4842464FF480310068FDF761
:107FF00001FD4FF00108002338681A461946FCF7C6
:10800000A1FDB8F1000F7FF47BAFFDF73BFEBBF1A4
:10801000000F3FF462AF2B686BB94FF40271009B05
:1080200001FB04911C600E4B0E481A68D1F8003217
:108030003C32F8F7C9F92B6801332B604DE74FF05C
:108040000008D8E7EC0F002090050020043E01084E
:10805000DC0F00208031002070050020F40F00208C
:108060004821002068280020F00F00206036002002
:10807000E80F002008B5FDF705FE1248F8F7F6F9FD
:1080800000234FF0FF31104A1048C2F80032C2F806
:108090000432C2F80834C2F80C340D4A13600D4A99
:1080A00013600D4AC2E900330C4A11600C4A136098
:1080B00080220C4B1B68DA6300F006FEBDE8084026
:1080C000FDF702BE68280020603600207005002001
:1080D00090050020EC0F0020DC0F0020F00F0020A6
:1080E000E80F00204821002007B502A901F8010D82
:1080F000064800F0FCFD0648002301224FF4003141
:108100000068FDF777FC03B05DF804FB7005002004
:10811000F40F002008B5034800F0E3FDB0FA80F04A
:10812000400908BD70050020034B1B780BB9FFF711
:108130002BBEFFF79FBF00BFE40F0020034B1B784F
:108140000BB9FFF739BEFFF7CFBF00BFE40F002028
:10815000034B1B780BB9FFF737BEFFF7DBBF00BF40
:10816000E40F002008B5094800F0AEFD08490120E1
:10817000FCF79AFD074B1860FEF7FEFC064B4279B0
:108180001A70BDE80840FFF7CFBF00BF60030020B2
:108190001036002080310020E40F002010B50B4C79
:1081A0004FF47A712068FCF795FD01280CD108483E
:1081B00000F08AFDFFF7B8FF002320681A46BDE8EB
:1081C00010401946FCF7BEBC10BD00BF8031002036
:1081D0006003002010B50446FFF7E0FF024B1C705F
:1081E000BDE81040FFF7DABFE40F00202DE9F341AE
:1081F0000D460646002845D019B3234F4FF47A7137
:108200003868FCF767FD012819D1204C204600F0A2
:1082100063FD10B9FFF79CFFB8B92C46DFF86C80FE
:10822000404600F059FDD0B9DFF860802644311B8C
:1082300004B3404600F05BFDE8B1013CF7E72C4693
:108240002D1B284602B0BDE8F08120460DF1070144
:1082500000F067FD9DF80700FFF770FFD6E7FFF716
:1082600077FF0028E0D0013C16F8010BFFF766FF0E
:10827000002CD5D10024002338681A461946FCF793
:1082800061FCDDE70546DCE780310020600300206B
:1082900073B51D4D1D4C4FF47A7301AA4FF0FF3199
:1082A0000020FDF75DFB0128F5D1019BDA0317D50E
:1082B0004FF47A712868FCF70DFD012810D1204693
:1082C00000F00AFD90B1204600F006FD00230646AE
:1082D0001A4619462868FCF735FC0EB1FFF70EFD6B
:1082E000019B9B03D7D5FFF7EFFDD4E7FFF730FFE6
:1082F0000028E8D020460DF1030100F012FD9DF8A2
:108300000300FFF71BFFDAE7803100206003002045
:108310006138C3B2182B9DBF0248D84000F001005D
:1083200000207047114110016238C3B2182B9DBF65
:108330000248D84000F001000020704777DF770145
:108340006238C3B2182B9DBF0248D84000F001002C
:1083500000207047251D3101652806D000F0EF0090
:10836000A0F169035842584170470120704700004E
:1083700020F02003413B192B0ED927280CD021389F
:10838000C0B21E280AD8064B23FA00F010F0010FE5
:1083900014BF022000207047012070470020704762
:1083A00001780046F8B5064653B31C7844B36FF025
:1083B00001050134511E1C44ED1A14F8010DA0F101
:1083C0006103192B03D9272801D0202804D1735C1D
:1083D000834204D1013910E0242802D16AB100207F
:1083E00022E023280ED1705CFFF792FFE0B1013943
:1083F000705CFFF78DFF0028F9D12B190133DCD118
:10840000012011E03A2808D17718B91B17F80109A3
:10841000FFF78AFF0028F8D1EFE75E2805D1705CEE
:10842000FFF782FF0028D5D1F8BD2E2803D1705C5C
:10843000FFF786FFF6E72B28D1D1705CFFF78CFFA2
:10844000F0E72DE9F84306461F4653B193F8009034
:10845000B9F1000F05D014469846A8EB07039945DB
:1084600001DC012035E018F8013FA3F16100192873
:1084700003D9272B01D0202B04D1305D984257D14E
:10848000651C04E0242B04D18A4251D125462C4698
:10849000E3E7232B0BD1305DFFF73AFFC8B1651C32
:1084A000705DFFF735FF0028F1D00135F8E73A2B72
:1084B00008D13444A51B14F8010BFFF735FF002841
:1084C000F8D1E4E75E2B06D1305DFFF72DFF0028E1
:1084D000D6D1BDE8F8832E2B03D1305DFFF730FFF6
:1084E000F5E72B2B03D1305DFFF736FFEFE7252BA8
:1084F0001ED1335D652B11D1651C735D6C2B05D1CD
:1085000033199B78792BC2D1E51CC0E7A3F1720027
:10851000012801D9642BBAD1A51CB8E7692B07D172
:10852000651C735D6E2BB2D133199B78672BEBD032
:108530000020CEE700EB41035B8830F81100181AE9
:10854000C008704730F8111001EBC20292B28118D6
:10855000825A02441A604A8802445A608A88024455
:108560009A60CA881044D86070472DE9F04F85B0F2
:1085700006460F4618460E9990469A46FFF7DAFFD0
:1085800000258346DDF840905D4501DB012031E0A8
:108590006B462A4650460E99FFF7D4FF019B44468E
:1085A0001A461878BC42A2EB030101D2884224D8B3
:1085B00088422AD1009B424639463046FFF7F2FEF8
:1085C00018B3029B224639463046FFF73AFFE0B126
:1085D000039DD9F800302A78934203DB691C0F9879
:1085E00000F034FC2A78D9F80030A4EB08009B1A7C
:1085F000C9F8003005B0BDE8F08F16F804C012F8D5
:10860000011F8C4501D10134CCE70135BCE72DE9D0
:10861000F84317461E46054620B12AB15BB9002330
:108620003B6001E0002AFAD116B90220BDE8F883C8
:1086300000233360F9E7002902DAF7F793FD0146DA
:108640002A46884600248C4291461AD099F80000A8
:108650000132FFF78DFE90B12246A85CFFF788FE3D
:1086600010B101328A42F8D315444445C7F800904E
:108670003560DAD0A2EB080358425841D6E70134FE
:10868000E1E72246A046EFE72DE9F04FB1F10009FE
:1086900087B0824693461F4602DAF7F763FD8146AC
:1086A00000252C460DF11408A94503DC204607B02F
:1086B000BDE8F08F1AF8056000F0A8FB334630449F
:1086C0004278494602F00302012A08BF2033A3F191
:1086D0006102D2B2192A9ABFDBB2603B0023002CA0
:1086E000B4BF0026109A0093A8BF161B5B462A460B
:1086F000CDE9017850460596FFF737FF059B054405
:10870000002B05DA002CA4BF002427461C44CBE72D
:10871000F61A37443444C7E708B500220E490F481B
:10872000FBF7FDFC08B1FEF77DFC0D490B48FBF79C
:108730000BFD08B1FEF776FC0A490848FBF7B6FCCA
:1087400008B1FEF76FFC0548FBF705FD18B1BDE861
:108750000840FEF767BC08BDA8050020703A00205D
:1087600008000020940500200020704710B5074C39
:10877000002207492046FBF7A0FC06492046FBF7EC
:10878000A2FC2046FBF7B9FC002010BD703A002087
:10879000743D0020343D0020002382B00193019BF2
:1087A00002B0704770477047222810B50C460AD1B6
:1087B0004AB9488800F00100FFF7F4FF608800F034
:1087C0000200FFF7F0FF002010BD000070B5044666
:1087D0000E46084D01462846FBF775FC2846FBF778
:1087E0008CFC31682046FFF735F8FFF75FF8002072
:1087F00070BD00BF703A002038B50D4DD5F8B832C5
:108800005B6D9BB940210B48FEF7FEFF044648B163
:1088100082B208492846FBF750FC2846BDE838409C
:10882000FBF756BCFFF743F8204638BD0120FCE7B4
:10883000703A0020743D002000210846FFF7DCBF9D
:1088400007B50E4B02689A4215D103F5DA33DA699F
:10885000052142F40002DA61DB69002203F400031F
:1088600001931420019BF7F7C7FC142003B05DF8B7
:1088700004EBF7F705BD03B05DF804FB005C0040B6
:1088800000F50C71D0F86802FBF77CBC00EB4113DB
:10889000D3F83C21D0F86802FBF7A1BC00EB4113F0
:1088A000DA6BD0F86802FBF7D4BCD0F86802FBF7AB
:1088B00068BD836810B5022B044601D0FEF7B2FBF9
:1088C000D4F868020121FBF746FDD4F86802BDE840
:1088D0001040FBF719BD000010B50446D0F868023F
:1088E000FBF73CFDA36923B1024A136943F0060379
:1088F000136110BD00ED00E0D0F86802FBF737BD52
:10890000082310B51D4A04461D48C0E90023022370
:1089100083600023C4F8C002C0F86842C0E906338F
:108920000362F8F7DFF908B1FEF77CFB0022182399
:108930001146D4F8C002F8F790FD58230022802198
:10894000D4F8C002F8F789FDC02300228121D4F8B1
:10895000C002F8F782FD4FF4887300220121D4F899
:10896000C002F8F77AFD4FF4807300228221D4F818
:10897000C002F8F772FD002010BD00BF005C00408F
:10898000B43D002008B5D0F8C002F8F72DFA03284E
:1089900096BF024B0220185C08BD00BFE7640108C7
:1089A00010B51C46D0F8C00213462246F8F747FA25
:1089B000032896BF014B0220185C10BDE764010834
:1089C00008B5D0F8C002F8F76DFA032896BF024B3D
:1089D0000220185C08BD00BFE764010808B5D0F8A4
:1089E000C002F8F7D3FC032896BF024B0220185CA4
:1089F00008BD00BFE764010808B5D0F8C002F8F769
:108A0000F9FC032896BF024B0220185C08BD00BF8A
:108A1000E76401080A06D0F8C03245BF01F07F01C3
:108A200003EB411303EB411393F82A0058BF93F86B
:108A30002A01704708B5D0F8C002F8F7ECF903280E
:108A400096BF024B0220185C08BD00BFE764010816
:108A500008B5D0F8C002F8F76DFA032896BF024BAC
:108A60000220185C08BD00BFE764010808B5D0F813
:108A7000C002F8F740FA032896BF024B0220185CA8
:108A800008BD00BFE7640108D0F8C002F8F74BBA90
:108A900000487047F80F00207047704712230148C4
:108AA0000B807047C4050020042301480B807047E9
:108AB000D8050020002370B51E46050FECB2092D25
:108AC00094BF3034373401F8134001EB43040133D1
:108AD0006670DCB2A2424FEA0010EED870BD000012
:108AE0001A2310B50B80094B186808331B68C0188F
:108AF0000AD0074B08221C680649FFF7DBFF042257
:108B000005492046FFF7D6FF044810BDE8F7FF1FD0
:108B1000ECF7FF1FDE050020EE050020DC0500203D
:108B200010B5044C0A4604482146FBF732FE2046A5
:108B300010BD00BF204000200465010810B5044CA2
:108B40000A4604482146FBF724FE204610BD00BF1C
:108B5000204000201765010810B5044C0A4604485F
:108B60002146FBF716FE204610BD00BF2040002026
:108B7000EB64010810B5044C0A4604482146FBF793
:108B800008FE204610BD00BF20400020F66401080A
:108B900010B558B103784BB102461346197801322B
:108BA0000029FAD10246013B934200D810BD197842
:108BB000147803F8014902F8011BF5E7F7B5151E13
:108BC000064600F1010424DC00291FD01CDA01272D
:108BD0004942354600E025462C460A22684600F008
:108BE000DCF8019B0099303304F8013B0029F2D1F5
:108BF00017B12D232370AC1C002330462370FFF7E0
:108C0000C7FF204603B0F0BD0027E2E73023037022
:108C1000F2E7002920D014DA0127494234460A221B
:108C2000684600F0BAF8019B0099303304F8013B24
:108C3000013D41B930232544A54206D004F8013B4B
:108C4000FAE70027EAE7002DE9D1002FD4D02D2341
:108C5000013404F8013CCFE730232246691E03703B
:108C60000544AA4201D10C44C6E702F8013BF8E7EB
:108C70002DE9F84380460D4607463B787A1C202BA9
:108C800011D03E4600244FF00A0900F0BFF83278B8
:108C9000711C1044437813F0040306D009FB04242C
:108CA0000E46303CF1E71746E7E7BE4206D14DB12C
:108CB0001C46C5F800802046BDE8F883002DFAD098
:108CC0002E60F8E72C46F6E7002303604360704708
:108CD00080687047406870474068B0FA80F040098B
:108CE000704783684068C31A584258417047826889
:108CF000436870B59A42044611D000686668A3685C
:108D00003044E568013B184005FB0040E268103044
:108D100000F09CF8012063680133636070BD00209F
:108D2000FCE710B504466368084683B16368013BFD
:108D300063602168E368E26803FB0141103100F0E1
:108D400085F82368A2680133013A1340236010BDFF
:108D5000002103E00B4B5B58435004310A480B4B96
:108D600042189A42F6D30A4A02E0002342F8043B32
:108D7000084B9A42F9D3FEF71DFF00F023F8FEF7E7
:108D80009DF970474066010800000020C8070020D8
:108D9000C807002020420020FEE710B591FBF2F446
:108DA000002902FB141306DB002B01DA01349B1AA5
:108DB000C0E9004310BD002BC4BF04F1FF349B1871
:108DC000F6E7000070B500250C4E0D4CA41BA41056
:108DD000A54209D100F0C4F800250A4E0A4CA41B94
:108DE000A410A54205D170BD56F82530984701352D
:108DF000EEE756F8253098470135F2E73866010866
:108E000038660108386601083C660108044B054ACB
:108E10001B681B6A002B08BF1346D3F8EC00704791
:108E2000F80500205C06002082B001B901A942B11A
:108E30004BB113780B601278101C18BF012002B0E0
:108E400070471046FBE76FF00100F8E710B5431ECE
:108E50000A44914200D110BD11F8014B03F8014FB3
:108E6000F7E703460244934200D1704703F8011B21
:108E7000F9E738B50C460968054609B1FFF7F9FF6F
:108E800021462846BDE83840FEF788B82C4B70B51F
:108E90001B680446834251D0436A43B1DB68002B10
:108EA0004AD1636A196811B12046FEF777F8616903
:108EB00011B12046FEF772F8616A11B12046FEF743
:108EC0006DF8A16B11B12046FEF768F8E16B11B1A6
:108ED0002046FEF763F8216C11B12046FEF75EF8DC
:108EE000E16D11B12046FEF759F8A16D11B1204690
:108EF000FEF754F8616B11B12046FEF74FF8A369F5
:108F0000E3B1A36A20469847A16CB9B12046BDE8F9
:108F10007040FFF7AEBF495941B90435636A802DEF
:108F2000D968F8D12046FEF739F8BAE70E6820462E
:108F3000FEF734F83146EFE70025EFE770BD00BFDC
:108F4000F805002049B1FF2A8BBF8A230A7003600D
:108F5000012088BF4FF0FF3070470846704700007F
:108F6000F8B500BFF8BC08BC9E467047F8B500BF16
:088F7000F8BC08BC9E467047E6
:108F780002030405060708090A0B0C0D0E0F101052
:108F880002030405060708090A0B0C0D0E0F101042
:108F9800209B0008918200080200000000000000E9
:108FA80080000000802F002088310020149B0008DA
:108FB800957C000800000000000000008000000010
:108FC800802D0020F82800202B9B00082174000821
:108FD800000000000000000080000000DC210020EC
:108FE800E02300202E2E2F447269766572732F536A
:108FF800544D3332463178785F48414C5F4472694A
:109008007665722F5372632F73746D3332663178BD
:10901800785F68616C5F636F727465782E63002E89
:109028002E2F447269766572732F53544D3332462E
:109038003178785F48414C5F4472697665722F5386
:1090480072632F73746D3332663178785F68616C40
:109058005F646D612E63002E2E2F447269766572EF
:10906800732F53544D3332463178785F48414C5F03
:109078004472697665722F5372632F73746D33323D
:10908800663178785F68616C5F666C6173682E63BF
:10909800002E2E2F447269766572732F53544D3308
:1090A80032463178785F48414C5F44726976657220
:1090B8002F5372632F73746D3332663178785F681B
:1090C800616C5F666C6173685F65782E63002E2E35
:1090D8002F447269766572732F53544D333246317B
:1090E80078785F48414C5F4472697665722F537295
:1090F800632F73746D3332663178785F68616C5FA3
:109108006770696F2E63002E2E2F44726976657220
:10911800732F53544D3332463178785F48414C5F52
:109128004472697665722F5372632F73746D33328C
:10913800663178785F68616C5F7063642E63002EB7
:109148002E2F447269766572732F53544D3332460D
:109158003178785F48414C5F4472697665722F5365
:1091680072632F73746D3332663178785F68616C1F
:109178005F7263632E63002E2E2F447269766572C8
:10918800732F53544D3332463178785F48414C5FE2
:109198004472697665722F5372632F73746D33321C
:1091A800663178785F68616C5F7263635F65782E9B
:1091B80063002E2E2F447269766572732F53544DB7
:1091C8003332463178785F48414C5F44726976653E
:1091D800722F5372632F73746D3332663178785FF0
:1091E80068616C5F7274632E63002E2E2F4472695F
:1091F800766572732F53544D3332463178785F4811
:10920800414C5F4472697665722F5372632F737491
:109218006D3332663178785F68616C5F7274635F52
:1092280065782E63002E2E2F447269766572732F2F
:1092380053544D3332463178785F48414C5F44721D
:10924800697665722F5372632F73746D333266318A
:1092580078785F68616C5F74696D2E63002E2E2FBD
:10926800447269766572732F53544D3332463178A0
:10927800785F48414C5F4472697665722F53726318
:109288002F73746D3332663178785F68616C5F7400
:10929800696D5F65782E63002E2E2F44726976659E
:1092A80072732F53544D3332463178785F48414CAE
:1092B8005F4472697665722F5372632F73746D33CE
:1092C80032663178785F68616C5F756172742E639D
:1092D8000049444C450057656C636F6D6520746F99
:1092E8002074686520426C756550696C6C53503009
:1092F800323536414C3220436F6D6D616E642050BB
:10930800726F636573736F720D0A003E20006461AB
:1093180074652072657175697265732079797979D8
:109328002D6D6D2D64640D0A0074696D652072657C
:109338007175697265732068683A6D6D3A73730D5B
:109348000A0073657474696E67732064657065726A
:109358007369737465640D0A004661696C656420FD
:10936800746F2064657065727369737420736574B3
:1093780074696E6773210D0A0064756D70207265DB
:1093880071756972657320616E20616464726573BA
:10939800730D0A0064756D70207265717569726568
:1093A80073206120636F756E740D0A00746F6F20EF
:1093B80066657720627974657320746F2064756DB3
:1093C800702E202031202D20383139322E0D0A0000
:1093D800746F6F206D616E79206279746573207483
:1093E8006F2064756D702E202031202D2038313982
:1093F800322E0D0A0020202020202020202020307E
:109408003020303120303220303320303420303595
:109418002030362030372030382030392030612055
:1094280030622030632030642030652030660D0AB9
:10943800002D2D2D2D2D2D2D2D20202D2D2D2D2D9B
:109448002D2D2D2D2D2D2D2D2D2D2D2D2D2D2D2D44
:109458002D2D2D2D2D2D2D2D2D2D2D2D2D2D2D2D34
:109468002D2D2D2D2D2D2D2D2D2D20202D2D2D2D3E
:109478002D2D2D2D2D2D2D2D2D2D2D2D0D0A002091
:1094880020200054686520636F6D6D616E6420272D
:109498000027206973206E6F74207265636F676E92
:1094A800697A65642E0D0A0068656C7020697320FE
:1094B800617661696C61626C6520666F723A0D0A4B
:1094C8000073657474696E6773207065727369736D
:1094D8007465640D0A004661696C656420746F20C8
:1094E800706572736973742073657474696E6773D9
:1094F800210D0A00277068272072657175697265E9
:10950800732061206865782073657175656E636581
:109518000D0A007265626F6F74696E670D0A0064E8
:1095280061746574696D653A2020002C206E657839
:1095380074207363686564756C656420616C61721E
:109548006D2061743A20006D6D6F64653A202000CB
:10955800636F6D6D616E6400627269646765007443
:1095680074730073706D6F64653A202000706879B9
:10957800736963616C0073696D756C61746564000F
:109588007365742000207265717569726573206156
:109598002073657474696E672076616C75650D0A51
:1095A8000064617465006461746574696D65006464
:1095B80061746574696D652072657175697265732A
:1095C80020797979792D6D6D2D64642068683A6DFC
:1095D8006D3A73730D0A006D6D6F646500756E7278
:1095E80065636F676E697A6564206D6F64652700CF
:1095F800270D0A0073706D6F6465006572726F7273
:109608003A20207468652073657474696E67200059
:109618006973206E6F7420612076616C69642073B1
:10962800657474696E67206E616D650D0A00646FFC
:109638006E650D0A0027737027207265717569724F
:10964800657320736F6D6520746578740D0A002743
:109658007474732720726571756972657320736FEE
:109668006D6520746578740D0A000000F097000895
:1096780091680008F49700083A980008696800089B
:109688001E980008389800084168000842980008A9
:10969800609800085D6100086798000879980008DC
:1096A800DD6600087E9800089A980008656600083C
:1096B8009D9800082E99000859650008C19800086F
:1096C80067950008E1630008EB98000829990008ED
:1096D800CD630008319900084999000841630008E2
:1096E8004E9900085041310050413200504133003A
:1096F80050413400504135004F5900004159000095
:10970800454800004B4B3300505000004A480000C9
:109718004E4E310049480000545432005252310034
:10972800415800004D4D0000545431004448310068
:10973800495900004559000044443100555731004B
:10974800414F000041410000595932004145000095
:109758004848310042423100544800005548000052
:109768005557320041570000444432004747330000
:109778005656000047473100534800005A48000039
:1097880052523200464600004B4B32004B4B3100E0
:109798005A5A00004E4700004C4C00005757000032
:1097A80058520000574800005959310043480000FA
:1097B80045523100455232004F57000044483200AC
:1097C800535300004E4E3200484832004F520000BA
:1097D800415200005952000047473200454C0000F2
:1097E800424232000A0000007365740073657420F9
:1097F800612073657474696E672076616C75652C79
:10980800206F72206C69737420616C6C20736574AE
:1098180074696E6773007065727369737420736519
:109828007474696E677320746F20666C6173680066
:1098380064657065727369737400646570657273CA
:109848006973742073657474696E67732066726FC8
:109858006D20666C617368007265626F6F74007268
:109868006573746172742074686520626F617264D4
:109878000064756D700064756D70206D656D6F7234
:10988800793B205B616464725D205B636F756E7405
:109898005D0070680073656E642070686F6E656D3A
:1098A800652073657175656E6365205B68657820F2
:1098B8006469676974735D2B00646F2074657374E1
:1098C8002D746F2D7370656563683B20656E636CDE
:1098D8006F7365207465787420696E2071756F7474
:1098E800657300646F20646961676E6F7374696380
:1098F80020746578742D746F2D7370656563683B8B
:109908002064756D702067656E657261746564208A
:1099180070686F6E656D652073657175656E6365DA
:109928000072657365747370007265736574207472
:109938006865205350303235362064657669636532
:109948000068656C70006765742068656C70206FCE
:109958006E206120636F6D6D616E643B2068656C7D
:1099680070205B636D645D00FFFFFFFFFFFFFFFF7B
:10997800FFFFFFFFFFFFFFFF0200000004000000E1
:109988000600000008000000FFFFFFFFFFFFFFFFC9
:10999800FFFFFFFFFFFFFFFF0200000004000000C1
:1099A8000600000008000000070000000800000092
:1099B800090000000A0000000B0000000C00000075
:1099C8000D0000000E000000100000001100000053
:1099D8001300000015000000170000001900000027
:1099E8001C0000001F0000002200000025000000ED
:1099F800290000002D0000003200000037000000A0
:109A08003C00000042000000490000005000000037
:109A180058000000610000006B00000076000000A4
:109A2800820000008F0000009D000000AD000000D3
:109A3800BE000000D1000000E6000000FD000000AC
:109A480017010000330100005101000073010000FC
:109A580098010000C1010000EE0100002002000092
:109A68005602000092020000D40200001C0300000D
:109A78006C030000C3030000240400008E040000EF
:109A8800020500008305000010060000AB06000078
:109A98005607000012080000E0080000C309000093
:109AA800BD0A0000D00B0000FF0C00004C0E0000A7
:109AB800BA0F00004C11000007130000EE1400005C
:109AC8000617000054190000DC1B0000A51E00004A
:109AD800B621000015250000CA280000DF2C000070
:109AE8005B3100004B360000B93B0000B24100007A
:109AF800444800007E4F0000715700002F600000AE
:109B0800CE69000062740000FF7F00007461736B0F
:109B18004D6F6E69746F72007461736B535030329D
:109B280035360064656661756C745461736B00FF4B
:109B3800FFFFFF4F2720EB986100B993108A81300F
:109B4800D9A017198B8840918A21AC900620ABA127
:109B58000401B99310C9A3A7BF721AE9A3501BA99E
:109B68000590890219C9914498A9813A00B238DA56
:109B7800996301AD911209B81393E0C386F2501EA0
:109B8800AA06018B894080A8210CA91261A8A912F4
:109B98002A0A9339E991531ACA02111BC9331A9D2B
:109BA800826DD711ABCA5481AA9139099131BD99F7
:109BB800245998A804890A021AB9A4728BB80230E9
:109BC8009BB9710A0E114F1501DAB97208B98408E8
:109BD800898228CA90261A8A8022A1AA23ABCB8719
:109BE800609AA012008BB312A1F806BE7019BBB61A
:109BF800382BAA159099121AC98144998B01398872
:109C0800B051BABA3758A9B13188AB050088E10517
:109C1800F2580CAC06108B894080A8210C9A03607E
:109C2800A0B8122B1AA429C9B0631AAB82311AFA48
:109C380021180D806AF7009ABA4581AA914908A1AE
:109C480022BBB9273A89A013890E130AABA3738ADA
:109C5800B903280AC83103AF887F2481DAA87108BC
:109C6800A994080A8228CA9036098A8021A1B934A1
:109C78009BCA064099B92301AD921001F804BF7040
:109C880019BBB5482BA9149099122BCA8245999AE9
:109C9800013981E120A9A927289BA12281BD83112F
:109CA80088F015F2481DBB17108B89408898228CC4
:109CB8009A0360A0A9121A0B9439BAC0541AA07753
:109CC8007FFF777AF9A52BA271AA9208B0231A0B05
:109CD800A180B5222CA928BAB52288049A88A9405F
:109CE800B02A0B1701F3FB778C88838A9538AB0170
:109CF80008D122988B188005109A1A9D0003010933
:109D080095AAA6009989A1A012137CF660CB093206
:109D1800BB272AB9210B8231C0B818896101B8A1C3
:109D28000C8151AAA140B97109A9A1901868013FF5
:109D3800F718D80820A94499A0188B114888B08032
:109D480091408A0290F8128999142DA3409A88911B
:109D580098B858289F772DB0922BA1729AA200B973
:109D6800223A8C828895399B180AD204099935BD04
:109D78000329A930890AA5D085FA758D88028A95A4
:109D880039AA0209C113989A18892608900A8D825F
:109D980021899050D9158A9018888B32C950F6615C
:109DA800CC09219A1719A9101B9122B0A8299061F2
:109DB8008891999D202189816AC032AA910198AB26
:109DC8006B0A7F9758D88029994499A0108B01492C
:109DD80088A189825888009AC0221A8A252F91481A
:109DE8008A008099B33A951F672DC1A309A1719A7A
:109DF8009101B9212A0B818805191B189AD20208EA
:109E08008C35AD04198A18080BA59887F9748E88C3
:109E1800028A84499B0208C112988A008823809884
:109E28000C8C111180B170DA2509A818809A32B00B
:109E380051F574DB0922AB1729AA201C9221A8A886
:109E480018905180B298BB40110AA36AE8419890D3
:109E580000909A4A8B7FA758D88028A94489B010C7
:109E68000D102888A00882380891C9A833008C15DD
:109E78002F91488A008098902C958F671CB0922A61
:109E8800B1729AA101B9223CFFFFFFFFF87918804F
:109E9800C0704A0F9082221B1C810091A982293D23
:109EA8009003268C8C083181AA8121109C00010224
:109EB800F981398E0AF7151ABF900411988B10088A
:109EC80080A812801F801313D9AB31591AD00121F1
:109ED8001B8B095819AA852A1F2F8714A8FA18223C
:109EE80020A0B818081A982193BD203268C8C81253
:109EF800291CA922241ABC08593C89958098BF714D
:109F0800509BF900411988B100918A802011F8010D
:109F1800313D9AB205918BB03511A9D083108B9938
:109F280016B2C4F8714A8FA182220A0B800081AA56
:109F3800201929F183148C8C812181BD8213489EBC
:109F4800880300AA9960990BF71509BF9004119826
:109F58008B181900A811011F902223D99C104800C2
:109F6800C982322ABE0941199B815B1B5F8704980D
:109F7800FA182220A0B818081AA11291AF1021319E
:109F8800D8C912182DA9223489D980580AA8A70837
:109F980090AF61409BF981411989A181918A802103
:109FA80000F801323D8AC104918C902231AAE094D4
:109FB800180B9833D1A4FA71698EA182220A0B80FA
:109FC8000081AA12191BF202130E8B922281DB92D6
:109FD80034209DB01680AA8840980DF61409CF0841
:109FE8000401898A181910B812810E801233D99C7D
:109FF800015900BA02232AAF1A3388BA815C2B3F71
:10A00800A72798EA193220B1C8108009910181A0C8
:10A018000FFFFE80CF9FF53728BFB98236180A8810
:10A0280082A9AB993723888B8A80B20A887A32A0B2
:10A0380099815029D8C809588AC21C7434A9FD8846
:10A048001123000A0A09C0C8805221A0B90B2800B0
:10A05800A1AC3131850AB8700AC9A921126A89CF21
:10A068007332DAFA082421889B0088999A04261802
:10A078000C889100800A908A15813B6882D8AD18B7
:10A088005188B998F37249ADE080313090BA0089AF
:10A0980098994325A0BB1B31138BBB8028790A866E
:10A0A8003208DABD096111AA8F86528BCE8012124E
:10A0B80009888019CC8023118D9085118B9A018293
:10A0C800DA91414119A9AA0BB825488AD03F0771EE
:10A0D800AADB1113118908810AFA002311BA802119
:10A0E80020BBBA1348DC90524808909B9CA34101BE
:10A0F8001C08FF7228DAD8303288B888238BD91028
:10A108002498C920429AA981010C9C025308A1B144
:10A118000CAC801708A098F1752BCCD121300AA07F
:10A1280080229CB821419BC111320ACA8042ACC02E
:10A13800217089800091D8083911E81BF7420E9DDB
:10A148008203188A880120CA9002489C9384398B1C
:10A15800B88140D9A133318AAA3AC5CB183021F940
:10A168001F2761CAC92238A0A3212CABA3041C9ABB
:10A178001307099C1211B9AC3020A399444ABBAC0F
:10A188001439B0A007BE5539DAD021298883820C4A
:10A198008C0103AA8A1154A8A94910C8AA4028000A
:10A1A800D21200BF982140E88012C1750DB98421F0
:10A1B800AC1140A9B0222B8CA421AB292311DC00BF
:10A1C8003099C82259B086990989230C88B94CE777
:10A1D80052AEAA3311C91148AAB3021A0F0280A0BD
:10A1E800202981C8822B9CB6022C9971899A915199
:10A1F800AB80114F9732FA983219B1032BAE118305
:10A20800989C2219B30001B9C2230F9B02878910B9
:10A218005989B9A440AD88159B644AEA91328B816B
:10A22800259AC82812A8A0500B9110B93AA24291B9
:10A238008C2B37C981102AA8963DD92042C8661CA4
:10A24800BC0221A91230C9A2389A98A311BC73087C
:10A25800C98A1939280420CB91289E9201430BD82A
:10A26800039FE2759CB82408A80219BA15180A0AAF
:10A278009180E0528B9120899A0388901853925FBD
:10A288009A0111E882350F8531DDA03209A1222B10
:10A29800DA3289988A30888373BF8298808902224B
:10A2A80008A05A88ACD138058BB62AAC3769DA02CF
:10A2B800298A1420DB1030BC07199888038AB23128
:10A2C8009AB8529D920222D8219A990242EC922978
:10A2D800E0742CD9130AA8422AD9040AA8221AB071
:10A2E8002123CCB368BA30819D0022180A120FA12D
:10A2F80088281B883BF1770E98228AA2411CA92541
:10A308008BA84189980358AB8410CB032B818D52BD
:10A318009B121A0BC852B990837DA561DA904089C7
:10A32800A332AD9833ABB358A9800529C9328BC87D
:10A33800230B9112A1DC070A810812A9A802DF26C3
:10A3480038DBA3409981629D901189902208CBA5A2
:10A3580040B9248A9099110D121AA41A1CA262C835
:10A3680000B80AB8773BF98138B83412AE9229B8E8
:10A3780080030AC96280A8138E00A91191310E3199
:10A38800CA8A160B320808AEC4729EA81319A826EA
:10A3980018CA20809A02110BB0378C921848CA212B
:10A3A800A2199B3C210AF158092C958A89A760BDFE
:10A3B80080128AA26109C8120BA08248AB9441BCE2
:10A3C80011820B890103D958B318D090032BA60921
:10A3D80018FC4719BB9151AA94318CB042AA891331
:10A3E8002BBC0539BA3002BD01923991C2288DBC07
:10A3F80024B268D039B2BC771BC98238AC16109B1E
:10A408009130AA01021BFA52989001809A93293838
:10A41800890020AF9807092B0280FAA6720F98834B
:10A4280009A03329DC0318A909519AD1300AA103DC
:10A438008C1B9485C0309B41D1A19059A109000F74
:10A44800A741BCA8418AA3331BFA339A880071E05C
:10A4580081192BA491919B310986A8001AC3B86869
:10A4680080A3891C9C3778BC8041AA82519BB1315A
:10A478009B09A728D93002BB106B82BA247FFF7FC3
:10A48800FD773FC91619A81019B8350AC90418A9C3
:10A49800032AC88340BB8812091149BAA023191D91
:10A4A800888D04528FF431BEB8530AA8120CA14308
:10A4B8009BD82309A9348BC81529B90010B91231C2
:10A4C8008B0381EC91609A92139FA778BCA1719A33
:10A4D80080218C9231ADA1328AA0429CA02609B974
:10A4E8000218A80609AA1138C89232AE9014DE558F
:10A4F8000ACB8458A90111BC1338CB92509A8032E8
:10A50800BB91628CA0210AA0359AB0232DB0150BFF
:10A51800C82240FA748CBA1719A80129C9421ACA64
:10A528000338AA0338EA82609B91219A9232AD914E
:10A5380022AD88539CB1214DE450ACA9440AA01126
:10A548001CA1418AC8230AA91609AA0529BA833079
:10A55800BA0439DA0321AD9051AB81231FB768CA19
:10A56800A072A991119C82409BB0428AA0349CA001
:10A57800251AC91218C8141AB92329C9A420CB82CC
:10A5880053DE450ADA8448A90020AC1338CC92403F
:10A598008A9140AA90439BC0221C90348CA0221C14
:10A5A800B0241AD90231FA748CBA0729A80129C92A
:10A5B800331ADA84289A8428CA8350AB91218C8173
:10A5C800509AA1418C98330DA8223CF2520CCC042D
:10A5D80010898120AAA814098880898520A8802D3F
:10A5E800CA2430BD83509E0120BBA2619AA1032FCB
:10A5F800A730ACDA331099851AA991228989889AEB
:10A60800371988921CC92419BC1618B92249CC03D9
:10A6180038AD01039F1720CCC0321899148A9A923A
:10A6280032909A91A1431A8091DF92138BA8440A21
:10A63800B1078CA8051AB82101FA7609BDA321191A
:10A6480098329BBB143099A908A252180A80CA00F4
:10A658000790B12028D217ABAA441A8A9018F4742C
:10A668008BEC0312899130BAB925188B9839823846
:10A6780082908FC0202A8AB7111D1011ADA0230C1B
:10A6880090A03F8771ABDA2312999419BAA22509D1
:10A698008AA108022288BA8BA03051AE94419B1837
:10A6A80068EA9143899A048F25318FE90124089833
:10A6B800A902180B912299F9124119C89893118C83
:10A6C800AA24119A80280DB238B1BF13F87518AFB3
:10A6D800B8125119AA900200AA11210CD815229C6F
:10A6E8009990030089AB3730A98100BEA32A089945
:10A6F8006BF4532AFDA112418A9A802108B81318D5
:10A708008FB12512CAA8001122C8B8510A9820880A
:10A71800BB322B1BB27E87738AFD81132099A90156
:10A728002809B81481CC805220D9A0013009B8A2D8
:10A73800339D000209F083901D91CC73239FC98833
:10A748001222118111AFBC902213090031AAEC9892
:10A75800583809A982003B26219CE819020E10A14D
:10A768007350BEB8904211000920DBCB8352109879
:10A778001801BBADA5212AC89A14111948B0ABF02D
:10A788000C23A819C74248BFB9822212081119FC24
:10A79800B90421399081099BCA226191F8002211DC
:10A7A8008A9AA1AAA33959C84E17421AFC980222BC
:10A7B8001109018CDAA83710898A00108AB9503932
:10A7C8000B998680089310A19F99B04B97807411BC
:10A7D800ADE99832210080009BEB88420209881479
:10A7E8008ACC9141208918AC1A8132611AFA1A80F0
:10A7F80039352881201DE0D88A822127022308DCE8
:10A80800BCAA813440011219ACC8CA9812836122CB
:10A8180089B4AD90909AC2B6052310ADE8A88821F6
:10A828003432200ADC8ABB9329426035811ABFA8DA
:10A83800B8100350202A23D9BE1A99C81724200912
:10A84800CBBB9093152223329ADCCBAAA8422505CC
:10A8580012888D8EA801803123290919AF9A9D1A73
:10A868003A34374099CC8A880312323332B8FBDA4B
:10A87800A0098613303112CAFABA080815334808F5
:10A8880049BEAA889A8356503999E9B90002141129
:10A898002212BEADAAA18232623000A8BEAC892ABB
:10A8A80005323828901D9DA090BA9743610A8BD92C
:10A8B800B8111202335218BBEBBD1A0582043011CD
:10A8C80089CADCA8018215214009B2FB898C881647
:10A8D80044100B9EA990021104301389ABFE9918FD
:10A8E80002313220198F8ACAA111213701101B8821
:10A8F800FA98B0D12526209ABCBA819242386121B3
:10A908003BBFA9C9085020122188ABAFD98082303B
:10A91800260290899EB0A8891A653319ABDCA880F5
:10A928002022240611AABCD9A1A421220123A3F91B
:10A938009D909810137218118ABF8A99AA8743426A
:10A9480009ACD998910114324119ABEBBC0093338F
:10A958003242210EE8BA98011317111088BAF98B00
:10A9680001891736108B0E9A90020100611119AAFD
:10A97800DBAA2912278410398AABEA981A420710F1
:10A9880018298CDA899A93544420A9AFAA80002206
:10A998002361188ACAC9B8095121429388AE9CA973
:10A9A8008101593314B38B0FC0A09A94454110C943
:10A9B800CA9A0820232172049BABDAA18142114173
:10A9C8002290EA8B990B8368513A12A8BFA9A899DB
:10A9D800973441089EC8A8081133160200ABEC99B9
:10A9E8000983233313192DE9C0B0910512402B2098
:10A9F800BAD8888D891272411B0F9AA01802324565
:10AA08001198ACCBAA892252271200998FD98008B5
:10AA180022150189880BF09889896136188ABD9AB0
:10AA28001120130811508B9CDAA00B50304212A150
:10AA38001DDCA091001074000289CD88FFFFFF7F04
:10AA4800F958BF711A9BA418D81610A98029CC826E
:10AA580040988401AB98301C0021A9C185908121C0
:10AA68002E9A1081D19494F1628C9D111AC04408D9
:10AA7800A8810AD902488B2311E8A2289A18488C81
:10AA880080149882200DAB201A0A426FD611A9BAF9
:10AA9800410F815109A8029BE8141999322BBB85F3
:10AAA80000B0022ABD0140B01410AD98280B88529E
:10AAB8003FB741D8D112BB05318B9830BFA124884C
:10AAC800B1320D9A310AA2048AC9321C003280E9D7
:10AAD8009128A89416FD611A9BA410E81410999166
:10AAE80029CC8141999412ABA8588A0013ABD22281
:10AAF8009A02588ABA858898A603FA738C8E121B14
:10AB0800B05318B9830BEA03598A1311D9A3289BA8
:10AB18002848AC9412B803398DA8119988217FF57B
:10AB280011A9BA518D81410999129BE814089A41DB
:10AB38001AAA0480B0022BBD2239B025889C993806
:10AB48008A19614FA731E8C112C9FFFF78FF7772F0
:10AB5800ED904119A8048AB92628BCA03419A0018F
:10AB68001DA90532BE992318991118DC83420BDA06
:10AB78000221E1520BFA83318B9841BB90632BE998
:10AB880091419880018D983439CC88222990229C53
:10AB9800DA14318CB9132EB7400CD904209A8039B5
:10ABA800BB94628BCA8421990011BF91333BEA811F
:10ABB800328A92119EB83440AD98121E15209FB863
:10ABC8001420AA922AAC86319DA90420988829CA03
:10ABD80083630BDA93328A9121BFA03528CB902367
:10ABE8008D5239EC9041199A138BB94538DAA8344B
:10ABF8000988111CC802619CA92328A80229EB8294
:10AC0800440ABAA232F0631BFB82322BB932BBC0B2
:10AC1800552ACBA2428888018CB92731CBB8251890
:10AC280099021ACA02530DB98349B5319FBA360041
:10AC38009B9258A892229E981419B880419A9834E9
:10AC48001DB91261AC91320CA80140BA00248F964C
:10AC5800209DC85108AA85198A8141BB99441AA91F
:10AC68009260AA88348CA80448BB81348BB9153902
:10AC7800E88024CB621ADB9629992218FA1230BB95
:10AC8800952AAA1440BC8121AA0519CA8341A98121
:10AC980010DA8422ABA1108AF4729EA9258980213A
:10ACA8000DC0331BB9249C90351AC9031AB0528BB6
:10ACB800D91518A9120AC91420AB00098F8758BBE7
:10ACC8009962A88131AFA1418AA031BB92630DA0DE
:10ACD800110B9341ACC84209A0229DA0421AC81189
:10ACE8008A9F649AA1884C8419B28B280408C02CC6
:10ACF800921923AA39F119030B0BF050A11982AC50
:10AD0800119259C18994E973BA08C41D130A93C8EA
:10AD180029120BC48C039130D01C938833C92DA3FE
:10AD280038920A3AF930020C94BA12F659B91A96BE
:10AD3800A9519A18B208319D11D930022CA38E025C
:10AD48008229D00B040913AA1CC229249D28A83ED5
:10AD5800872BA21D18C231C0599090809868A029ED
:10AD6800A00823AB40C01AA88863BA43AB8939C985
:10AD7800629A009CBF769A829B2D8508822C8888CF
:10AD880090843BA31C909050A21A91AD00A2789198
:10AD980039A8981BC558B01991F9709018B38F2924
:10ADA800819408102D80A0AC40A16090288BD21C03
:10ADB800938812129A2CB10B9B658A21C04AF32DF5
:10ADC800100903F01A191490821F0900B038A43A28
:10ADD80003991E81BA48A24080041F818AA031A924
:10ADE80070901F07A8188A39D3902A218294D81CFA
:10ADF80008B40A141A30B2AD29E02983080311DC1B
:10AE080038BA0229A74C829C31D30B020F03C11018
:10AE18009030B915F938A01000010889D14CA41C4C
:10AE2800038902A012AD83B994010850F86A82AA76
:10AE380025CB78A101A1199038F03BA30809130B81
:10AE4800B9178F13BA32A9210A919C23D832C904A1
:10AE58004AF30B59B050E12C01199219904DA5995C
:10AE6800028800119A9823FB60B030A028A838D037
:10AE780039A80922018F07C04B924DA799011A02E0
:10AE88009A830F02A820901019A29979E22BA41A8C
:10AE9800931A938BB33F940910198D78C38B130FB2
:10AEA80013D8128B319904DA59A12982188818C14C
:10AEB8002EA40B138A1498918A05F811892088C248
:10AEC8007D12B914CA599120A858A938F11A8209D3
:10AED8001288890AD68C128A21A83089A4A91AD383
:10AEE8003AC350A9D70C48B840D12A010AA509800D
:10AEF8003E949A22B92218B92942FC31A018002B95
:10AF08008839E049A119011D8B37B16C914BC6995D
:10AF18001019828984AE12C020A1118901BA79D191
:10AF280028928A1389A14CB32C13BC420BAB72F242
:10AF380009828F13B8128B40A925E938B31A8319EF
:10AF4800A119D23F948B02290198908A87AB22A934
:10AF580061B8B55F029902FFFFFFFEFF97094A1A21
:10AF680039A4A9018C309200A78A028D01B008A7E4
:10AF78000B238901B11F920B948812B25AA32D8218
:10AF8800BA02F26B907B20A820E84A811A13B832E3
:10AF9800F83BA28A06A950A12A94AB12CA58A22942
:10AFA800958B31BB5AA12F9788948B4A911AC40A62
:10AFB800110A69A13BB30D108948C329A21C31F0BD
:10AFC80018B03A018A71B848B02D108F41A887B1DE
:10AFD8001B820D849801812C830D829B39916B848F
:10AFE8000A039A3BC22DB409118069B24AC2898109
:10AFF800EA709968A29911BC41B110A58B23CB3195
:10B00800E018921D32AA32D01B849C04A811A33FD9
:10B01800038C83B000F34C805C11B010C04A8119D6
:10B0280013C958C83AA38A15B960A029A3AB32EA54
:10B0380040A118869B32BB39C22FA788948A4AA19F
:10B048002AD40B110938B25BC22E109820C32A9358
:10B058002D01B839E03A020A42E848A82C000F410D
:10B06800A805C11B010D04A811A13C848C03BA39A1
:10B07800905B960A03A93AB22DB58912A869A23C39
:10B08800929B22FA788948A4AA21AD489108948B0A
:10B0980023BC31E109930D32A940B1FFFFFFFFFF47
:10B0A800500808080881880A1181A20D2000D2984A
:10B0B8001A0128B270BCA530CB19448F812B07A187
:10B0C800A4AA4A9839D308021920C01BA08F129A43
:10B0D80041933BA60D189889A41B132B22182EA167
:10B0E8000F801F419887B28B821E83A012A13993CB
:10B0F8009CA6C9109839869013BA29A9AA97A814AA
:10B108008849100D84BB84F8790A5993B802AC3089
:10B11800A040A22A10CA30F829A23A33B132F00B63
:10B12800989A13B227A40810AD01D894F408907C1B
:10B1380028A001C839812A048919AA6BB30A85890C
:10B1480059003AC2899999490850039810AE3BCAE8
:10B158006D8791B6982A9019D30A030A31A12CC396
:10B168000F828902A32A041D01A998C028827A2087
:10B178008010F01B9838F7FF7F7F45F04D2902E3D8
:10B188008C4A10A20D4993A0093B05E12C2893B1E4
:10B198008829A5B03C12F4A829A6B1009811E30C9F
:10B1A80038B5A01B5B11C20A3B12B86B84A81B6B95
:10B1B80012D2894C1198191A87C11A1882C21B1207
:10B1C800C3A82B17F38B6B10B4A02C3A839A390BB6
:10B1D800698930E392E38A194A94A94A01B4AA7AA0
:10B1E80002E39A6B02B28A5C12D3981A39A4A2C3FA
:10B1F8008C48A292B04D3900A03E20A1882C4A0864
:10B208000019A40F38C4908093C22F38A109821D59
:10B21800028C32E13F3A01B38A5C2880894B11A045
:10B228002A81A6B1919815E849B5A2C23F2881B4F0
:10B238008B498008894A949B6A83D4A84D30C4B14D
:10B248000881C5A019A5A01B5B11A03F4B018A6C02
:10B258004B85D30B3A01A3B194AB7B13F4B12F5AAE
:10B26800A7E30B4994C39A5B10A2894D3B20A10A1E
:10B278005C3992B2092C86C3991092B2896C02A0EB
:10B2880095B85C3B21E38B499291A12B85C04C106A
:10B2980092B4A0080882A949C59911B219E7991072
:10B2A800A2A38D48A2901D5A95B03D20A28A3C3099
:10B2B800C3993B20D38A3A4E3A00A49910903D296D
:10B2C80096B05F4B03D2893C12D4A81A39B7C38A07
:10B2D8004A84D38A4C38901B3A18810D30B5B3C3D1
:10B2E800A193F3B5C20A298082A811B11C5D38A1C7
:10B2F8004E101C208C6B181982980081C4A001E4A0
:10B30800A10B49B7B11A2994C21B119A380B07B976
:10B318007B0298000A20A03C181985D3B20E6A93C4
:10B3280098008913DA68B491B07C119081991198CA
:10B33800190949B200B15C831CB78A07D119800189
:10B34800D38A1190801B87D30D4A82B39A7C3981A6
:10B358008A4D3982A01A3B04D20A1A4A95B3C21CF4
:10B36800390A398803AF7B1080A30F4992A2A86CD1
:10B3780012C2983D20A2892C3A02992A2C48B15D24
:10B3880011B4D4993B0018B309948F5992B4B05DA5
:10B3980030C4A82B38B6A95C2881900A4A0082C21A
:10B3A8008B5A02C6C11A02B29818A7C39B69929019
:10B3B8000911E30D4A83D30D5B01900C7D38918808
:10B3C8001C6B03C2892B05F5A0092A84B1093F39F2
:10B3D80093C38D6C02A10B6B03D20A3A84D21C284A
:10B3E80092A10B59A3995C20C4981900901A109443
:10B3F800E13E12C292A000A2A4B838A1A7E22D2073
:10B40800A2A10C48B4981B49B7993A0895C12D399F
:10B4180082B21F4991929B7A95B0191A12C03D28A1
:10B4280081A12B97B0289800B40C4B4981B7C11B58
:10B438003B499288922F20B193B87C21C4B11C3A21
:10B4480082B48B6A83B1894C04C188FFFFFFFF79FE
:10B458006AB5B29A394C13A199588D2808B021C8F9
:10B468004829A329E0100C950A08020D218B094AE6
:10B478000F42F2A3082F10A2C1019B6881A218B83D
:10B488004A1C8119B4011D122C91029F12988281C5
:10B49800BB6090A211FD790883A2BB7A199391C170
:10B4A8004A19830AC4888B048B8492AA349B12A1FC
:10B4B800F950A80100C14990A489F42D2B4882F2C3
:10B4C8000B3C1008B5092B210C02B2B931AE318200
:10B4D800C121C9201BE239A83909B72B8821AFC778
:10B4E80080883A2DA5B189383C23B2A929CE398163
:10B4F800B332A86818D10BC8182B862881309D82D2
:10B50800ACA9480F43C3B4080F10A1C2818A708048
:10B518009100D01B19A311B5102B948CA090AC35B9
:10B528008813019B59C9B21AFB701884A3CB6A0906
:10B538009282C2391A848BD3991D121995839A2243
:10B54800DA91A1CA70081281B83ACB9698F33C4BAD
:10B558003081F10A1C2019A6081B118C82B1AA514E
:10B568000A2303F838BA0890E140884088B32E8B44
:10B578002818FFFFFFFFFF0A08063A8E123D48A36E
:10B58800C6D21D4B2994D4900A4A1994C2A11C3BD7
:10B598005A82A3A0913F2900A3A3C03A1A11A2F38B
:10B5A80090A29F7B4A20E6C01B4C3994B3B22D3C35
:10B5B8003992D4A0803D2902B2A3AB4A2A01A6C27F
:10B5C800800A3A08B7B3D4D30B4B6D21D4B29A5C36
:10B5D8004981A4A18A5C2A11B2B5993C4A0093C258
:10B5E800881C293AA5A2A02A3F209881F7B2A22F49
:10B5F8005C01B4C3994B3B22C3D3992D4A0803D2AB
:10B60800902C2A39A3B3B02A6D2800A2919B7B2BDA
:10B618005E30B4B6D21D3A18A6D4881B4A18B6B202
:10B62800A12C1A48A3C4A0082C1882C3A3A94A3B7A
:10B6380002B4F209801F7C2A21F6C01B4C3995B34D
:10B64800B12C3C3992D4A0803D2902B2A39B5B3B2C
:10B658008295E2800A3909A7B2B5D30B3C7D12D393
:10B66800A19A7D4900A5A18A4B3C12C2B48A2B5AE3
:10B678000083D1882C293A93A3C1192F398882F7DE
:10B68800C3A21F5C02B4D49A5B3B12B4D2881D4A91
:10B698000884C2902C2A39A3B3A93A6D2800A29134
:10B6A8009B7B2B6D30B4B6D12D4B18A6D4900A5A7B
:10B6B80018A5B2B12C2B48A3C5A0082C1882C29299
:10B6C800993A3C02A3F389901F7C3A21F6C01B4C9F
:10B6D80039A5B3B22C3D2881D4A0884C2902B2A345
:10B6E8009B4B4B8294D2800B381AC7A1B5D31C3B15
:10B6F8006D12D3A18A6D4880A5A18A4B2B13D2B4B1
:10B708008A3C4A0083D1882C293A93A3C02A3F2037
:10B718009881F7C3A21F5B01B4D4A95B3B12C3C3D2
:10B72800992E4A0884B1912C2A39B4B4A9294D39E3
:10B7380000A281AB7A2C4D31C3B6D12D4B18A6D4BB
:10B74800881C4908A5B2B13D2B48A2A4A0094C18F1
:10B7580082C292993A3C02A3F288881F7C3A21F669
:10B76800C01B4C39A5B3B22C3D3981D4A0884C29D3
:10B7780002C2A39A3B4A9294D2800A391AB7B3C438
:10B78800D30B4B6D22E4B18A6D4880A5A18A4B2B5F
:10B7980013D2B48A3C4A0094C1801C292993A3C1BE
:10B7A800192F288801F7C2A30F6C01B4C3995B2A2B
:10B7B80012B4D2892D4A0884C2902B2A39B4B4A96C
:10B7C800294D2800A281AB7B3D4C30B8FF777773B9
:10B7D80057FF19289013282930E98C88A0002438AD
:10B7E80040049BA9C99C829141232120BA0FAABD7C
:10B7F8001CF710090830F9882A912482885AB1A9BF
:10B808000C981113836931B90BD9BA20D3583280F7
:10B818003A8A8F0B8B2F972299106DB1A38C113117
:10B8280002A32F08B88C828022051838B89F98A8E0
:10B8380018158041808A20DA9AA3FF511098048F46
:10B848008882B803203886AA0AB1CA100140338515
:10B858001AA8BD8BA29B53042112988AF8BB11FC2D
:10B8680071188815DA1A28B014102932F08B08B923
:10B8780000033160049989BBBE00A169132811A98E
:10B888003CBCB90EF6101A0030F9802C91238109BE
:10B898006A90990CA00112125A43B90CA0AE0893F1
:10B8A8003924282A000E9BA80FB73299027CC1922E
:10B8B8008B013282A51C88B09D818121051848A87A
:10B8C8009B99E909041041038910BEAB80FF51011F
:10B8D800A0840F8802B8022810869A0A91C9080223
:10B8E8001225933B98DA8BC09A53824112A880F9AB
:10B8F800BA01FA7229A116DB1920C013182A41C807
:10B908008B09D818121050850A89B89CA1A0501329
:10B918002239929CDAC91FF510090021F9802B9170
:10B9280024818859A0A98BA00042825937998B801D
:10B93800BB2AB179222119809EBA800FB732A8118B
:10B948006DB1A38C013102A42D88B19C8802230516
:10B958000868A88A9ABA0A070841028819BCAD8102
:10B96800DF6100A0030F9083B9023018079A0AA17B
:10B97800BB00123127833AA0D99AC88B349252124D
:10B98800A088F8B982FA71299016CB1A38C0140029
:10B998001932D88B09C808213050850A09C89BA0DC
:10B9A800C050041039800ACBD82EF510090831F997
:10B9B800802B9123820979A1AA1CA00022115A4345
:10B9C800A98AB8DB88B45822112B18AC8FA81F8716
:10B9D8000299015CB0938C013102B52D80B19C8035
:10B9E8000111131870B09A8AC90985104202880893
:10B9F800CBBF81CF610098030F9802B9133828870D
:10BA08009A0A90C900021116932A98D98AC19A34C1
:10BA1800925112A009E9C881F970299105CB09381A
:10BA2800C013282A42D88B19C808213050868909A2
:10BA3800B88C989868032120909AF9C01DF51009D0
:10BA48008030F8882B9124818859A0AA1CA0002254
:10BA5800216933BB1D98AB0AB63925012A009CA879
:10BA6800FF77FC7D38E01009A78A212809D21F86B4
:10BA780000AA8959B588882018A2B18E1C020A32FA
:10BA88000862CA280BBAA289531122E83AB9C80039
:10BA9800BD8307AE7108A0A12E0981823A9401C224
:10BAA800D03AA010920801A8462F0190A1828E11C9
:10BAB80021D8399982103AD1E3520D9912BB292B1A
:10BAC8009749092909A98E80011050812910AFC111
:10BAD80099810228252BC2AA32AB5FB25BD61089A6
:10BAE8008A13C8A00201A871990A04AA1908A049D2
:10BAF8000C4229A20CC481A10893B5C1080419B14C
:10BB08009F3F8523D99829B4C101139082C8AB956A
:10BB1800C08110121B4A019FC82A0A1602A3C290AC
:10BB2800D100A802CA53AF6118C8A23D9983130077
:10BB38009248E0A01099D231B28321A8991F892197
:10BB48001C9C2266C1889818C10898D4611CA984D5
:10BB58009A0A828341921C10BBBB80D29433251968
:10BB680080E8B39D2AA244B358A92B889C89917B6D
:10BB7800F611899A03B8A95001A02239AF01980A91
:10BB880030798A185B00A385A09C11B101B397ABEB
:10BB9800953994FA1B3710AA0B49B3C0802213A019
:10BBA800C50D99A29B60219820008B8F8080B85288
:10BBB80003A23DA0801B4FB315CB7308B9914D0963
:10BBC8008201398010B2DB22F28921018A02E80C55
:10BBD8004A2B220C008094DB4A9036D93899D5300C
:10BBE8001ABC822E2C028309103D018AC902B14178
:10BBF80004192889D898B492C249001D6299B38C57
:10BC0800A9205EB7319A8B23E890191490012B8EE6
:10BC180001991A31959B28893B398080808C304B5B
:10BC28008C798F833D9188AE6382CA8910E2A11016
:10BC3800201300C18BDC0399944828318B3FA0B0B6
:10BC480030D300831B8478A30BBE9324DE60088066
:10BC5800A12D0B8210390018B2FA39A1881C509115
:10BC680003A0AE190A15888F2308E03A9A31B22F3B
:10BC780092B5682C09828D1A208480100C0199BA1B
:10BC88000803483282C319AF0F010093080139C86D
:10BC9800080F9B121E0CC740898912E99028108151
:10BCA80058A92B019A2E8850A9021B3BC72AA0022B
:10BCB8003AD9861C8088322BA41F8FA733D9005D00
:10BCC800B1930C286082B21D1B91B0884823941A46
:10BCD80020C0BAA0BC4B2780282089A1BC0BB3EF99
:10BCE8007100A0018F88019914181913BC0A80BD2E
:10BCF80002101846901A809D88B109368139018A48
:10BD080098F8A883F872199004EB0938B03411191F
:10BD180041E88A88C821820071908A18DA0902A04D
:10BD280061828019A80CB8BB5DF6200A0848F8881B
:10BD3800199132029069B89A1D9010118458009890
:10BD480089F09929924012913AA88E0D901F070206
:10BD580098804DB1A28A024110A51B99A09F911805
:10BD680020061918808DB1B01C142828138AA8BD84
:10BD78008F81AF710090921F9801A8033018069A1E
:10BD88009991DA82011955901880BC08B1AB54809A
:10BD98002032B980F8B982F9722A8815DC1910B0F6
:10BDA80024010932D89A09E810028060818808D9EC
:10BDB8000A91C051811049991BB9F82AF6110A084D
:10BDC80030F9892A8042029069A8990CB118228416
:10BDD8006901808BC88B1AD35001022B900E8BA857
:10BDE8003FA732A8806CC1A28A014101941C88C077
:10BDF8008C801011870928819D91B08B86101013B3
:10BE08008998CB8E81BF7281A0830FA082A913313C
:10BE180018879A90FFFFFF7FF860A3F34A983F00C6
:10BE28008A3018102CA10D00100B689828B28019C0
:10BE3800940F000A1020084C928B80111E389C6DBC
:10BE4800C718A3AC20C11118100D01B91813A97A8D
:10BE5800811B02A20B23FA39A02860A32F818A80B4
:10BE680029196B1C5F33AA04E818A2028011AC18C8
:10BE7800C18822C41D119A30918820F01B9318188C
:10BE880027BA21D91398B79893FB729A4AB20C0231
:10BE9800118110D00B92803B07B821C84888932D98
:10BEA800A28AA4119060E010B812B015D085F23AB9
:10BEB800984D81992028101AB29E10802B68B13AAB
:10BEC800C31909048F019A2389025CA21BC2398A0B
:10BED80078A95CD708929B10C12018110C81D81042
:10BEE80081907B811B84888821EA48A94009130F27
:10BEF800018B822A916B096F24A983D01AA302822D
:10BF080001BB3AF10802B50C12AB41909038F10927
:10BF1800B2480925CA22BB0599868A84DB718B4AF7
:10BF2800A20C11100010D82C10FFFF63FFFF7951ED
:10BF3800B1F1982A192204090BC899890117131A13
:10BF48000B8AA8D809143104A81A898F90934992AA
:10BF5800B494F87A6A1C82C289002024A08C898A49
:10BF68008082258588899B88A189513002E10981D1
:10BF7800E888105A008089F7950A1F1982A0922034
:10BF88005881B999B90A11713291A8BA8F8891125A
:10BF9800226B10098AE091011A6A802F07A6A1C8AE
:10BFA8002C289002023A88D889A88112504098A873
:10BFB800A1AE098222122C49982EA89214A00A2414
:10BFC800BF7841B0F1A93B1833060A2BB99A98A259
:10BFD80027232B1A9AA8F909032214A11898CF89A4
:10BFE8000120A4A007F14A6B2D82C288083013B043
:10BFF8008C8A8A81813407090A8A19C088122970B3
:10C00800A28901D90A015C109038E58493DA8A087C
:10C018001932023484BCCA8A392A1064201AC98A9F
:10C02800A09C00237010198AAAF0A01B79292D3230
:10C038004291FBA9821A31524081D9A9C808010549
:10C0480023291BA1D8D0C810412830809A0F9A9074
:10C05800A60002AC71692CB0B801911235304ACCF7
:10C068009A91A8032532109E98A0B8D03143A10A0E
:10C0780018A9B1C8190790B5F383392F8B0988011E
:10C08800135402A99D9C0908010723088B88F99974
:10C09800801853148299B9F9988830316884C79107
:10C0A800BA8C080120133223C8F9B9990A315324EC
:10C0B800828AAC8BCBD8835051101098FB9A1829E0
:10C0C800226C502108F9A8800811433209BAEAB055
:10C0D800A90115612818A0E8A99800051331283F7F
:10C0E800ABE08881201388706A1DA8B101913142A4
:10C0F800211CACCA88A0011734080A8CA8C8992842
:10C10800344304A088AFBA80149314F402299F9A88
:10C11800801082142112ABBDAB2E00021416918A36
:10C128000D0A0A9191502133C2AACE899030125932
:10C13800A706A1BC8B280810431312DABAC80D0849
:10C1480011434391D0B89A9F01832031598998CDE2
:10C15800990239107B602190FAA0018001512129B0
:10C16800D9AAA0C2A01432701AA1E099A801031597
:10C17800112A1BABF9BA06802399706A0BC8A081F3
:10C18800839433383CABDC09B3A22712208B2BC92C
:10C19800C8D109521382080C8DB9B0149327C40270
:10C1A8002B1FAB0810011522018C9D998B081307D2
:10C1B80024908A1D0C0AA101503102A2BD9E89A2B9
:10C1C800401840D79391DA89081828333313F9AB0C
:10C1D800989B3E215123A3D8AA0B9B01946149380F
:10C1E80000C8CBA98241286D4032A0FBA080101165
:10C1F800423139D9E8A0A8983261580898D0A8AA3D
:10C20800101512214A1BB9FAA88411848A72FFFFFB
:10C21800FF7FF97A9434AD99408BB2432C89419BC6
:10C22800D80119092441AC90189AA94320AA1539B4
:10C23800BD81109B995010BA5F2721E9912AAD055D
:10C2480021A90259CA9218A912510A9030DBA120DB
:10C258008A2313808900BFB88222A90710FD535B87
:10C26800C9840ABB5328B8152CC90209B014308BED
:10C278008149CBA22099403398B928AF991240C977
:10C288003409FB760BBA258BB8631BB1349DB832E1
:10C298008B913508AA832ADA8410A91228B90322B7
:10C2A800E9A8122FA0331FC373ACA941ABB3620B2B
:10C2B8009152BCB0309B024218AA140CE9121A9091
:10C2C8003318A8001BCAB1528E0341BF8451DA92B9
:10C2D80038CC0520AB1248DA8239BA15209A984131
:10C2E800ACA1418BA333ACB2428E901289B81780AF
:10C2F800CA445ACA850AAB4328B8242CBC0219B8C8
:10C3080042409A8020CE91319A8342ABA140ABC182
:10C318001318B8268AF9570BAA258BD0331AA025EB
:10C328008BD9210AA03510AA8129DC8338A9234892
:10C33800AB822BF902209A94409EB543AF9040BB44
:10C3480095388C1418CA012BC8251998318AB90850
:10C358000AB147089120ABB12AAF1418A0240F9254
:10C3680042DB8249CA0528B8241AD9020BB0538A7D
:10C3780001389BB989190857889120AC9019C04396
:10C388001A9022DF153AF9041BB94489A0420DA07E
:10C39800029C91519882289B8980BA10720884085F
:10C3A800AF8819A833301802F9428FB024BB8171C5
:10C3B800999312BF9120C913499803B8992998C233
:10C3C800043C8A250BA8158AA2498D9238D373BEDE
:10C3D8008020C9A4480C1321EA012AD8130808119F
:10C3E80081DA002BD18581882082DA903E98141852
:10C3F800192AB738FA003CB8271899321BFA120CD8
:10C40800914298802899E0010B0232B89538ABE147
:10C4180011BC0708A8129C263AE0820D892301B1B5
:10C42800412FC822AC01408881881AB884AA80703C
:10C438008A05089C90309A0211B994E1721F9011F4
:10C44800CA0050099411AF8128C9033B0913080E8B
:10C458008081D01228A8428ABC121DC2500B8021AC
:10C46800F234AE8020C8B3401B0323FD8219C824D0
:10C4780009882091BB825BA93599922009C1FFFFE9
:10C48800FF7FF978088AA544AC9A509AB2432B9951
:10C49800349CCA1139981541BB811A9BB95418901C
:10C4A8001329EB00038C9048A18A2F3742F9912A6F
:10C4B8008C83348A9060BAB011098A5529B9020A66
:10C4C800CA885209B2348C981889BA1528D2829F22
:10C4D800446AC9830BBC4331C9152BDA0209A0147D
:10C4E800210C8139E9911089013300D810BAA88844
:10C4F80063C08400FA741CB804A9C03339B8368CF8
:10C50800C9228AA12421BB042BDB0210B021500AC6
:10C51800B228CC90321D98510AF2569C9830ABC381
:10C52800430B9052ADB022AB014328D8139CBA31CB
:10C5380029B024218E031ADA00109983781F837199
:10C54800BD9220BD8431AB0338DC9320BA12410C74
:10C55800A8238CB8438C90221AC8428BAA2509C8F4
:10C568009428BF2749D9832ADA2518B8132CBB1475
:10C5780019B814209BA151BD9231BA0241AB821067
:10C588008CAA361BD83208F9642DBA258AC8421AF3
:10C59800A0248CB9320AB02718AA8238DB0410B953
:10C5A8000238AA1221CCA1339EA1438DE2638F9851
:10C5B800319CA2518A9041ABC0328B905209C91369
:10C5C8001BCA341AB8151AA91329DA8321AF012016
:10C5D800AE0552CBB258BC8431AA0258BBB221BCBA
:10C5E800036109A8319EB82309B1530AA9111CD9BE
:10C5F8002121CA1629CC3549DA842ACA2510C8133C
:10C608001BD90319BA3520BA9248CB8331AE02310F
:10C61800BB9341BE913199C0349AF0532EB9259AF3
:10C62800B86209B0248CB9348AA84319D8022BBC43
:10C638001518AA2329CA0339CA1238AF8131ACC5E3
:10C6480053AEA032ACB2718A9132BDA041AA9242D7
:10C658000BB0148CB9431AD0230BC9331BC8141957
:10C66800AC0429BF1361CA9239BE84219B1248CBFE
:10C67800A220AA13538AB823AFC0238AA1360AA9D5
:10C68800228CC81338B9330AFF253ACA842ADA2417
:10C6980028A9134BDB1219B815308B9121BFC13172
:10C6A8009A03249BB148BC90348A90231AFB732EBA
:10C6B800A8149CA06189A241AD8020CA1240A80399
:10C6C80009AB9001AB1738892289EA109B93430D77
:10C6D800123AF8458E9832BD93509A0330EB013ADE
:10C6E800C91429893298BAA018F0051908229BC8DC
:10C6F8002A8B0611A9315FA342DB9359CB1618A9DF
:10C70800331AF9120BB0350A81208BB0920DA86349
:10C7180009A130BC8109BB4122B224DF2439FA8542
:10C728001BB94409B0430EA012ABB3618A8220AB97
:10C7380098019C92718A9420BC8000A8223B020335
:10C74800F8153DBA169CA251899241AF88119A9367
:10C758004089120A8BB000ABB3770A8129BA829854
:10C76800B95200A810A3769DA851BC9431AC1338D7
:10C77800DA813AEA2419A1240AB9889091241898F0
:10C78800540DA8029AB36980030E9163CCA268ACD9
:10C798000428B9341AE9120AB9448991208D9020E5
:10C7A8008A90151AB87199A011BD140888902A5357
:10C7B8008AF9211FA03698A2309E91119D8240A827
:10C7C80001299B92919B39638B941A8DA3589B22C4
:10C7D800B180A3D8761CB002BC897180A403AF8055
:10C7E80020BA0238081209AF8108E01039093090E0
:10C7F8001E9020C986098933D134BF8138F8923810
:10C808000B1611CC012AE82219082190DA211AC046
:10C81800138A2853ABC9228EB178991209C441CB27
:10C82800813BC096108B2339FB841C9022099128E8
:10C8380029F8100D80249992381BB9130FA0129073
:10C848009379430EC8021F902509A0221DC0219E7E
:10C8580000408901088AC110890222B8833BC8AA0E
:10C8680071DA12988241FA461BC814BA98610A9381
:10C8780033BFB121CA0359089101AD8220D9835928
:10C888008984819C9030D002190908C720AF021909
:10C89800E08238898510CD1119D8230A000219CCF5
:10C8A800111CB1340A91409BAA071D80390A020C59
:10C8B8008533FB003C898601AA334BF9130D90326E
:10C8C800A000280CB013BE8223A8924A29CC23AE1C
:10C8D800924198012F131AF9220F88249890418CBD
:10C8E800B0219E8331B810189BF112AB1230F83288
:10C8F80089B8922BBB74A8B141AD434DB823CAA0E7
:10C9080070089221AFA121BA03588A01029E913082
:10C91800D903209982948DA041AA82389A91B7713F
:10C92800AE0110E882490A00FFF777776F88D912BD
:10C93800083719029DB08AC14002518981CB90AB5A
:10C948001341153A908D9998913482188ADF53B91A
:10C9580015C92AC81290548912AE908BB428044085
:10C968008808DA09B01210441A83BD909B932123DA
:10C9780013B8FF709938D01BA1229172A838DB80B8
:10C988009D03183420981DC88A903184339949E84A
:10C9980088C8110022882DF61B038F03D920A140D7
:10C9A8009030C81BE01A02210339B19FA1AC13884B
:10C9B8003688028E81A9818120201A2FB78931EA11
:10C9C80069C1299249922AB00DA2891320250A81AA
:10C9D800EB28D83091419021DA18BA028124081046
:10C9E800FF60B129D32F930A841A831C819C01A864
:10C9F8001210418819F81AC12994389239D01BB8F5
:10CA0800190419040AF17A950D969C13AA249922FF
:10CA18009C11CA28A1218338902FB28D820A160949
:10CA2800020B93BD018A248923AFB71C22AC41E8CD
:10CA38003A920913A048A10C909B93AA72833A14C6
:10CA4800AE10E819A118140120888AD89D819F2763
:10CA5800A139A14CA39D11A039841A12A989BC2916
:10CA6800C328168048A20F91AB119131232920DAEF
:10CA78000BF91AC971B71A859C11C828A30A33A0E3
:10CA880030D089C81C038851925A93AE00AA1882E4
:10CA9800131230819CCAAB9BF17B379923E94AB2C8
:10CAA8001C039950A13AA00BB39D22A268831C11C4
:10CAB800D919C01A0410130901ABAAF88CC71B6056
:10CAC8009849C21D829A31A23A848B00BC02D84888
:10CAD800941A24A93AD00C928A3201519109B0AF24
:10CAE80088AF36C138A32F949B20B13A841B23BA50
:10CAF80018D92AC32B268941B02CA19D10A0481310
:10CB080029128C0AEA19DA71B609859C21D0199381
:10CB18000A14A028A00BB01D858932A25AA49C0033
:10CB2800C8199318358820B80DD00AD37B239A34B6
:10CB3800E93AC21B049840A12B908CA3AB52A16880
:10CB4800830C01C91AB11B359242902AD09E92AA31
:10CB58001588709028C10C81B930B5181489189AB5
:10CB680098CB38912A538868900C909B29934B2531
:10CB78001A26D928BA52F21A932F03AB40C12A9326
:10CB88008A23C039B828C21C04B850982AA41C812A
:10CB9800AA24B228079984C949D879A40B049C31DE
:10CBA800C83B931E219838A029A00D83AB60C32AE7
:10CBB80094AB32B01A912D139825C01BA78AC33F96
:10CBC80013A923F03BB30B23D848923C830B81AEC7
:10CBD80022C03C038C23C859901A83C912883C94FC
:10CBE8002E02ABA78B78A049C31D018920C21A0366
:10CBF8008B22AC30C83AB58C32B960B21B11B9116E
:10CC0800B23E850910CA30BF43F22B933F839C2163
:10CC1800B03A940A23D010A82BC30B04B168C13AC8
:10CC280083AB38B81AA420032F02C009CE79A50A0D
:10CC3800838D31D829920C229948A110C12D928B4D
:10CC480031E32AA40C22A982B28A390927A920B083
:10CC58003CE26B139A37AD39C21B848931B13890E5
:10CC68000DA31E02B812B44B95A920C94992B82247
:10CC78000B3AB40C088DD70B33BA70D02B938C3287
:10CC8800B12A850A01AC15AA19A36B930B32E118D6
:10CC9800C21A949929084A801A84BF27B958C23AF7
:10CCA800C58A11C820B31A038A34D880C12C810BD5
:10CCB80035D120981C949881A8280200A19F29CEDC
:10CCC80070911A968C02B949A13B069921A019C105
:10CCD8001AA38F219830D41A02AB58A08811800368
:10CCE800B979A699E24C128B16BB30B22D948A22E0
:10CCF800903AB22DB28A03D943D22B948901D84BEA
:10CD0800000811D833B20BD3AFA71B229A60E019E1
:10CD1800928A12A148B23A928F818A48B149950BFA
:10CD280022D01A921A82B850BA78A01B31AF17A82D
:10CD380039A07AA20D12AA31B21B179802B918B8F5
:10CD48004D838B43AA39B78A93A980930908790040
:10CD5800D020DD78912AA50C02A938E118838B50E0
:10CD68008881B01CA20A27A838920C03B991A03870
:10CD78000069A3B80895B1F97A978C13AB58D21A01
:10CD8800928921B1487F77FFF6A41AC126D928884D
:10CD980009034C90208D0083AA3978D832C881962F
:10CDA8000BB385D2A0101C8480B4A8930A4AA59519
:10CDB800BA1B708990388B03A01F383BB6B4992AE8
:10CDC8002A93A7C11A190280F4980A2192F0011E29
:10CDD800209082B20C5C1882088A4E39829B400CE3
:10CDE8002895A909058B83B4A5B20C3D3894B0B237
:10CDF8003F589092898979A290018D490801992814
:10CE08000B4F380899015C29A294E20A0292D28059
:10CE180084D1A13B92D688892A28D3902D3B299585
:10CE280090091B3A8398D383AA42B2F1032F0A834D
:10CE3800C30A894131F18A2A9D798291920C192875
:10CE4800A4AA7A1B5A02A09B212B52A992B02F198F
:10CE580015B2B1588A98879C010938A481D10E0867
:10CE680092943A5A0910DA93A2014111F0180D0868
:10CE7800D318819500AD4919D1013A194892E909A9
:10CE88004D3A04B3984B1C10B5B01A3021D4B18A6E
:10CE98002D2A91878089301F91809081391A103FFF
:10CEA8001982F2109C20208D0081C38D4A1488B409
:10CEB80080C1C22B1A40A4E48989588A82892B2808
:10CEC80038C100AA5A4D0491C23B0A3F11A1008BF8
:10CED8003A279B283F12C3988E2100B3A11A5C1BE6
:10CEE80011888A4020F3A3BE5B2902A195B82B5A6A
:10CEF800B7B3B04D3982A10C4C20A2983D38A4C3D9
:10CF0800982A84F290191995A03D4B29A1093C282B
:10CF180085989B5895C1893C11B7A1982A2A080A77
:10CF28002A3B4B319884F298C5A202D2A3D2984AE0
:10CF38000B2A58080B382E11B82B251F100A21D19F
:10CF48001A0901A6818099A2B6A882B38905830827
:10CF5800D91A1AF83509AA2853F0008A1B2292D345
:10CF680021E991319C489889402E028A02AAA79A01
:10CF7800699884900A8950A100922F8090D30580E7
:10CF8800BA580898079B8201B9C712BC0158A9A5CD
:10CF980018BA1860A8029891905B802DC508109A5D
:10CFA80030A99F3820A08840B808C60E0190508A42
:10CFB80009800D3890FFFFFFFFF9782AA7B13D3CA3
:10CFC80059D6B0810D5A0802D398895D2882B4A138
:10CFD800093D2900A3C1092A3B3894C2981B5C2A41
:10CFE8001E60D4A1885F32D293C04B194A82A2D363
:10CFF8009B5A2A03C3A2993B2B28E4A1801B598082
:10D0080082C180982AA97C17B3C59D6B8010E598CA
:10D01800803E288895C1092B5A0192C20A192D20F1
:10D02800A292A13C2919A4C1A288F61F4A1885E238
:10D038002C193C04A094A94A1B38D4A1903C292956
:10D0480094B1809B6A0180A5A0191B3A80A3BAB746
:10D05800B27B5C59D6B8001E598803E288895C10F7
:10D0680081B5A0192C399192C20B391A31D3919AF2
:10D078004C2A2A0F61F498085F32C193C04A095AB2
:10D0880093A1C38D4A1903C291894B0808A5B01012
:10D098000A5A0191C3A81B4B8A7B17B3D59D6B8095
:10D0A80002F598803E288895C1081B5A0192B39AC8
:10D0B8002A3E20B391912C3A2A93E3B298E71F496C
:10D0C8008096E22C194C04A094A94A1B38D4A1904C
:10D0D8003C291894C1808A4A087777F75E028C93B6
:10D0E8001B382A41E18A92D21B5A11B2180BA4F2BA
:10D0F800FF710BC1139E8131A99508AA138C912247
:10D10800A98229A029896B99220BB3718D013CA1B1
:10D1180003BB0033F8F4709E0110BA0428BA350A2C
:10D12800C0139C9148B8148B022A9001AB942F012C
:10D1380031BA020C0991A1811F3BF740DB2129D8A4
:10D14800231BA9518BA140BC033BA1488B138C9393
:10D15800099218AA622D0012BB131EBB232B5F076E
:10D1680048F9211CA124A9A2319E8229B9148B92C5
:10D1780048A8F7FF977DF10F418910F06990099150
:10D188002C2899539C28992E9348C022A81A806B62
:10D19800E31A804B9690A40B82D003A04A00AA28D9
:10D1A8001B4A588E380919E419C139A499033F92CA
:10D1B8008A01C071B84A980A011A159108B20FA4D9
:10D1C8001900B825BA58985AB020C159934AF82975
:10D1D800020F228B001901BB459D21A848C1299245
:10D1E8000B10A971B04AD119A50B23B912F828C49C
:10D1F8001A941D839B40A020C199051A81A919AAD8
:10D2080079860B969A829001B0329F139983F048E1
:10D21800C838A42BA32F939008021BA20891CB27F0
:10D2280089809970800D9492D1822A91AB4A0E69B7
:10D23800011A83AB22F829A42B84A848B84B911B68
:10D24800A42850CA38C12C120A31E93E1389A7A96B
:10D2580030F020B21A028D309958B29A83BA72C14E
:10D2680049A10C12AB21B35C012B859B21BB20C3C8
:10D278003F608C20C039C319B6A812C03AA14C82AD
:10D28800A848B059A38B859011A88CA388239972BC
:10D29800D819A20D86C068A969911C010C21A0307B
:10D2A800C31BB49B21B058A31E139B12D039B800DE
:10D2B80034BB52D829A28803AC58F210F31B04AC33
:10D2C80021AA5A814B039C14B928928E13AA51A8FB
:10D2D80039B81A02D9619819A40C019B51B96C0587
:10D2E8008A979A12C010B31C128D309A48A20B0369
:10D2F800BB51C149A21C119B48C13C832D838A386C
:10D30800D829B50F320E21C03AC209A79922C028E0
:10D31800A03C928A30C159B40A839B03B03CA60B47
:10D32800059B32B088B51C87B858AA79912D010B96
:10D3380021B149C409A38B20C03BA61C049A20A094
:10D3480019B48C14A922C03AA30C84AC40F310E39E
:10D358001C03AB21AA7A823D028B13C819920C15C3
:10D36800AA50A83A911B84AB40A169B31B019D3117
:10D37800D86C030AA79A21D028B22C138D48993863
:10D38800C10A03AA51C13AC40A008A21D039A33C70
:10D3980084AA30D84AC40E318D32D03AF27F7F78D1
:10D3A800F1F4996F2801D38A4A81888805C4B84B5B
:10D3B8002980803AC5A8191832F3C00180A20B133E
:10D3C800F6C1081C30A0000C20918C3A34F2995A0E
:10D3D80081A1884B38C2A4A93D5A01B3888D5B4806
:10D3E800A3A82B108B50A0A6C14E3A83C2892B202C
:10D3F800B6A188A4B3A1928A2C1288499A7C3A4F84
:10D408003981A21E4A0801A10C4994B3A000B6C3F1
:10D418009928B6B01A5A190081B29A6B11D5A01979
:10D4280093992B6E399291882F3982C3A119A192B1
:10D43800B39C7893D2892B3985D20C3A0183E39A2D
:10D4480039903D28B7A03D280900A84B04B13BA25C
:10D458004C82B1802A8D7C20903A2B0D38818B121A
:10D4680080A91790A2B21F000282C0A30E3A26C25A
:10D47800991B0803921B32C8BF3889A784A98B302F
:10D4880038492ADAA5814E2093E1A12A10A208A2E0
:10D49800897A812B82F930196A82A0B2D19048200A
:10D4A800B3F0892C4902A8983B7008C2A099203291
:10D4B800E2B294F2A03A90902910017C4B0892E2D3
:10D4C80083B17A0B2A2883A5890A99B6896A400903
:10D4D800A9000B798000A8997081D8392AB2924D99
:10D4E80089481C93A32D91129E8203B1AB7190F1D0
:10D4F8000A5A0095B4AA291802A82E82A0386A925E
:10D50800D3B11C3C2100B3F499202D11E2B13B5951
:10D5180081808B5C12B3C83A4AA6B3980A03C4A99F
:10D52800084A20986D191898104E20A19109090BE6
:10D53800B7818196D28A200C8201BC4038BF1292F2
:10D548009B83B811879239AB9D81341E11019A8A49
:10D5580070C2A20C3B12802006B8E81933A11E093C
:10D568000E38222C2C90BA815A43B5D1998120913A
:10D57800B01CA2A0621920F1C089791880A4D0013A
:10D58800193BA001E02B619181C8BA51389985B83F
:10D59800C1848B5839AAA8681B33D2B1E2083992E2
:10D5A80098A09C6B302A95F1901A7A0892981A598B
:10D5B8002A188C2B958A5A921A82E11916B29B80E6
:10D5C8000970A10995B8881819A23B5D22C24D18A7
:10D5D80091B3293B12F1083BB30801B848B04A9609
:10D5E800C48D592B84C2882C21D082B32F3910D3F3
:10D5F800B1995A4AA083D38B799008080A29391817
:10D60800A31F3C13C39093C1B4B393A1B5A39E19B0
:10D61800014B3B5B312B3D1F21C01A022E13C18ADF
:10D628005A1092E10A0803938F4B40C3B00B3A801B
:10D63800168994D11C6B1090910A3985990997A085
:10D64800993B6B10C4A2991C582B83B4B00C4A1296
:10D65800B2E20902C2904A01B1B48979A3D87D4ADD
:10D6680002C2881A2A83B95A0293D12A1918B6B85D
:10D678001B29192108896199D2B4C19A311C3C88A7
:10D6880014B87C388990891A960059B0010109AB01
:10D6980071D3B9921A48A872B1B14C2C8384D29034
:10D6A800092B38C7983D4B1910A80B51C3A101C2CB
:10D6B800C3C32B188CA70C291090920F3A0004B200
:10D6C8008A0B28992698935E1900A3A3811F894A7B
:10D6D800009015C29A4D4A01019B2E128A23E390AD
:10D6E800A48891F208808029028C6B1C5992A802A8
:10D6F8001A4C02C3980A4E029091181098B6A1F0DD
:10D70800094B280200D983B81B0113F23991C401CF
:10D718002F1A83E8207F7FFFD7918B290907A498C8
:10D728001C8B838310920C6B8818D224C80968C29A
:10D73800B4081A20A0C82429AD4F917310DC9900B1
:10D7480022110180099D0C98029303184B00C9957A
:10D758000B8C8A0415800938C1A8CB885881FA3700
:10D76800711BCBA80121232101B8E9BB1A3400821F
:10D77800113A3D2988F9C390186130A199DAA04976
:10D788003082C1FF23731AFAA800311203229EBC0B
:10D79800B084208802139AE980421ACC9812210A90
:10D7A80034610CCC9011188AD357208CCAA011115F
:10D7B800124310BDCB882218102323CBD981218A8C
:10D7C800CA043488980811DEB816218BBD94471016
:10D7D800AE9980118113421ACCBA801211114029D6
:10D7E800DAA82428ACD8080322351889DCA9828055
:10D7F80002BC574419DC9A81120323419BCCC9000F
:10D80800228213101CDB915118AAB9103902652223
:10D81800ABFB08018091A177310CDAB901212243D1
:10D82800418CBDB900102123348C8D88108899A8AB
:10D838002024591418BADB1B8A2B2AA777408CCAD4
:10D84800900121233310ECB9FFFFF797271F18F831
:10D85800192A425E308D1909985B03398291CB10E1
:10D86800F00180122B038F19991A4980691A7F22B7
:10D87800C181B11AB5A3A104A821E81B1A940B51C0
:10D888002B281AD01BB30913878A24D929899218FF
:10D89800A41892BF79083BC30F18019213E208C27B
:10D8A800A0A986A03188388CA18E82901222A16806
:10D8B800E008A8829927A195F31C182D02AA3A3AE4
:10D8C800205A830E00A0AA41C321A200AC01CD11A9
:10D8D800081329952E910AA838A871994AF7A081AA
:10D8E8008A20D10818112D309D3A88A05B0408833E
:10D8F80080D818C829904289238F109B912A927A40
:10D90800197F22B193D019B5A29184A838D01B1AD7
:10D91800940C410A200AB10BE21981419834E93983
:10D92800AB138B871A84BF798829A20D28818112AD
:10D93800C219E2989905B04198280D818C82880215
:10D9480048A259D108B811A817A196F22C181B02A1
:10D95800BB6A29104A838D82B8FFF7FFF7B6C5F175
:10D968005D381C209B5A09209822A858C28A92A286
:10D97800C121D33C049A1099801D859A23B058A1DF
:10D9880081AA02F1F7A0109948C03B895A084A8138
:10D998003D029B2989932C878A31C119A0888B2342
:10D9A800C978922B08199D6B1E34F381B21AD4984A
:10D9B8009209822C048C21C82A0A128C34C04991FD
:10D9C8000A8918B968C33C020A192B986E1F7B8212
:10D9D80009A58C12B884A0959812D029B3988921EA
:10D9E800B878A31C0299911BD33D869912A001A86F
:10D9F800B7B1E34F381C21AB7A902A8219830B9771
:10DA0800AA12F108828810009189A1C818940A17EF
:10DA180090819190B8D6C2F7B020A958D21C182B83
:10DA2800201B318D48B84B938A13A0202C119C29B8
:10DA3800C04C020A4009209B4A0F4B1F35F480C393
:10DA48000BA7B802A8309848B05BB31F1088209085
:10DA5800108929992E911B32B078882A0A3C9B7D1F
:10DA68003F7B83A0B79B23F118B319932C958B04A4
:10DA7800C939A04A81108289A5AA02C938C32A02D5
:10DA88001984A1F3A0F17F5A1C31C84A920A9598CB
:10DA9800839A14BA40F20992891188000902D810B1
:10DAA800C11AA798029002A9A7D2F7C83A8A7AA2FF
:10DAB8003E110C219921A940D04B949A12A8208894
:10DAC800109938E20A938E31A812A129AC7A0E2750
:10DAD800F6B9841D13C85B913E118A209028A97A53
:10DAE800928A03C04A921C31A94AA11B011D218AAE
:10DAF80068A97B1F7B96D086C940E50B959A21A91A
:10DB080048A129C41E119928B40A029939911D0106
:10DB180090009839012BF490F27F6B9841E23D8593
:10DB2800B913E118A21A038C86A928B13D85991169
:10DB3800B219A49A109884C118921AB790F7A95BE1
:10DB48001A5B923F208A48A129A48A029C23F119D2
:10DB5800A31C13AA31D12AA49A129A40C219930D70
:10DB680012BF17F590A22E04B949984B011B218BBF
:10DB780030AC79A20A849A30A05B821D11B849A101
:10DB88003C039A30CA798D7A95A0A6B922F309A4E4
:10DB98008A12A838B12AB25F018A30A13B948C213D
:10DBA800AA5A911A039D40A02AA48CB37F488A32AE
:10DBB800F03AB59883B012D2089289B7A920B04A32
:10DBC800940B14B828B20B018802B13AB70AB7B25D
:10DBD800F7A95A0A6B922F208A48A12A838A029DA4
:10DBE80023F018A30B14B830D209A499019810B4E3
:10DBF8001B139F31D932F208920A95B83A913D1118
:10DC08000B21A028B968F209810B690A4A811B0215
:10DC1800A001083F20A83BC07B0B7985A803BA2147
:10DC2800F20B84A011B211B489A03FA5A801A228C3
:10DC3800C41A920F21B83A911C128A33F12AF25E63
:10DC4800288921B84B949A21B021C30A04A0B6AA06
:10DC580039A03B069A32C028B12CB70B21BA58B369
:10DC68000BB798D7983A883AA21F109829083A1201
:10DC78001B20C928F82AA50A318B699299A5A920E1
:10DC8800C149B32D120D289C37F398820A03BB595A
:10DC9800A11B120A4880119E3AB23F18893980495F
:10DCA800938C498B38B10B879929C9798F6983A8D7
:10DCB800839C13E000B389030933C818C12E949AD2
:10DCC80011A23B960A819A28C21A12815AB401F20B
:10DCD80082F07C280A22BB79918A03A112B110A292
:10DCE80019E48E12B028A49A048A40C188A4099421
:10DCF800B1829A3CA7A1F699389948C12E10892873
:10DD08009029834A808E22D818A23D129822C810E2
:10DD1800B31D811C12A028085D192F97B380B32B5F
:10DD2800D69A20B11A014A838B14AB4AE22A929AF6
:10DD380040B048A21A920E287777777726B8907C59
:10DD48004A82900E5A01B4B20A3E2983E4A02C39C3
:10DD580094D3A83C20B4B11A2A84E38A2982C49AAD
:10DD68006C28A4B2893B10B6B180801900A18A5EE4
:10DD78004B21D3A11E5B28A4B28B6B2893C28A5B6C
:10DD880029929181A1A28A6C109291893F4B02B588
:10DD9800A10C4994C298290882B01C4A3995B04F01
:10DDA8003993C3980090802C49A590888A4B2922E2
:10DDB800F5B0083E291911D3A10B4995C3C5A95D32
:10DDC8004A10C49A5D4992A2984C20C3A83A00947C
:10DDD800E39A5A82A1882B3B84D209291A02C11CD2
:10DDE8004A18A7F5B83C3A84D4A95D3892A28C6B3E
:10DDF80011B2893B3AA6C20B3982A3C21D39A39836
:10DE0800191A39A49A7E3C5B05D3A11C4A96E49959
:10DE18003B2995C20B5A82A1882C39B6981A291821
:10DE2800A3B03C119191804E02E208097F4B02B4E5
:10DE3800B13F4A95D3892B38C6B11B2881A3A94D78
:10DE480020B3881A3B02D39B598291A00C39A7A30F
:10DE5800C20E3A1884D11A2A2A02B3983B8B00942E
:10DE680086C2894D2A02A0290193F1B13E22B11040
:10DE7800C86C289290B7B1290D69A4A82A2A29014B
:10DE8800C10908281910F2910A4A19C13A492A8485
:10DE9800F28D489180920D29181D68C4A2B13F11D6
:10DEA800B491982B28C380092B0118903895AC2C75
:10DEB8000390383F1882F85A011AA4A019181F7C39
:10DEC8001190B59A6A8191A3993A03D192A0180842
:10DED800A02A10A09120A6D18A111DB73D180A03C7
:10DEE800D39092F40F391A13F11B291883D20B3AE5
:10DEF8009103A21B0BA6A8292009808802D231BF52
:10DF08009798801B4099902BF7C21A2E59B59808FC
:10DF18002B3A94B83B1830B00B3B8184890D13A081
:10DF28008858993BBF52E118882A99197E50D3A284
:10DF3800A04E12B290883C20B399082910A84B39FA
:10DF4800A186B91A31913F8118B9798189B51A8AA0
:10DF5800150F7C11A2C49B798092A2893B7777FF29
:10DF68007C3B83F7D21D5B11B5B289093A82B4C2F2
:10DF78000B7C2881B39B7A02B3C20880B5A0080045
:10DF8800A4D30C4A0088812F3A10A3C39A4B05A149
:10DF98008A30B3C05E2912E3992B288808821AA216
:10DFA800970E1931B88018B7A83C193A93B7B80D2D
:10DFB80058888196B83B38A4B109C5993C4A95A1BF
:10DFC8001B820B91940993B60F3A12D18029883C91
:10DFD8002BA4D41D4A1881C20B5B03B29A32C5D256
:10DFE8000B49A290082C4A3C1818980B793E1094BB
:10DFF800D2983A801893D5C20D4A02D3A109198341
:10E00800B28B48881A5F4B28800A2B5A02B4C10089
:10E0180092E4A18A2181C20B7B0191A20E498180E1
:10E02800892C39B4901880A2887C809038A84C4AF2
:10E038002B21A5D0A31A8B4380F8284C80820AA0F4
:10E0480053AD29849A1B48B6994A0001D2A21D4BA8
:10E0580021B29000B938C7803B98A3BB7B4891A2F6
:10E068001C833E292B2BBA702D2922E1A1108B2469
:10E07800B2B9B7891A3838E831E4C2903E11B3B45E
:10E088008B5A0984A2999121990A02C04C5D13A860
:10E0980081A25E01929B6C59888181A03D20C4B108
:10E0A8002E3993A0095C20B3A02A2E11B4918803BD
:10E0B800F2B13D1995A2A84B4A8091A22E110918D8
:10E0C800E4900B3A4A88A7A2892A28E39949985BE1
:10E0D8004A8A580A09079A2A13D2A39A181A7B84DB
:10E0E800D2882C4992B3993B83D1190289802C4A52
:10E0F800D3993F488081A08B78A19097A82B22B311
:10E10800E028919A6919D6A03D2901B2A38A39D588
:10E11800889000919B7A3AA6901E2928A1802AA06F
:10E128005A49A2B5998895C4B1180A40B2D12D3977
:10E138009208B230AA4F281AA4B21F5A10B3901BE3
:10E148002B23F0192A2B23B3F28A3B5E12C289399A
:10E158000C48A4A81191E3900982E5981881809D44
:10E168003997B0194A83B38C3C813E298295AC5AC1
:10E178001892B4A80B7901C3992A20B80187C29ACA
:10E188005909A4808B6A10D3904D2901A192B29BA2
:10E198006B24D4C1190A20A28C5980FFFFFFFCF719
:10E1A800FB518080081991119AA241F882219DA300
:10E1B80032CB9350CA042BA01390C21BA078A1A104
:10E1C80013AE189408A82851F9021A088098827189
:10E1D800B9830FA240CAA443BD8339AD8328C002C6
:10E1E80049DA3489A9231F90238D80230DB151ABBF
:10E1F800A430CA0328B8129C0409BC006829C94481
:10E208000DA8410C9034AD0218A91830D9032D007F
:10E218000290E04080D0821899B2A5218AA8259F53
:10E22800905089C260BC1310BB043BD82209B95571
:10E238008C90309AA32A801209A71DD1239AD00561
:10E2480009A0112AAC85189A8B73BC02229F9248A8
:10E25800CA2229AB163DA81309B9338BA170BA0697
:10E268009A011980841D808101AD002608D110B162
:10E278009B41A92708D91339CB8430EA12229EA4DE
:10E2880038CC1338F9132BD02188B8428D92119AC3
:10E29800B2689A050BA060B9032ACA261AB92120C8
:10E2A80099880979B924A1B8440F823AE8230BC8A0
:10E2B800439D93108B0068B9101981929B345BC8F9
:10E2C80043BF9231ABB272AC81100B8231F011AD09
:10E2D8000349D8230CB852A9A1258D921098B143AF
:10E2E800EA041A98229AC1248D900580B00020C9AA
:10E2F80082301DE061AC02209D824A990318BC342B
:10E308002AD9230D914A9A340B8039D8860AAA341F
:10E3180029E0128ACA458AC1230DA11280C8128B2E
:10E32800814A09038AE9520C80A0248A09049D8441
:10E338003AB91B710E0139C8041BA90609A8311086
:10E348008CAA4182CA8B2769AA1318F912088B066E
:10E3580009D1111BB972AC8328AA8430EB0609993C
:10E36800112AA220BA418F9240CA241AD93288A809
:10E37800933A92A0978D92210AD0378D903189A037
:10E38800118B250C98212AA0A60BA0509B1242CFD6
:10E3980092480AC142CA833AD8143BE8149A813891
:10E3A800BB8628BB132C9194A2849F8408AA034897
:10E3B800F8128A100888128CB05818A1A596AB9448
:10E3C8000993A282C12C8950AAA3729F8248D911AD
:10E3D8000819902000CC131C882499D50A812AA8F2
:10E3E800B728E81018009A0270CB02499B230A93B9
:10E3F80018AA33AFE340CA8351DA022099A1229ABE
:10E40800C102DB638AB243AFA230CA2238EA143AA7
:10E41800AA0121DA832C08271BE212CB0319C205B3
:10E428009AC348AA91359E80300B9041AC0158ACF4
:10E438000230BB030B3388F8279C9202898049E19C
:10E4480021AC2029A8210F111991891038F9850AC2
:10E458008101C8071CA140CA1141BD8439D9130BD9
:10E46800A0508B953CB8418AA3FF477FFF236CAA35
:10E478001589880011D8C3082C81718CB8512BBD1F
:10E4880083420CB91729D98410CA0331ACA0510BA7
:10E49800B92428BD1140AC93408D880329CB025183
:10E4A8008A9005A98A9438E08509B9360AC0128B82
:10E4B800B8450AA8539D98300AD200194A90868117
:10E4C800AD19200A84A5A18B1A58809A28492F8152
:10E4D80025A8B9205809C1A6808B02280D3A2AB769
:10E4E8009198108929C508AB403AF2931A3F09025E
:10E4F80083D891480C19001031DAC594899D3030C1
:10E50800B1D3819C0004A2D1191189925B3F800389
:10E51800A8829281B8E681891C201890F18220ABEC
:10E528002B710E0293E8813A2B80A7020F09100085
:10E5380090A3B691A9084298F8032A2E1A03859841
:10E54800AF29591A981209899222A0E92903A48AA5
:10E558002E4080A9985A5B4B0894829C199793BCCB
:10E568008127A0B1013C989480900A3F282888F21E
:10E57800802D4D2001B0C2183D1B10942B0C289300
:10E58800D21A3B92A5C3B0B583B3D000192F1A4B4A
:10E598004A0881814B1F181109C1858089A3C59933
:10E5A8008920C6A0000092B8915C2C2B4008C82294
:10E5B8005B9D821490F0112A8E0238BAC305989890
:10E5C800182901C3F1882C22C5B4AA1930A2D11B7D
:10E5D8004800AB2A7928D1A518899193D1B2048132
:10E5E8009A118BA20C6A58A2D4000D1B23B4D1989F
:10E5F8005A2982F392908D08321AD984388F88313B
:10E6080080E081282D0A2285C0C1102A98C6939AD5
:10E618001C3001B099284A1C2B6091C3829C90142D
:10E62800A2C9820408A95831FB80321B9E501A9156
:10E63800820B1E2C3894C3B0692E2911B8A3811BF4
:10E648008024D4B18B4C5980E3A2192E18000FFFF7
:10E65800FFFFF7C7918C3A00B1885A392093C2C896
:10E66800990A2913178188199ABA908B2872303819
:10E67800198D08CAD9887F4815B4D1891A80A48011
:10E68800293A3909C0C1C10938310492990DA9B193
:10E69800A00233722A3C9880FB9812CB797029D358
:10E6A800C29B09059392183B1C9A99E2912040223B
:10E6B800A4B0AC9A90B297030383B1C98AB9F0B7F2
:10E6C800F4814C3C1891AA1A4812A592988B1C0AFE
:10E6D80092B582103849A8BBAA1D0925121121A29A
:10E6E800BA0FCC0910F697008A8A8888881952517F
:10E6F80080B0B8BA8E092423012938BDC9AC882056
:10E708004112602A09BADA8D2A5F302692C0A98898
:10E7180090A28152580989A0D0B988341322A3083D
:10E72800CBBEA991825213231B0DABD8D0918F7801
:10E738005008B0B88988939704180A8B09B8E881FB
:10E748003150101289CACAA99214242403B8ACAC57
:10E75800B0C0B6F311782C8998991A10252400A80E
:10E76800AB0E0AA094232139208BDC9CA91125101B
:10E778005111B8B8AE8B893AF787818B1B8890897D
:10E7880029515180A8B0B99E0922232381010DAFD8
:10E79800AA90004022413A9B8ABF9C0B6D4026926A
:10E7A800C88A0990918243681A8A90D8A889412317
:10E7B8001382089BFCA8A1113136211ABA99F9B81D
:10E7C800800F787818B0A88988928515180A8B0A5E
:10E7D80098F0912131392029C9FAA981020425121A
:10E7E80098C989E8A0B4F322793D0998890A1014D8
:10E7F8002680989A0B8BA99712113821AABEAD884A
:10E80800110303684EFFFF7FB1F08403FE6219A86D
:10E81800B11AE831983488100B999C9081122878A5
:10E828009223D89A2BCC82801268120880BD0D9B47
:10E8380001FA770909A10BC12991408231A9BB0DC1
:10E848000C1111B7810900188AB2D0099C51101413
:10E85800894A8B1D9A5FC541A80A819CB4199418EE
:10E868008318B1B8A8CC402B051881080B0F8181FB
:10E8780098D2380022901CA19F891FC748908B28E6
:10E88800BE138A041A111A81A9D2D0018840819333
:10E898009008BA1F219D8409284891A881E911FF91
:10E8A800432A80C01ADA41982398319B0A8B92F840
:10E8B8000209511981B3ABB9C858F031B821698838
:10E8C8009A00C88CF9778908900BC138924090213A
:10E8D800C80A898CA168021190189908ADC084985B
:10E8E800481A4200BA1C5D890DF531980B81AF9327
:10E8F8000894298219B19AB09C0408240881819C43
:10E9080088BBB923A7319A708988B51F889F873833
:10E9180091AB20EB130A2509020A80AA90AC25982E
:10E928003308018918BBEA80888701851909898617
:10E93800E981ED541990B019F811882288219B1BA0
:10E948009A0AD8408252AA281899BBF0920831290D
:10E9580007008C8931FB10F174AA10939EA239C16B
:10E96800489120B8188B0B833A8079012990989D9B
:10E978009102F0319028AA209189E94FF548C019F1
:10E9880011AF021B9239923AC080088B8499131CEC
:10E9980011282C0A8F1828A229A2799994810F028C
:10E9A8008FA75AA10810DA239B141A120C91908091
:10E9B800C823C01219948090AD9821CC420AA709A7
:10E9C800800A189D14FE538C829019D831BA418858
:10E9D80021AA088889A169A220B12310F1A89181F0
:10E9E800BC2698178988192BB959FA779A18828DF5
:10E9F800B34AA131A030B808AAAB05090539080205
:10EA0800AB9A0CA08990720A72B910C01BD02FF66D
:10EA180038B81902CD841B9329932A9180B9AA0486
:10EA28008A17008940A9099B0109B720B279A80271
:10EA3800090E818FA779A18920CA23AB140A220A5B
:10EA48008189AAD02199458981198899E8018C245E
:10EA580009834BA11B99F814FF538B81902BF84025
:10EA6800A82189219918899B98408050880308C853
:10EA78008AB210DB649A269A018908D808F9779A2D
:10EA880018920D9139B131B148A0089A8B841A9225
:10EA98007908110C900A0808A0709A709881902E35
:10EAA800A12FD720B81902BD841B9239932A9191BE
:10EAB800BBAA078A86190821AA09C91108836B917C
:10EAC80078B108918F829F874AA18938EA249B13DD
:10EAD8000A13A87FFFFF770A8FB71E1081199218B3
:10EAE8008B91890A968228A4AA39C28D01A229216C
:10EAF800C27991AA38E20B22B813F65A80BC25D9FC
:10EB080028020A84089A01A81E28010911A13F01B8
:10EB1800982C838B31926B00B10C30BB7A105FA7B5
:10EB28001889B850E108129A1388AB28A1BA501373
:10EB38001B40B0981CA1AB34B87825AA28D00C206B
:10EB4800B21B206F45989BB27BA28121B8410AC0B5
:10EB58001980F20821A10881B18B20E84B06982082
:10EB6800B32D91A12BA6A195DA718980A22F9100CE
:10EB78001980331F810909A190399102833CC82C5F
:10EB8800C39950B86290A81B80BA68B2A4F0729971
:10EB98008B07AC01802A0033AC229AAB19B9412407
:10EBA800895882B49BC2C38B060859918A58AB39DD
:10EBB8001C5FB728908912F91000891211D0119999
:10EBC8000C8982002943BB18B60BB8820B07012BAE
:10EBD80092D13CC12A987F160991A84BB01101A97E
:10EBE800513AC121D0B08830B23086919C008991C9
:10EBF800D32880050958E18A880BA7CB748908A314
:10EC08002F90800080250BA21988B0983BB58862A8
:10EC1800918A990880A3AD88E6822AA5B8B3AA424A
:10EC2800F07198A8879B08001880619B010A0980E9
:10EC3800913F00127809A88B008958920811963FD5
:10EC4800199A88A16AC738A0A813FA180888062054
:10EC5800B912A98A8183AF19124A208A1E81081A1B
:10EC680029090A272C69A82D822F170A098849C063
:10EC78000180983418D288B0B01023E80284A10922
:10EC880009F900A30941009832F13DA88E02A97440
:10EC9800090AA13CA89138AC5239008C19989B609C
:10ECA80089A91412902AD89BB71969089928970B33
:10ECB800290D03F151809D8298909238B1538A3B77
:10ECC8000D0C0900590A105929291CD88C2A1369D6
:10ECD80018A01914AA9D0E3CB73189A905BA8895C0
:10ECE8008A91449800809C90112D81A6808020A054
:10ECF800B0B37D12801C81A120C1A1B50F16208A56
:10ED0800D83AA91932B80720A92999B1D903D1202D
:10ED1800B70218B8A9B8D0882783801A9201F0C121
:10ED2800E2AB73190AB41BA90A48983609094C11B1
:10ED3800A0C8308A0913903969BAB872C829118CE9
:10ED480021A5A8801BE6F122089BA69998920802A3
:10ED5800420A93D91A0D90111C397019993D0B0B61
:10ED68005999405199803A9F093C1CB731889B3288
:10ED7800F990022B0232B020D29B9A395A93B62BC3
:10ED88004A1092BA190F813970A81A22D0998A3F6D
:10ED980097409AA95AA91932AA2278A118A2D8C8C4
:10EDA80020822897A281A2F080C389969309A29114
:10EDB8001AF193C0CB74080BA33E88092098234B03
:10EDC800828C91A891219B0D1523A2929FC08599B1
:10EDD8001082BA58119D890B04F06389AB97889A01
:10EDE800810981520981AB1C30E0192B1B71292A3A
:10EDF8001E891B49986A110A2858AC1B3C2CB7502D
:10EE0800889B32D0A8923A0433C888B991913A1BAA
:10EE180083F3681A991A99B17A11B03A25B110C8D2
:10EE2800F9804F05129AB958AA0902A8072199181A
:10EE38009099AE0108B197418883D9A2A299A7A356
:10EE480093019002F9B195DB70FFF78777F25DA324
:10EE5800AA48A319849B58A19A02A92A024A801891
:10EE6800970099D81A93807B010A78A01A83CF510A
:10EE7800B22B958E12B83A839A35C12B02BB22C8A1
:10EE880049B22A27A8080B5BA59921B02A830F034A
:10EE9800B30AB0F970921C16BB49A20B14B058A360
:10EEA8008A18C0198890218844918BE03D02C04B94
:10EEB800940A02AB7090081FB71A20A841F00A11F3
:10EEC8009931B22C15A82B900A8188482879809A04
:10EED80082BD399209588001A38F20AB8F17C33B9D
:10EEE800934F82C818A32C24B03AA39B18C12A9523
:10EEF8000B228838F02B929A60B33891C029E39995
:10EF080013FF78A389028E28A20B039969A309022B
:10EF1800D818918A14B012B25AA29D32DA59920CBA
:10EF280012911A928D22F16D12A934E82A939A301F
:10EF3800B25C039A39A10A02C931A211A51D82B88F
:10EF480011E11985BA69028B10993FF78928883829
:10EF5800F29A289839960A20A11C819900A12B12AF
:10EF680048028C3B8B0F938D488010039819B09FF3
:10EF7800A7C519A26D83C818A30B33B059A39B3A30
:10EF88008B4AA588231C29902BC1A917B9698280AF
:10EF980000A02D03FF588289838F28A01A02A96830
:10EFA800920A12B81BA11B959023A248C2BB02E982
:10EFB80012E38820B251B4C0B1F97A319924F82B00
:10EFC800828A11B34A848939C18A901A31B051832F
:10EFD8004AA2CB2BD84A96A200934A08D88DF78824
:10EFE800298838F28B20A83A858921A22F008981A7
:10EFF80098180029148B29D089A28D48811135B819
:10F008001AA29FD7B408924E82B029B21C24A848ED
:10F01800A49A109888A109058833B81E929B13E812
:10F028003B239833C82F80FD789389848D28B10AB3
:10F03800849958921A12C809901C8309219360B0C8
:10F048000D00E000A30931094893C891F97B419864
:10F0580016D93C000A12B24A830B59B189981C2070
:10F068007F280F7FF0BA2A541F119A018349A21FE3
:10F07800F70A83A950E02A829A33C038938F20A8D0
:10F088003AA32E83985AA03982BF29813A81A96A66
:10F098009180A0883F978931F12BB69B23C839A668
:10F0A8008800902AA08922BD50A41C849A22E11AC3
:10F0B800829912A05B03A9A3B88F71B21AB70C1278
:10F0C800D820A02A24B911811F828A00B27A828AA4
:10F0D800109939C21F11B228939959D2B905F0492C
:10F0E800821C04BA59B12AA68A31B108939D11B07D
:10F0F80020E41A12B938902F00C159008922B93B6F
:10F1080084AC4BF68A309A60D28A019B40921A04EA
:10F118009B58A00BA4A926B04A849B12A93CA59B86
:10F1280040A22D028B28B84F15C128B15C83BA4084
:10F13800B21B848B41C32B929B20C860B31C22A8AE
:10F148003CC58A13D859A39911A00AA5BF50A21B80
:10F15800840F11B119A30A20B16A938C28A950B25F
:10F168000C14A969A11B85A949B30A13D04A939A1B
:10F1780084F979018A13C93BA40C129958A21A037D
:10F18800C910B14CA68921B129A1AA31F82086A9B4
:10F1980039010AA7AA2AF50A209968C38B01AA5837
:10F1A800B32A859B49A20AA40D209039A48D20B0CA
:10F1B8003B979B40A20A219B49AF7F17B1882C7BC4
:10F1C800C6A9083B51F319980B24D948911A049BF6
:10F1D80021A92AB50A821921B868D11AA39B24FC4F
:10F1E80072C291A23F84D181887BA589809A58D127
:10F1F8003A828932D839A18B14C8218829831F847F
:10F20800AA10B138F27B1092C7CA6AA182B70D3131
:10F218009980B24DA40A20A149B22B81BA68A001F5
:10F228000189239F28A81A907DD70B3A2A23F84CE6
:10F23800081887BA589809A58D13A828932D930BF9
:10F2480000B13AB042818927CA39982C951F0780A6
:10F25800B0A87BB21282BF51AA80840F831929D12A
:10F2680048A88823CB13009D843AB80159D0208838
:10F278009B37BC783C0AA68AA12878B822C1AB067D
:10F288000A00A349D18020BC24988B0509A1012834
:10F29800E029928B979812F1509B1F33BB94842CD2
:10F2A800A14988C941992B070B92913AD03881BB63
:10F2B800358A08942CB29030BF31903FB711C0AA5C
:10F2C80078BA12078C831A1CB248A00B629C1802E9
:10F2D8001D921918C832A91A251E088118D849186C
:10F2E8000F2408D1C23AB82052CA13988F822981B4
:10F2F800B070A919049C83882BB250A1A944AC19F9
:10F30800021BE21082FA711C0B978AB12079B8317E
:10F3180090CD140A08A529B80841D912918C8329DF
:10F3280090A251D908120F828181F1508B0E24AB23
:10F3380082043CB14888E8239A1B170A90813AD086
:10F348002081BC240A09843AE08021BD30181FB707
:10F3580012C0AA78BA03078C82191CB150A008FF02
:10F36800FF7F7F3C493102E99AAD101612131B1E2C
:10F37800AC9A98124351181B0DAA99880021621261
:10F38800011A9E8D9A8A101325714908C9D9C9187E
:10F3980033621390ACBCAB9022372120890BD9B8CB
:10F3A800990832433430999CDBAC9030A725122B56
:10F3B8000BDAE9A80233722198BAE9AA8812531322
:10F3C8000298BDAD09A0923270120888ACCBAA0190
:10F3D80009561214892FAC8AA1052332388AFABA41
:10F3E800A81923722003A9BAAE19A092842070200C
:10F3F80009B9CC9B002E511423A29ECAAC881434A0
:10F4080033188E9BBC9910512240000AE8A9AB1012
:10F4180004140320929CAABBFA800370422098CD62
:10F42800BAAC20317412889BACCA88031620228992
:10F43800A8E9998800040421148C89CAAA9888A785
:10F4480054233ABEBEB0802441318999D9A8BC184A
:10F45800223613119A0EB8BAA2885332440989DCAD
:10F468008B991008173613999FBB99841522200988
:10F478009ABD99BA8123703420A8BB9DBA80833382
:10F48800723118BCB9FA09912B455133C8BEAC0981
:10F4980003240500889AAAAAC0A223625010A8C90A
:10F4A800AC8B00140423113CABABD9A0A2897740E4
:10F4B8002899E9C98821601380889C99AC8800261E
:10F4C8000322089BCBC9B9013361240299BBBEA9A9
:10F4D800B128D535323C0DBCC89132513108A9ABA1
:10F4E800ACBB8A327324210AABEAB9B8320551227F
:10F4F80018A8EA0B9B088C277480AA9A1C889196F6
:10F5080013301A9BA8CADA814230321100ADDBBA37
:10F51800B2239720413C99B8B0E8080F515188D0E0
:10F52800A08A09000703008A8A8ABAC89361312130
:10F538000189AFBB9B103245131109AF8BA9A1A557
:10F54800C874491AB9A2D80A19522481A98A8C9C6C
:10F55800B0834410380399DBBC9B38386483108A25
:10F568008D9B89B1E0D626188C8980B0A0187221AD
:10F5780008A9A8BC9C893424121930ABDCBA98239A
:10F5880011713101B8E8AC8A0A3F0763ABE8210B77
:10F59800A1250099A9101B9116080A8C0808923415
:10F5A800180D9888A093613C0B84B2C8A2488F17A5
:10F5B80070BBC1218B015280B9A8008B015591996C
:10F5C800890A18838680BA0A39012594A98F1818E0
:10F5D800B2B693FA644BBE8210A921401AA9B18031
:10F5E800AA227108A0A2B81C3013A0C998311B87A1
:10F5F80022D0B9195C190186F1372DAC1110B0145D
:10F60800200B9C8188A014382A98C1B10809413977
:10F61800F982010D412BA0E191091A315FA554BB74
:10F62800E8211B912501AA9A190A9126100A088C2B
:10F63800918288121DA08311E4211E8B02A2A918B1
:10F64800604F8471CAC1219A104200B9B9188C015F
:10F6580043019A0A0F289181288D8A3200A416AB9B
:10F668009B0920C3C503EB743EAA148AC0520B88B9
:10F6780022AAD82219A81500C982289B8313CC185E
:10F68800310C8428B9AA231D882698F2669D9941D1
:10F698009AB3529B0020ADA2210A905189BA13292E
:10F6A800CB422AD9122A092139EB95881B18592FE0
:10F6B800A733FAA248AC0421B9822AAC9233AB82B0
:10F6C800518C9A338AD1133F980308A84019BB0379
:10F6D80018E882508E0368C98309BC2238B1152006
:10F6E800CB810BC993141918749AD821AC985188F6
:10F6F80080339D8A3809D1A79998535BAB358BE83D
:10F70800121A803480BA102EA881229903718CA213
:10F7180011DB92488A0335B9094B0BC2949BD35726
:10F728008A9A608CA1120B005189A0109E888211C0
:10F73800A00538AD021AF80119894308A99218BD25
:10F7480080209F0612B9A2598F81018992518AA1FE
:10F7580011C9988060B92719B8221E990390893178
:10F7680079998391DA003B996268BA841ABF1110BB
:10F77800A814288D8118D888024B904799A1010DAB
:10F78800A1119881233C8D382AE0821BB3543C9BFD
:10F798002699D91318C00600AA111ABAA243AE8333
:10F7A80043BC005B8D01188883201C9886B1D8283B
:10F7B8001BA705999A419BD8322AA8520AC0129BC6
:10F7C8008E0034AA8539AC300BC0834C181395B021
:10F7D800983B1F98082A0734A9C048BE92038B0299
:10F7E800618A8011E9991021B10719C8111BAB274B
:10F7F80089910339DA93009E08590B3170D8931A0E
:10F80800BC0420BC2331AB8369D9A283998A731ABB
:10F81800C205AA8A2890C315181A2A29FBA311D849
:10F82800624BAA258AE91308B02510BA218E98A23E
:10F8380011081B639BB582AE982001B1440B0A14D2
:10F848008CE01089C3370B98509AD0239C93418839
:10F85800B103BBBD312A8007288C201AF0B3882B4E
:10F868004140A1A2C1D8A92B798435BAB1699D823A
:10F87800119983488A9883D00B1050B9232B7FFFA6
:10F888007FFFF35700CBA981421200939ADCC9127B
:10F898002410088980D9A8143298BB818300837802
:10F8A800899DA8A842802F25730AFC980230210858
:10F8B80002ACCBC0132508880809D890132099E812
:10F8C80081120202909EBB89961296E943601EBA85
:10F8D800901321220949ACCCA132339088081F9893
:10F8E8009112209CA8032822B6A1C9BA81A7008337
:10F8F800F207509F9A811211101818CDAB8142302F
:10F908008808809C9D210319B8AB43852A388CBA96
:10F91800C88040197C141711FAA901212202939971
:10F92800ECAA112428888110CAB931239E89B340D2
:10F938001499789A9C829039A17F306289F9A8112C
:10F94800212828019AEBB923368808001BAAB2158A
:10F9580004BAA9223005A40A9BF9081200C7D041AD
:10F96800780CAAA11222202A399FBBA13262988959
:10F97800108C0B813328E99A12382824AA9EC00BD0
:10F98800482924F487109F9A812112001019CDAAC2
:10F99800813250809181BB8D113129C9882102792A
:10F9A8001889BCA091582D5E841700DA9A0221228A
:10F9B800810088FBAB123518888108D1B820328CB9
:10F9C800ABA26011281AA9F980B32104AF483241CB
:10F9D800B9FBAA9952420011219BFBBC99225222E1
:10F9E8001380B8D9F998812042228099A9AC9AC885
:10F9F800E1B43273588ADAB98811512320318DCC99
:10FA0800C9A0824231210099AFABC88031612182FF
:10FA1800098D9C9B8A15C485332AADBBBB941341C1
:10FA280015220A0CBF9A9011413112818C8F9AA924
:10FA380081235122029AAABFB9BA3B264724999C2E
:10FA4800AC98011322224101CCDB9A9104341211A3
:10FA580082BBCF9998020335110119CAC9C9B90ED9
:10FA680070422199CCAA9921332252308BADFAA940
:10FA7800011243132881BBFCA9810123242219A860
:10FA8800AFB8E8A2B23377288ACAB99130312512C3
:10FA980020ABBFACB82140412128999BFBAB113268
:10FAA8004415808A0A8DB8A098C7152229ADBAC90D
:10FAB8008113222623198FAABAA10242324121A911
:10FAC800CFA999A2123631190AABDABA802A07628D
:10FAD8002219CDAA8A00150221231ADB9CB8909519
:10FAE800211124598989E9A889124133608A8B9B9D
:10FAF800E0C00A30734289CBCAA938333253318CFB
:10FB0800CBCBBC1014331161A892F9AB81049325B7
:10FB1800183AC98BB8F181A0417220ABDAAA9005D6
:10FB28003023214C1C8BD9A812207011108A1ABAC4
:10FB3800F9880051229493BA8E88AD10B69434197E
:10FB48008DB9A9920410412400C9CC99A0825148CA
:10FB58002108989F98BA1023682848099ABA0F8AEA
:10FB68003A8527148A8D8B98200321422109D8DBF6
:10FB7800AC8212070110091ACB8C9809351385102D
:10FB88000D0C90ABA02A713433A9FAC9891016025A
:10FB9800011088C9F8998220320481089F98AA8B9D
:10FBA80022268384188ABAC0E0A2A143733899FA3E
:10FBB800B99830412411208CBCD8A91121710018A2
:10FBC800819CB9D9A39152111418CA8C8B8C18C571
:10FBD80086322A8DC9A9810221432688AABDA9B1E6
:10FBE8000420503010A1DBA9C980327030208899D8
:10FBF800DE1B0A3A971522899FA98902840220519F
:10FC080089ABE99B0113060021190D9BBB8A807201
:10FC18002203498B8BC9F8B93A6126210BDAB27FE6
:10FC28007FFFF77788ABBA9004232402118BDDCAD3
:10FC3800A9823533202888BBFACAA8134334201870
:10FC48008ACACBCA988B62752199ADBA89032224D6
:10FC580023310BCFBBB9822533222008BBFCAB9ADA
:10FC680012460302088ABADBAA91D143744899BDA7
:10FC7800A9882121413131A9FCAAA91134412111B6
:10FC880009BBFBAB90034513210099E9BBB9B1F35C
:10FC98001742299ADBAA8022413241289CDBCB906B
:10FCA80011433322100BAFDBAA802336222810BA67
:10FCB800DACA9A1C036524019BDCAA902434121822
:10FCC80099ABCBAC988345342299ABBCBCA89216AF
:10FCD8002333381CADAAC9998A337641009CBE9A51
:10FCE80000234321098BACBACAA80444422189BB2A
:10FCF800DAC99800342513109B8DBBC980983752F8
:10FD08004108AECA9A11344201099ABBBBBC983467
:10FD18007232219ABCCBBA981336333418AC9CBBD8
:10FD2800AA809073524028ADCBC998243532000C74
:10FD3800ADABA88124523010AABCD89988023512DC
:10FD480023008CCB9CBB090425721118AEBD9A0008
:10FD580023623208ABDBBBA803542411089ABCBB4E
:10FD6800B988162422320B9BEADA90982274320062
:10FD7800ADBDA9921362100098BABBCA8A21543447
:10FD880022099BDBCAB980532433308CBADBBC010F
:10FD98009187525088ACCAA902353221999ABAEA99
:10FDA800A89A2273331199BDBCBB98042345312905
:10FDB8008CACB9C988083762280ABDBCA81344129C
:10FDC800100A9CB8BAC8A2353522109BBD9C9998D8
:10FDD800233433422B8CCBE98A2B214725019BDA2C
:10FDE800BB912426120099AB9ACBBA03723242080F
:10FDF800AADACA899017841118088CAB9B9998269F
:10FE08004541189BFBA991343233088BBE9BAC9AB1
:10FE18002155231109AAE9CA980132621380A1BCAD
:10FE2800E99898B22672209ACBBA983331433312A4
:10FE3800ABFDBBB01224317932D4AA8BC0A1012208
:10FE4800421396C88C09D2A88307321B8BCCA09288
:10FE58001858402300AACDBAA8582322580188ACC4
:10FE6800DAB98821436011189ABABF991D2137233E
:10FE7800899CCBA902033341350A8DADA99184220F
:10FE880041011899CACE8A01221343101A8CBEB9AF
:10FE9800AAAF43742ADAA80228201011AAEBB023CB
:10FEA800440098899AD99244118AC89019882242A4
:10FEB80012CF991803D2F953600EAA80121111209B
:10FEC8001ACCBAB134410809080DA9813428BBAA53
:10FED8008583030933E0FA8821195CF30720AEA96A
:10FEE800002211020299DC9C0203200088198F8AE3
:10FEF800103381CD0A2103810A688ACC08212B4F4F
:10FF0800A54410FAA88131111182AADC9A83242809
:10FF1800018188E99882338ADA88510190122D2D5F
:10FF2800A99059298F54599CC128BA037289918183
:10FF3800CBB0510991349AA9120BC0132BAE0221F0
:10FF4800810828D8B880B0C787E8423C8D930AB8A2
:10FF580025588A0019BCA3318A8431BBB052AAA2A1
:10FF680013ABF8331A18132BCD0818AB2369F357C2
:10FF780089CB138CA12710A9182CAB85180A123825
:10FF8800CA8138AB3049AD92229A48338BF9883907
:10FF98009B687E0408B4B81AC140A22298C11BCA43
:10FFA800609010009921D8128A9248EA221A930484
:10FFB800A008AA93C0E483AF702E01A19A924A02C6
:10FFC80031A9D3A9E139910388B038E00198933A6F
:10FFD800F9310D0310B893C892A3D4A7F0508C3A06
:10FFE80008AB160A212A0C10AAB60A021189A33DE9
:08FFF800A0011B001CB5299AB1
:020000040801F1
:1000000071898099AA5089101CF731F81908C82401
:100010009812099A3C9C32AA33399C158C882099F5
:10002000039E0308A4298B48ABA32B93720F850A68
:10003000A7A910A818B509814098029DA11DA23A50
:100040000441B833EA90A901A2332B8719C829D8F3
:100050001119AF780B50A10AC11C039081429E1365
:10006000AB828F108805808291D2A1C920A835C1AA
:100070002299B239CB20B1F279087B828B938D2102
:10008000000832AB04BC01E920083300935BAC8C60
:10009000903C9502932A19B6BA94D881F680931DA4
:1000A00011AB11AA203A1279803AD92BB3198639AB
:1000B0008215CA881D010A185901282C08897D89D2
:1000C0002E2491A5A938D818B120800608918AD08D
:1000D0000B8288171B0239B92ACF01800598202886
:1000E000A888B89DC28F781B51D108A83B92000107
:1000F000129296BC089E110013991519A989E93826
:10010000D328A349B9862BA098B7F149095A910B76
:10011000828C200A234A0A21FA20C9208058911390
:100120009A81CDB30BA422B4392B20D909DA13F666
:1001300001B41E12AB11C93190151A003BF829B851
:100140002884491922A989CE018C142902092A3B45
:10015000E94ABD5B1580A7A818B938D2108013985A
:10016000802F900D9218141B1048A9B2BF01A8222D
:10017000185489A119C12CD18F792A30C11AA01C19
:10018000831A0152A0A4AD83AC820024B1024C0AB0
:1001900080D089B2429241B0A48E828BD4E1392BB7
:1001A00079910C829C2288203A8829EA10BD310975
:1001B0007090118A800BF0199340803C0A33E882DA
:1001C000AC01F680822E02AA02D831A0212A192B76
:1001D000F928C03881598121B9890F909A8618056C
:1001E000898839C939BF4D148897A928A829B3002F
:1001F000A31588882F902CB400830A1239C800CD2B
:10020000119A40001798920AD209C83F680921D173
:100210001A982D83088222B893AF93AC02808790FE
:100220000209A089E819A311A37088A48AC3ABC7E7
:10023000C049197A818A918C3109113B2911FA211F
:10024000CB308142B0158B088CD11A8140845A89F9
:1002500083CA20AE02F481933F01AA02C830801104
:100260002A183FB02AD038943A0941BB2A0F918905
:10027000031115890A59C94A9E3D1591A79918A9D4
:1002800020C110821390810FB20DA328840B125845
:10029000A981BC02C81101529B08007FF7F208B780
:1002A00092D03C398080808080808087F1083E7ABF
:1002B0008F380080808087FF7E59802D1080B6980F
:1002C0000A7B2A1808082D12C8492D03A922B083D9
:1002D000F19282A808C79A201A083F84993C398075
:1002E0008080808D79808A5980A5982AA5C28A59F4
:1002F000808082D849A498008800880800F7D38AB3
:10030000193908800B691C2883E108083E101C4B32
:1003100084989120D10808083F10808080C69808F2
:100320000808008800F69802D101C10A50E4A01A1A
:100330001911A00B69808083F12C1939808080808D
:100340008080808087BD3C7980808A6980808080C1
:100350008088E34B0808D7980802E3D21908802D5B
:10036000108083E3B1083E84980007F2808087F70D
:10037000A5F194A08080808B790808B7982C12C1D1
:1003800002F200B3D3995B180808080800880088B7
:100390000F791E3901B1008800C60C10A498A598E9
:1003A00008080B7B30C108083F108082D288002EDD
:1003B00010808080808D798080803BC6B102D1081A
:1003C000083E108A598080B78B4B39A2808080808C
:1003D0005B8C30800880F7B10A5A9489A208A33C4C
:1003E0003F3D390808080808B790808800880080D9
:1003F0008807F12F4B3992A11980808B43C084BBB1
:100400007D392A9048C2808088003F3A0803F84925
:10041000893C5B1808080803F108A7B2B21908085C
:1004200083E1207F2808080F77F1800880088E3448
:10043000B08C798080808B70C03AA59808A338F37F
:10044000A0A23BB7980808084E10808A6A0A23B316
:10045000F10802D1912A080C691E39939080808896
:10046000008800887F10082D102D84B5B180808011
:1004700083E1080802E10808A698A23BB70C3B10EC
:100480008080808086E108080808080808F7980836
:1004900008A6A0A23BB79808083E10802E1080083E
:1004A000800880088007F194A08A6982C108A59815
:1004B00094A02D1082D3B28A591A928080808087AE
:1004C000E108080803F3AA32B0088008807F5B2B9C
:1004D0002808080B7980A4980B69808080B798A2BF
:1004E0002A02E10A59A491C03A083BB7B2A4B1026A
:1004F000A8B798080808080D7980808080C69808F9
:10050000080804F108082D10A50C108A238E10820B
:10051000AD5993980088A79808A5B39808088B79D7
:100520000B69808080B798A5980808A50F3901B19C
:1005300001C28A5980802E1080808A691AA068B210
:100540002E0182A0803F19398A7D3993B3B12A08E0
:100550003F108082D2808088008C7B10803F10808A
:100560008080808080E6980A5A2C03A083E194A0C2
:10057000800884E03A08A7B108082AB06980808022
:10058000C69808A6B3A0A7B2C48A1080808088034A
:10059000F84980808080C6982F39082C1080A7B138
:1005A000807AFF79F7980808A6B5A9180A5980A299
:1005B0002B00808800F698080B33B84F108A5980BA
:1005C0002D3C39A22F3908080808B42B08080E6002
:1005D000C101C03C49A6A9101B822D398082AE30D2
:1005E0001A008B798083BB304F10A40C193980809E
:1005F00080C78B21C282AB3084F10808A69808809E
:100600000803F3C8491D3995B11B8491B1080B79D2
:1006100080A4B4A083E101B4C1949A49801C1083E2
:10062000E108082D282AA2080C7B10A498A5980898
:10063000080B70C1080A5A0808080088C7980A5BA6
:100640004A2AA5B3C28080B6980A5A0800884E107C
:1006500080808080C7982C1080808B7982AD50B1CB
:1006600008948B2A5A02D3B1080803F849A49808C1
:100670000808B7982AA3B69A40F39081B28080B751
:10068000B12C194A001F39080808080084F03A08FC
:100690002D2880A5B4A94A0A22A808008D34B08864
:1006A000006F848C39008808008C79A6C2901908E4
:1006B0000808A5B21A0B33F3982F3A29082D1949C7
:1006C00080A22B03F108A7B11B2883E3D21991194B
:1006D000808A384B84E108A5B4B3A083E1080A5AA4
:1006E00094982D1080088008805F03C3B392D3C014
:1006F0003C12A2F390893980803F84B3982D21A9C0
:100700001008800D6980A5A08008800880D791C25C
:100710001C3D49808001C1949889283BC69894A0CB
:1007200002E10894A0088A384BC798939A5A0800A7
:10073000884F3993A08A698808A69894A08A59821C
:10074000C1083E3B194A08A69A498912AA33C08CAF
:1007500079A4993C30C10A498A59894A0808A6985F
:100760000B6B39808080C33F3A2E30B108922B0842
:100770000808080808F792F3980912AA7AA4908941
:100780004B3A0802E2883F3980A498924E2A180A10
:100790004980800880C78C3909120F119080800829
:1007A00008C7B3980802E10A23BB7980808A68D41D
:1007B0009801B288008B79808080808080E303C0BC
:1007C0008C34E398A59802D10A4980B69808A7B15D
:1007D00093A00B32A880C79808A6B5B0093C3B4946
:1007E000A282AB78B21C280808B7989282AB7B39FA
:1007F000808A7D3991082C3B39A5A2C194A0A5B36C
:100800009A49A4B4A02D1080808080808080808F41
:10081000798080C69A22A8A204F12A080B698080F8
:100820008A6A0088008C33B8C79808A7B19102A2E1
:10083000E12C194A008800880C79894A94A008089C
:10084000B304B804F84B39A4B12D498082D03A944E
:10085000A0800B37F20A029895B84B182C10808AAA
:100860005B4B3A0800880C79A49A40C013F2A28925
:1008700011A0A202A80885BF32A8080B34BC6B4A9D
:1008800000A4C398002E108083E194A0A2083F1218
:10089000A0808088B43B80880087F3980808080807
:1008A000080F69A4980808B79A4993AA59A7C2885B
:1008B00008089398A32E1077FFFF1678829B8C4B25
:1008C0004991850A0843AAF901008816B2C1A050CF
:1008D0002C9881C10B2912278813F8AAA2884222DA
:1008E000C2918C3D0988D0301078818C00A1AE0A6D
:1008F0002917138880CE092B12228A0F301184BA4F
:100900009B0B18C525289A09AB3DA182D418440930
:10091000B4CB902013D001B0A49D104221D5C98042
:10092000C210E310820D288D083B11D0138080B2D5
:100930009798AF2029B2D588883B041D929903016E
:100940000CF1200198809A482B78AB13A50BD0337B
:1009500090B2205CCC231A098491F38A6A99408969
:10096000B1130D921898004C31F811A2A8020F2172
:1009700009A023B980500CD208FFFFFFFF74339BFE
:10098000BCB9CB9C106233128809BDDBBA013315A8
:100990002350289BDABB9B901F376380CB1A99901A
:1009A000B0442332999D99C9D9084232210019AD2A
:1009B000DBAA812135142218BCBBBAD8A1CA763271
:1009C00020D9AD9A101222123211AECCBA90135225
:1009D0002221109BBDBFA90023422111199CCBBB32
:1009E000D880E373321ACAEAA8102231243118DC05
:1009F000BCAA9014334221880BCCDBB901344222CB
:100A00002189BDAD9B990CA754210BBBEA90112302
:100A10002043210AFACB9A01343323102AAEBDBBFE
:100A2000B013452212209BCBDAAB980E3744008BD3
:100A30009DBA8102331252208BDCCAB801343332A2
:100A4000200ABCECBB9013442312289BDADABA913B
:100A5000BA774110AAAE9A0102221323209EBEB992
:100A6000A811424221000ABDBDBA80235233130AA5
:100A70009BEBBCB980F2635108BACC9910124013B9
:100A80003208BEBE9A8012333411109BCCCCA9819F
:100A9000335231218A9CBDBC991B9764200AABEA72
:100AA0009001222142211ADBEAAA002343322208C4
:100AB000ADBEBBA802363131389ACBBCBDA81D36BD
:100AC00044208C9CB99101340233200CDBDAB8113C
:100AD000333433111ABDDCBB9022443221188BBE53
:100AE000BBCA91BA773318ABBFA9001141023211CA
:100AF000ADCCAAA002432332210BEAEBB9903253CA
:100B000023221A9CCBCBC980C4635118C9CAA9102F
:100B10001340241208ADBDAA902242333111AAEC31
:100B2000CAB9822362311109ACBCCBA91AB773319F
:100B30008ABBFA90003221342109EADAAA00234361
:100B4000232119ACCDCAA8022531232899CBCBCBC0
:100B5000980F3544118C9CB99101331352208BEBC3
:100B6000CAB9113433421109BDAEBA9813353231C6
:100B7000009BCCBCC9919B754300ABBEAA0013324D
:100B80000433009DCCC9A0023422212089CCCCB9E9
:100B9000902353321208ADACACAA80E3636108B96C
:100BA000CC98001321152108ACCCAA902234421114
:100BB0001099CCCCA9002433222109AEACAD980AFF
:100BC0009744210ABBF99810221133311AEBEAAA93
:100BD000002343322118BDBDCAA903253232209A11
:100BE000CBCBCCA81C3744208BADBA910233126218
:100BF000208ADBDAB8103343330219CCCDAB901224
:100C00003621220099CBDABA91AB773318ABBFA962
:100C10000003220432109DCA07FF4FF582EAE90A59
:100C20007718B88A0AB0168120893599AB0CAE00C6
:100C3000027838C7D3892D1911C3881A82928888FF
:100C400093892F290987198800A9B2938B313978A4
:100C500035BBC0A2B0A883718944ABA992A93873EF
:100C6000D0A2B338184EA89DD827718BBA820088BD
:100C7000213A14618BFA800080122020202BEABBDD
:100C800091BA0711433801CCC888889C0096572137
:100C90009EA900888021210362ADBA811AAA43105F
:100CA00032133CFB08B81A9152034008ACA98AD908
:100CB0009882377718BBB911998242113431CFB875
:100CC000808889334012228CDC8898880241404019
:100CD00089ABA9A0F9919965721ADA9818888230BF
:100CE000025329DDA8009A8223303610ABDB0A0AB2
:100CF000A2871130300CC9998B8B98F067610BDAA1
:100D000090101082122231AEEAA81110013331295D
:100D10009CBFB9911121342321BAFCA9008890000D
:100D20001777109DBA81110822222419AFD990019A
:100D30001002322288BDCBAA9022513241288DCB9D
:100D4000A8880A8149566508BF990100002031131F
:100D50000ADDBA81101023522809CBBCAA80126187
:100D6000234188AEAA99080A1292776209FAA8115B
:100D700000011222220CECA90100012423109ACCBC
:100D8000CA98101314334299DBCA88090910867572
:100D9000500CDA90201883032231AFCBA810110237
:100DA0004331088EABD8908023334320ACEBA900AD
:100DB0001990200776209FB981101812221218CDA1
:100DC000DA901010124221899CCBBA0101612315DF
:100DD000098BDAA91989933A757408BFA9020080B2
:100DE0002231228ADEB98011181432280ABCCCA91B
:100DF0008022337112899DAB99808A208476718814
:100E0000FF7F7F39FB73F48F4B3B14F4B1094E5BCA
:100E100002C4C21D5C3A96D3891A5B85C292A84C63
:100E2000108883C11B3B6B109801983B00093AB7AF
:100E3000A97B1920E49929190092A1901A20C49243
:100E4000D15F28B5A1883F4A82A1800A28888109FC
:100E5000298D7A01B5D3981B6A0081B6B8280B5941
:100E6000B690910B30C3A181A298815F39B318D499
:100E70000E4A0884E59B5B4C12D4B28B7D38B7E6F2
:100E8000C86F59B5C6E22D282D3981A4B03A8829FA
:100E9000A48C17D13D2800C6C03C2982B4B03C20A8
:100EA000B28082D21E5B20B4B3B21E280A30F30B8C
:100EB0004B2A13F21D5AA4994C4C14F7C96F6AB708
:100EC000F69C7F58D7E4A97F6B82B4B20C5B298271
:100ED000A2A82C49883B969D6A93C4D5A94C5C1066
:100EE000A5D48D7E33F6F40C6F34F6C04E7E15F526
:100EF0009C7E38B6B97F41E7D04E7D97F7CA7F7B9D
:100F0000C7E31D5D5BA7C97D02A2D32F6AB6D4A833
:100F10003D39A5B1818C7C002C04D200A22E281D65
:100F20005B95C2881B23F3A2A02AB79C7BB6A1C401
:100F30000E7C94A0913F30C4C38A4C12C290896C3D
:100F400013E4A1894E32F6B1A14F48A3C5D31E5B6D
:100F500001A4C22E498802D12B86C1803F5B10A616
:100F6000E4A84C39B7D49A7F59A5C20C282C21D1BA
:100F70004B921C129C32F389003C96C2918A5A957E
:100F8000B181A84B028A06E12A08190193F38C4B20
:100F90004B86D2882C4A82A1901A39A3A0094F49C6
:100FA00093B4B11E38B31C13D10A4C30E390910BAB
:100FB00050B03AB68C24E22B822F04B0018C49A5A4
:100FC000B3C30E6C0290D6AD7B8813F49C5C4B03CC
:100FD000F59A292D31F41D200997CA7C83A1C6AB4F
:100FE00069B32C839A129E40C4B20E7D85C1810DD7
:100FF00048C30B97C12B3D49C6B84D5C04D21B4C6E
:1010000030D6C82A4C22F59A293AC7BA7D12C4C2F2
:101010002F7D04D3A39E7D0280C59B5A802AB7A84A
:1010200039A04AA23F21B822F12B2918938D391CEF
:101030005B2903F38C388A40F69A182F41F50C2966
:101040003C05E22B2A13F30F6A0893C20A02B05C34
:10105000109182B96C20A84B85B10A5D3994B29881
:101060001A5C1092B6B84A0802F59C49088077F7D6
:10107000F7F921B6B7F490982980A3822F5E4B2808
:101080009192982D5B3B01A3AA7D4A1892A291B43C
:10109000B4B3B3B4C3B1092C38092F5C4B2A290966
:1010A0001883B1883B02F4B2982A97C3B398189278
:1010B000A2A93901A5D2A5B3C3B2B480A1C7A3B870
:1010C0002B6B2B04A3F2801998028A891932F11331
:1010D000B99A495D002A02B2C5A86C2A1093D02A99
:1010E0003C1910891985A6A1B181B2B7B12A19821C
:1010F000F6A2B29000AA400E4B5A2B0002A91A6B1E
:101100003E3A2900802C2E5C3A1984A0881A21A12D
:10111000A28F3A4980C395A1C292A191B8580B13EE
:10112000E6A0B395E3C2801C3B3992C39109A6C3E4
:10113000981A28A4B12D4B39928B4C6B29182C800E
:1011400094C5A81928A6C4A08809109193882D8356
:10115000C5C3B2891C4A11B5C4B1A4A2A1B3A4A04D
:10116000A2281F2B5988093B7C10A3B4A11F3B392F
:1011700082B2893C39818A2802D2B789910A1A87BA
:10118000A3E3A1895B2B1828A82C61C0821B2F29FF
:101190002098A1183F3908B20C7B5C18180A02800D
:1011A000B390A5B4B28C4801F1B4081A188C023A75
:1011B0005D2C391B1A6B3901B6B0191B40B81A984F
:1011C00070A302C0FFFF6F7E1982C7C21A1B49823B
:1011D000C1912D30B2C2913B60E281A90A590181CF
:1011E00080A20D1C7980C2084D2801B18931B93324
:1011F000CC07B3A88128A3F3B299290033F0922F2A
:101200001903C3C00B7A80180882B82D4C49928A02
:101210005C4C1000A82808881B7A01D4981A12C5C3
:10122000D388098292C010089299288A23AF3F3848
:101230008192A5AB23A8E388A5A2E49088A5A4C1C8
:10124000800891080C14A8A14D389002AC4E4A19A0
:1012500018029A3C4D2883D10A3B30C4B28199824E
:1012600083E0B79082A931D3E49809109194A91929
:101270001028C109499E591980312F984A2B11B75E
:10128000AA4B5A9010A299040D84A4C0081A08967B
:10129000990039A1B23F4C20B3A028A106E00082FA
:1012A000C1812A81F5A00818900399B62BA087B1B7
:1012B000B21929B6C4980929180C86C3892C11982B
:1012C0001B3C28B6893D3993C29D6A198292AA13A4
:1012D0009A860D1198C789091083D0020F101890B3
:1012E00080818C4C39A6A20C3B389B495C18180AAB
:1012F0001A41C2A0805C02C5C3A8292B180803D1DB
:10130000997A2C03C10B6A00829A2A49C2018D2066
:1013100083F18029A2A4C0081C1124BD3A3A991374
:10132000B3E0297C1912B1C4901B12C6C2089119EE
:10133000B05B2801918A2F4A2B14A0A18813C3E126
:10134000A2C33991B5909B9078AB528BD25A8092C0
:10135000C32F1080981082A9E428A1C086A0809A8B
:10136000239095B598984AD3B5895C0001B12B3B81
:1013700019A5920F0101900B7C0280A8120D8068C4
:10138000B2892B5D3A00986A2B3A1A2D3894D03CDA
:101390004A00B6A0808080B58880092A1E22A3F169
:1013A000802C3B09588C013C1C4903E0280A10A002
:1013B00086A1C30A1C42B881818880F3904A8903C0
:1013C0005B0B01C68C291194C0029A921D28E592EC
:1013D00099109819B4A6C20E3A2993A298811809B7
:1013E0003F099790893D30B3A1092F841C916A80F1
:1013F0001A195C292B2B3D210A013F181A0A5A2B76
:101400004A1A10A688D212E0008812F100A4A2B2F3
:10141000A002D3C591C1000B03A8810A4893A0E2A2
:101420001D2B5A4A9309A97A0895A9922B390C3990
:101430005C004D11A2D3893D2A04A00C591A8202E6
:10144000BD2811C40C3818D21A08A7A1A21AA010DE
:101450003B0C58B308C3B19B7C5A000B493F193C65
:101460001081B2190C6998100C319A1B358CC6800A
:10147000B3A3D1299016D19180800090914A4F2832
:1014800091818B3928C30A037AE283C02B8083B40D
:10149000A12F499895AA3A4B0F77F708FF7C15C002
:1014A0001A6C10A5B02C4A10A3A08A3928D3B21800
:1014B00090B4B79090A6A3B93C5910D0821B2B3A98
:1014C00033F18B7A18B2000F4908090081890A4864
:1014D00081E5B5B00911D39082B4993B2C04C5C302
:1014E000B04D3A009280900A29A4885C282C29905B
:1014F000884B2B48B49A3B6199092B9913B5A05F8F
:101500003A289B040BA491C690986C4A1B12A00029
:10151000A804C191290F4A3B1A2A2D0103B39894BC
:10152000D4A1B014B94C2A12F5B29290A39C22C453
:10153000D3895B1983D3C1080A2839194AB03F2BD4
:101540007B2A28199018A7B2D481C181908888314C
:10155000B1F5C4B3A8290801A8081B06C083AA10C6
:10156000301F2901A83C4F3B5A0A5A2B1083E4989C
:101570000A3929B2008F491903D3C2089181092B76
:101580001E2A3E4C391880804C1B0109A3A7C4B405
:10159000B1093A90819C6A1895E4A19192C2901B7E
:1015A0004A181A3D2B30A28D7B4B29080008A5C490
:1015B000A0A3B4B3995C4B390993A8A021914B9295
:1015C0002C2F7C3B180018893B3E391B02E3E49129
:1015D000A1089101C3D4B2A0829193B5A3F2A10C4A
:1015E0001930B2882A38B17B9086C10A3C4A84B34C
:1015F0009B4B5A0881188B1887A1932D2F1082C2FC
:10160000082E4B289000A21C03C3C3A12B7E182ACE
:101610008000893B3F5A1A095A2A19818983C7D009
:10162000FFF77F7F7B97F5C12C4B02D4B3B02B3CE7
:1016300038D7E6D21E7E38B6D4993D4C3982C29056
:101640002B2A1892E5C3B2092C3B12F3C4A82C280C
:1016500095C3983E4B02C3A080093E5B11C4A02DE8
:101660004B11C3982A00810C5A83E5C3A02D3984FD
:10167000D5C3993E4B11C5C38B6D5C20B5B20C5DD3
:101680005B11D5E6B84D5B03E5C11A2A1882C4A1E7
:10169000893E4A0080892880893F4A0092B11B4BCD
:1016A00002E5B288090911D11A1A2A03AA101BF3FC
:1016B0000AA22C814AF4A1A97A0800A4A0A48980D6
:1016C0002C012BA70A0921B6C2894B21F4B3918BB7
:1016D0004A28B6B4A83B5C11B3A21E5B2982C39012
:1016E0001C4A28B5A0082B4A008082A2C489094060
:1016F000B4D21A081880100B21984E5B1888A3B832
:101700004B193C04A2A02B11C0C681A94B8985A905
:10171000888A00A959C3094D180082BA0F1981B3EC
:101720000F1B7992900A49C023F018890290E200B9
:101730009A7A0894B0985E281993A19A2918B389C7
:10174000905B0133C8B69F388A03B1A30A905B93BC
:10175000A2F13B9923B3B16AA153CD6A282AA39879
:10176000A8944B48E2B5891A3800B319A7C01829C4
:101770009A8A26A0811C4B190911B1027A3AC83CF9
:1017800021709A282F8180B1992E3A3882993C3F56
:10179000A2A1B783808C8293F0022B086A8911A2E0
:1017A000AC384F1101908818D216B1904922C981E6
:1017B0008A8418A3179829D86AB4198A59089229D3
:1017C000A099123CE00589C319C882B0192A4D3A84
:1017D0000A94960A013D93C3E0891B8182C128B90E
:1017E0004980808781F11C309893D8110A1F10C658
:1017F00090892C193D829191085B9A9292C2195B53
:10180000B869A0B298080A79A3D1A70C193B0811AE
:10181000C1903A8B0A82A794C9593A89B58C9259DA
:101820000C01840A1B38051983C9212C791A988167
:101830002B7B1311FFFFF66771AF8A0011B4804252
:10184000298EA991A10B505030B8B9B18C19806282
:101850001109A0290E8D081128884F8614A2F98934
:10186000182A0285228B0F890892A023504A98A932
:1018700092CA090252020A190C3EB900048923AF28
:10188000785089F0A1801A201423B8CD891A10B39A
:1018900027030A8B8B18C98A1451209981A89DC9E6
:1018A00001179081F248691F888082982832399800
:1018B000F990892A014325A9999A3CA0C1151129BB
:1018C0009838B1CDB01850882AF70381BF8A00112B
:1018D000B481421B0CC892B10C315131C8A8B10D72
:1018E00088A0440118910989EB00914A106F1405F2
:1018F000A2F889082A0383348A0F990892A8333200
:1019000069989A92DA9882521389800C1DC9000452
:101910001B12AF784809F0A1810A300422B0CD88AB
:101920001B28A225140B899A18F09083482198103F
:10193000B98FA00835B184F1306A3F90A182A039F7
:101940004220B1F990892B032425A989A81BC8A995
:10195000353148A118B0DD908030084BF70480AFD6
:101960001A0810B301512B0BD891B10B336040A969
:1019700098918E888834012A001B91FB08016A1017
:101980002F1504A2FA09182A0395139A1F99189281
:10199000B014214A989A93DA0A0061020A110A3EA9
:1019A000C981921B329F71580AF0A0810A31052229
:1019B000B0CC890A10B344132D889A19D8098333FF
:1019C00023B012F898FFFFFFFF6A2F682AD6C48A57
:1019D0008B699094A20A2959A093A09B385B9383AA
:1019E000A19A588AA3890C1961B284898993F3FA60
:1019F000783F2094C1B15C1A21B5A0813D1901A2A4
:101A0000C0100C2812A2C1190D2090A1823B906039
:101A1000A808A2AAF712CE7C4998B7998A5910A1B2
:101A20008499092A08C3819B593808A498AA4A8036
:101A300008852B9140989D297F9792D3895C1B1430
:101A4000C1A21A5A8012C0800A2C0101D2802A3CFD
:101A50001298B28A108B270B020900BB788F31785D
:101A6000E3D3099C3802B4C42A0C2891B8B259199E
:101A70002015B1A08B0C0902A2250041A9A89AAD9E
:101A8000D285F8783C1995A0D83A3A10A700A82A30
:101A90001AA9B6800938589191A8AC8810A23402CE
:101AA00058A888AABF9111F3271B3F1088E18839F5
:101AB0004B139291BC1B1C01B584002B1008E8A8A5
:101AC00080090341222AA8A9DBBF085E8604B2ABC5
:101AD0005A1BA2C4820B581090C0988B2A132692CE
:101AE00088391D9AC092992433128B199BF9C90029
:101AF0001F5151B4F1088D298283B2283A2CC0A11C
:101B0000C00A404002A2809E8B9081983362119857
:101B1000A8ABBCE885D9705A2AB4A1C92C3821C514
:101B200081880C0988A2A03169208191CB9B080192
:101B3000B4334140A8B0C9ADB803F6051B5E1088A8
:101B4000D298283B2393A2DB1A0C00B503183B2044
:101B500000FA9A08199513237777FF0D17358D989A
:101B6000AA305B2F46A1E2885C8914D0083009B501
:101B700009AA2801B8035D0112A09B38BAF2102906
:101B80000021E0842C90A1B8DB751A94C39C0A68EC
:101B9000A2A2182E0490A81A19B2148B4810A1B151
:101BA0004B9B84B29B4160A010AD0902A1F2788CDE
:101BB0004895C8803D0094829C4089B2881B0023D0
:101BC000E0113990C39B9C309296011B80299B3B6E
:101BD0000CAFF700984B38E0938C391282F0388BB9
:101BE00002A1AA8068A3110B0A83C8C06A0081926F
:101BF0001A141CB81B992F3710E3996C8803D0086E
